:020000040800F2
:100000000000012091460008052800080728000884
:10001000092800080B2800080D280008000000002F
:100020000000000000000000000000000F28000891
:1000300011280008000000001328000815280008F7
:10004000E1460008E146000819280008E1460008DA
:10005000E1460008E1460008252800082B28000892
:10006000E1460008E14600085D280008E146000876
:1000700031280008332800083528000841280008E6
:100080004D28000859280008E1460008E14600080C
:1000900000000000E14600085F280008E146000873
:1000A000E1460008E1460008E1460008E146000894
:1000B000E1460008E1460008E1460008E146000884
:1000C000E1460008E1460008E1460008E146000874
:1000D000E146000869280008E1460008E1460008FA
:1000E000E14600086528000875280008E146000878
:1000F000E14600080000000000000000E1460008A2
:10010000E1460008E146000881280008E1460008B1
:10011000E1460008E1460008E1460008E146000823
:10012000E1460008E1460008E1460008E146000813
:08013000E1460008E146000869
:1001380010B5054C237833B9044B13B10448AFF319
:1001480000800123237010BDBC08002000000000BF
:10015800F846010808B5034B1BB103490348AFF340
:10016800008008BD00000000C0080020F846010813
:1001780014214160704714207047406A704700009E
:10018800790100087F01000883010008990100082F
:1001980010B5044604F1100000F05CFCC4F8F80047
:1001A8000148C4F87C0110BD88010008F8B5E6B024
:1001B80004460D4616461F460A4906A800F0CAFE20
:1001C80070996F9A05910492009733466E996D9ACB
:1001D800039102922A466C990191214600F060F839
:1001E80067B0F0BD94010008F8B5E6B004460D46C6
:1001F80016461F46094906A800F0ACFE6F996E9A8C
:100208000491039200976D996C9A0291019233467A
:100218002A46214600F087F867B0F0BD940100082F
:1002280038B500281CBF01680029184A23D1184B8B
:100238001C684FF6F0710C404CF24025AC421FBFD1
:100248001B6819404CF27024A14212D1114D296843
:1002580079B911490B68C3F30B03B3F58A6F1FBF54
:100268000968C1F30B0140F28343994204BF01219D
:10027800117028B905E0094B994204BF012111709A
:100288004068BDE8324001F09FBE00BFD80800209A
:1002980000ED00E0002004E00010005C000037489A
:1002A8002DE9F04104460D46216816464A681F4666
:1002B80090478046B8F5403F2ED122680A99936846
:1002C800204698478046B8F5403F25D12368089ACC
:1002D8000799D3F80CC02046E0478046B8F5403F60
:1002E8001AD12368069A39461F692046B8478046BE
:1002F800B8F5403F10D1236829465D69324620464B
:10030800A8478046B8F5403F06D123680B9A09995B
:100318009D692046A847804621680A68204690477C
:100328004046BDE8F0812DE9F04104460D462168BC
:1003380016464A681F4690478046B8F5403F2ED17A
:1003480022680A999368204698478046B8F5403F46
:1003580025D12368089A0799D3F80CC02046E047AE
:100368008046B8F5403F1AD12368069A39461F6976
:100378002046B8478046B8F5403F10D12368294643
:100388005D6932462046A8478046B8F5403F06D109
:1003980023680999DD6900222046A847804621681C
:1003A8000A68204690474046BDE8F0814FF4403047
:1003B80070470000F0B50C4685B0114600281A4673
:1003C8001CBF0568002D0B4B11D082B104B971B95F
:1003D8000D9860B10F9E0E9F0A9B0290049603979A
:1003E8000B980C9E009001962046A8470346184695
:1003F80005B0F0BD020003002DE9F04F0646D0B06D
:100408000868F56DD6F860E0726EB76EF36E00BAE4
:1004180000906C46486800BA60600DF14008886832
:1004280000BAA060C86800BAE060086900BA206134
:10043800486900BA6061886900BAA061C86900BAF1
:10044800E061086A00BA2062486A00BA6062886A95
:1004580000BAA062C86A00BAE062086B00BA2063FA
:10046800486B00BA6063886B00BAA063C86B00BAB7
:10047800E063402058F80C1C58F820CC58F838ACE9
:100488008CEA010158F840CC8AEA01018CEA01099A
:100498004FEAF979401E48F8049BEBD187EA02003D
:1004A80000EA0E00784010EBF5610098DFF824C4EC
:1004B80041186144C81882EABE032B404FEAF06134
:1004C80053405918636859186144CF194FEAB50366
:1004D80083EABE01014081EABE0111EBF765A1681C
:1004E8004D196544A91883EAB0023A404FEAF1650C
:1004F8005A405519E26855194FEAB70282EAB0071F
:1005080065440F4005EBBE0E97EAB00717EBFE6592
:1005180027697D194FEAB10782EA0701654401EAB4
:100528000E01EB18514011EBF36561694D194FEA63
:10053800BE0187EA010E65440EEA030E15EBB00012
:100548008EEA070E0EEBF065D4F818E075446544A2
:10055800AA1881EAB30505404FEAF26E4D40AE4451
:10056800E569AE44E64477444FEAB00080EAB30E4A
:100578000EEA020E8EEAB30E0EEBF765D4F820E011
:1005880075446544691880EAB2053D404FEAF16E4A
:100598004540AE44656AAE44E6440EEBB3034FEA09
:1005A800B70787EAB20E0EEA010E8EEAB20E0EEB1C
:1005B800F365D4F828E075446544281887EAB1053E
:1005C8001D404FEAF06E7D40AE44E56AAE44E64415
:1005D8000EEBB2024FEAB30383EAB10E0EEA000E45
:1005E8008EEAB10E0EEBF265D4F830E0754465443E
:1005F800EF1983EAB00515404FEAF76E5D40AE4447
:10060800656BAE44E6440EEBB1014FEAB20282EAF2
:10061800B00E0EEA070E8EEAB00E0EEBF165D4F8B6
:1006280038E075446544EB1882EAB7050D404FEA97
:10063800F36E5540AE44E56BAE44E6440EEBB000B5
:100648004FEAB10181EAB70E0EEA030E8EEAB70E41
:100658000EEBF065D4F840E07544654481EAB30ECA
:10066800AA180EEA000E4FEAF2658EEA010E7544EA
:10067800DDF844E04FEAB000754480EAB30E654403
:100688000EEA020E15EBB7078EEAB30E0EEBF7650E
:10069800DDF848E04FEAB202754480EA020E65448C
:1006A8000EEA070E69188EEA000E0EEBF165DDF80A
:1006B8004CE07544654405EBB3034FEAB70E1427C5
:1006C8000DF1500CDFF810528EEA010B82EA0B0B89
:1006D8000BEBF36A5CF804BBDA44AA44504483EA9F
:1006E800B10B4FEAF06A8EEA0B0BDA445CF804BBF4
:1006F800DA44AA44524480EAB30B4FEAF26A8BEA1E
:10070800B10BDA445CF804BBDA444FEAB000AA44FF
:1007180080EA020BD6448BEAB30B0BEBFE6A5CF85B
:1007280004BBDA444FEAB202AA4482EA0E0B0AEB8F
:10073800B10180EA0B0B0BEBF16A5CF804BBDA44FD
:100748007F1DAA44282F0AEBB3034FEABE0EBBD382
:100758003C2F61D3502F4DD204EB870CC7F15407BF
:100768005E4CA7FB04A504465D4FA8088EEA010A63
:1007780082EA0A0A5CF804BB0AEBF3655D447D195A
:100788002C1983EAB10A4FEAF4658EEA0A0A55443D
:100798005CF804AB5CF804BB55447D19AA1884EADC
:1007A800B30A4FEAF2658AEAB10A55445D444FEA52
:1007B800B4047D1984EA020AAE448AEAB30A0AEB51
:1007C800FE655CF804AB55444FEAB2027D1982EA33
:1007D8000E0A15EBB10184EA0A0A5CF804BB0AEBBD
:1007E800F1655D447D1915EBB303401E4FEABE0E5B
:1007F800BCD12046F46D1B19F365336EC9183166F8
:10080800716E71447166B36ED218B266F16E40189B
:10081800F06650B0BDE8F08F4EEA010B0EEA010A0F
:100828000BEA020B4BEA0A0A0AEBF36554F827A015
:10083800DFF8B0C0554443EAB10B654403EAB10A96
:100848000BEA0E0B28184BEA0A0A7F1C0AEBF06524
:1008580054F827A0554440EAB30B654400EAB30AAC
:100868000BEAB10BAA184BEA0A0A7F1C0AEBF265DD
:1008780054F827A055444FEAB00040EA020B6544FB
:1008880000EA020A0BEAB30BAE444BEA0A0A7F1CE1
:100898000AEBFE6554F827A055444FEAB20242EA33
:1008A8000E0B654402EA0E0A0BEA000B15EBB101C8
:1008B8004BEA0A0A7F1C0AEBF16554F827A0554455
:1008C8007F1C65443C2F05EBB3034FEABE0EA3D350
:1008D80040E700BF9979825AA1EBD96ECDCCCCCC38
:1008E800D6C162CADCBC1B8F00B581B00168074A5B
:1008F800914200D110B9064801B000BD7C2113F027
:100908005FFE4FF4003001B000BD00BFFC090008D5
:10091800030002002DE9F0410B4A92E8F85188B033
:10092800694681E8F8510268084B9A4200D118B923
:10093800074808B0BDE8F0811422083000F04FFBEA
:1009480008B0BDE8F08100BFDC090008FC09000818
:1009580003000200152904D20268044B9A4200D110
:1009680008B903487047083000F048BBFC09000884
:100978000300020010B481B013460268074CA2427B
:1009880000D118B901B010BC0548704701B000F19A
:10099800240210BC083000F035BB00BFFC09000879
:1009A8000300020010B481B013460268074CA2424B
:1009B80000D118B901B010BC054870470A4601B00B
:1009C80000F1240110BC083000F070BBFC090008DD
:1009D800030002000123456789ABCDEFFEDCBA981E
:1009E80076543210F0E1D2C300000000000000008D
:1009F80000000000F10800081D0900085D09000852
:100A08007D090008AD09000801040008790F0008F5
:100A1800C50F0008810F0008F0B5A3B004460B48C5
:100A280002900D4616461F46094B0822402104A88D
:100A380000F0D1FA28980190009733462A462146BB
:100A480002A800F01BF823B0F0BD00BFFC090008A5
:100A5800100A000810B5040008BF002408D0054893
:100A6800054B20600822402104F1080000F0B3FA89
:100A7800204610BDFC090008100A00082DE9F041C5
:100A880004460E46216817464A681D469047804628
:100A9800B8F5003F19D1226806999368204698470F
:100AA8008046B8F5003F10D123683146DE683A46E3
:100AB8002046B0478046B8F5003F06D12368079A1C
:100AC80029461D692046A847804621680A682046AD
:100AD80090474046BDE8F08110B500F033FA4FF476
:100AE800403400280EBF034C4FF4C07113F068FD6A
:100AF800204610BD0200030010B5044600F022FA9B
:100B080008B9054810BD0021A160D0F87C21116802
:100B180088474FF4403010BD0200030070B504460A
:100B28000D4600F00FFA064E40B1D0F87C0141683E
:100B38008847A84224BF65604FF44036304670BDF0
:100B4800020003002DE9FF4715000C4600D02CB128
:100B5800064600F0F7F95FEA000801D16448C3E0EF
:100B6800D8F8F80001684A689047B0F5003F17D1F7
:100B7800D8F87C118A68404690478146B9F1810FC0
:100B880080F09E80A94508F1FC0A17D2D8F8F80031
:100B98000368D3F80CC02A462146E047B0F5003F69
:100BA80040F08E80D8F8F8000368D3F810C06A4681
:100BB8005146E047B0F5003F76D10AE0002004E056
:100BC800215C0AF800100098401C00900098A84288
:100BD800F6D34FF0000C4749474A484B01AC009800
:100BE800844558D2D3E9007001ADC5E9007010788A
:100BF80000281ABF042086464FF0000E085854F803
:100C08000E5028443E4D05600127D0F800E087606B
:100C1800019D4F681AF80C007D408EEA050585F0A5
:100C2800040E65680F687D4085F0FC05754485F005
:100C3800A30568400AF80C000CF1010CCFE7D3E9D2
:100C4800004501A8C0E9004510782E4D002814BFC2
:100C58004FF0040E4FF0000E01A8744651F80EE054
:100C68000459A6440127CEF80050DEF80040CEF81B
:100C780008704D68019F40687D406C400D68684071
:100C880084F0040480F0FC00041984F057040AF886
:100C98000C400CF1010CCC45D1D3D8F8F800016810
:100CA8004A689047B0F5003F0AD1D8F8F8000368C1
:100CB800D3F80C804A465146C047B0F5003F01D0F2
:100CC800114811E0002006E05AF8201081F06A313E
:100CD8004AF82010401CB0EB990FF5D3B06840F0EB
:100CE8000100B0604FF4403004B0BDE8F08700BFA9
:100CF8000200030090470108D8080020240F0008CC
:100D0800ADBE4ED70DBE75A10100030038B50C4627
:100D1800017A1546CA0702D500F014F908B908483F
:100D280032BDD0F8F80003682146DC682A46A0479F
:100D3800B0F5003F01D0034832BD4FF4403032BD1A
:100D480002000300010003002DE9F84191B00546B7
:100D58000E461746402101A813F032FC297AC8072D
:100D680004D5284600F0EEF8040002D1DFF8A4808C
:100D78004BE0D4F8F800DFF8A0800368D3F810C07F
:100D88006A4601A9E047B0F5003F3ED1D4F8F80023
:100D980001684A689047B0F5003F36D1D4F87C1115
:100DA8008A6820469047D4F8F830024618461B68EF
:100DB800D3F80CC004F1FC01E047B0F5003F24D1A2
:100DC800D4F87C0141688847D4F8F83002461846C0
:100DD8001B68D3F80CC001A9E047B0F5003F14D157
:100DE800D4F8F8000268696893689847B0F5003F3E
:100DF8000BD1D4F8F80003681C693A463146A0477D
:100E0800B0F5003F08BF4FF44038404612B0BDE887
:100E1800F08100BF02000300010003002DE9F84142
:100E2800A5B0074688461646402115A813F0C8FB0A
:100E380000220492402105A813F0C2FB387AC107AA
:100E48005ED5384600F07EF8050059D0D5F8F80090
:100E58002D4C0368D3F810C06A4605A9E047B0F5E1
:100E6800003F3CD1D5F8F80001684A689047B0F5D2
:100E7800003F34D1D5F87C118A6828469047D5F8C8
:100E8800F830024618461B68D3F80CC005F1FC017F
:100E9800E047B0F5003F22D1D5F87C01416888478A
:100EA800D5F8F830024618461B68D3F80CC005A9D7
:100EB800E047B0F5003F12D1D5F8F800026879682C
:100EC80093689847B0F5003F09D1D5F8F800036852
:100ED8001D6904AA15A9A847B0F5003F01D020460E
:100EE8000FE00A4B0A490B4A0396029101924046C9
:100EF8001C68049B009415AA796800F0E5F900E0E5
:100F0800054826B0BDE8F0810100030098470108B4
:100F1800936E030026C703000200030004B001011A
:100F280000170145E10A0008010B0008250B00081D
:100F3800B50300084D0B0008150D0008510D0008F9
:100F4800250E00080168024A914218BF0020704728
:100F58002C0F000810B5040008BF002404D0034873
:100F68002060204609688847204610BD2C0F0008DD
:100F780020225C3013F022BBF0B58468A30800225D
:100F880004F0030407E000F15C0555F8226035BA67
:100F980041F82250521C9A42F5D300220BE000F18E
:100FA8005C0502EB830755F82360D500C5F11805E9
:100FB800EE40CE55521CA242F1D3F0BD30B5C46804
:100FC80003690022E31AD5188C5C0544521C082AD0
:100FD8002C77F8D330BD0360C1600261704738B523
:100FE800044615460022626023685A68904700202C
:100FF8006061A061A5604FF4003032BD81604FF49C
:10100800003070472DE9F84304462079D4F80C8065
:10101800450748BF244845D466691D46A8F1010024
:1010280000EAD60306EBC506B6EBC50F666102D229
:10103800A669761CA6611746A66906EB5576A661D1
:101048000E46E918884225D2A8EB03094A463146DC
:10105800F81813F0B3FA2268136839460FE04246CD
:10106800384613F0ABFA23681A6839462046904789
:1010780007E0311811F00300F1D122681368204607
:101088009847484600EB0809A9F10101A942F0D3A5
:10109800002300E000202A1A3118F81813F08EFAFD
:1010A8004FF40030BDE8F283040002002DE9FC4F44
:1010B800024685B0D0681369DFF86CC1DFF86C812F
:1010C800A0EB030A506840F004005060002703A812
:1010D80002900DF10C0ED8E9003403A8544DC0E974
:1010E80000342878534D00280CBF00230423994668
:1010F8005CF803305EF80940234401261D601C6833
:101108009E60DCF80430039DDCF80090DEF8046093
:101118005D406540484C654089EA0606474C664094
:101128007519474C6540D8E9006B03AC0028C4E941
:10113800006B0EBF002404200424029E5CF800000B
:10114800345920183F4C04600126046886600398CF
:10115800029E43406340384C7068634089EA00004F
:10116800364C6040034438484340280018BF0120EB
:101178005B1E9B41042F2CBFC0B2D80F02F1140391
:1011880053F8200007F00303C3F10303DB00D84042
:101198000DF807007F1C082F9DD315460C466A6979
:1011A800AB69E868D20842EA4372401E00EA0207C7
:1011B800002302409B420AD8524508D28020E055BD
:1011C8007F1C574516D2AAEB0701E01910E08020D2
:1011D800E05500E0E355E8687F1C8742FAD32A68A7
:1011E800136828469847BAF1000F03D051462046A5
:1011F80013F0E6F92A68069E059F93686946284613
:1012080098472A68D2F8009021462846C8472B6894
:10121800DA683946284690470EB1A86830604FF41E
:10122800003007B0BDE8F08F90470108541200085D
:10123800D80800205FC5109304850012FC68017A65
:10124800C0F524FF24AF33D426AF698B04B0010165
:1012580000170145F8B501240094002300240DE08F
:10126800009D065D0F5D7E40F643761CF60F86F006
:10127800010635400095641C009DEB189442EFD39D
:101288001846F2BDF8B5002301240094002A11E0A5
:10129800009C85188F1815F8016C17F8015C6E40D2
:1012A800F643761CF60F86F0010634400094009C45
:1012B800E318521EECD11846F2BD00005D1200087A
:1012C8008D120008010000002DE9F84F1D46DDF8D9
:1012D80028900B9F0D9C4FF0FF3300930E469246CB
:1012E800D9F800B0804632465146D847834664B3A1
:1012F800D9F8043032465146404698476FEA0B0207
:10130800521C42EA0B0200996FEAD2735B1C194027
:10131800C2430091521C024300996FEAD2735B1CCE
:101328001940009186F05531484087EA000181F064
:101338005531216080F05531C943491C0843009A52
:101348006FEAD070401C82430092D9F80800012847
:1013580009D17540E943491C0D4300986FEAD572DD
:10136800521C90430AE0F11C85EA9102D243521CB8
:10137800154300986FEAD5735B1C984386F0AA362C
:10138800009086EA0B0686F0AA33F243DB430C98FA
:10139800C2F3C0725B1C42EAD3720099D243521C5A
:1013A80091430091774000998843009987F0AA37C4
:1013B8000F403843BDE8F28F034613F8012B002A8B
:1013C800FBD1181A0138704781F0004102E000BFD4
:1013D80083F0004330B54FEA41044FEA430594EAED
:1013E800050F08BF90EA020F1FBF54EA000C55EA28
:1013F800020C7FEA645C7FEA655C00F0E2804FEAF9
:101408005454D4EB5555B8BF6D420CDD2C4480EADA
:10141800020281EA030382EA000083EA010180EA0A
:10142800020281EA0303362D88BF30BD11F0004F58
:101438004FEA01314FF4801C4CEA113102D040428E
:1014480061EB410113F0004F4FEA03334CEA1333C9
:1014580002D0524263EB430394EA050F00F0A780E1
:10146800A4F10104D5F1200E0DDB02FA0EFC22FADC
:1014780005F2801841F1000103FA0EF2801843FAD0
:1014880005F359410EE0A5F120050EF1200E012AC1
:1014980003FA0EFC28BF4CF0020C43FA05F3C018FF
:1014A80051EBE37101F0004507D54FF0000EDCF178
:1014B800000C7EEB00006EEB0101B1F5801F1BD321
:1014C800B1F5001F0CD349085FEA30004FEA3C0C25
:1014D80004F101044FEA445212F5800F80F09A801B
:1014E800BCF1004F08BF5FEA500C50F1000041EB1F
:1014F800045141EA050130BD5FEA4C0C404141EB23
:101508000101013C28BFB1F5801FE9D291F0000F1D
:1015180004BF01460020B1FA81F308BF2033A3F1CC
:101528000B03B3F120020CDA0C3208DD02F1140CC3
:10153800C2F10C0201FA0CF021FA02F10CE002F1FE
:101548001402D8BFC2F1200C01FA02F120FA0CFCF7
:10155800DCBF41EA0C019040E41AA2BF01EB045140
:10156800294330BD6FEA04041F3C1CDA0C340EDC3E
:1015780004F11404C4F1200220FA04F001FA02F381
:1015880040EA030021FA04F345EA030130BDC4F13F
:101598000C04C4F1200220FA02F001FA04F340EA34
:1015A8000300294630BD21FA04F0294630BD94F0E5
:1015B800000F83F4801306BF81F480110134013DCC
:1015C8004EE77FEA645C18BF7FEA655C29D094EA3D
:1015D800050F08BF90EA020F05D054EA000C04BFBB
:1015E8001946104630BD91EA030F1EBF00210020A6
:1015F80030BD5FEA545C05D14000494128BF41F045
:10160800004130BD14F580043CBF01F5801130BDA8
:1016180001F0004545F0FE4141F470014FF0000033
:1016280030BD7FEA645C1ABF194610467FEA655CE4
:101638001CBF0B46024650EA013406BF52EA033586
:1016480091EA030F41F4002130BD00BF90F0000F74
:1016580004BF0021704730B54FF4806404F13204B0
:101668004FF000054FF0000150E700BF90F0000F69
:1016780004BF0021704730B54FF4806404F1320490
:1016880010F0004548BF40424FF000013EE700BF60
:1016980042004FEAE2014FEA31014FEA02701FBFF0
:1016A80012F07F4393F07F4F81F06051704732F022
:1016B8007F4208BF704793F07F4F04BF41F4002179
:1016C800704730B54FF4607401F0004521F00041D7
:1016D8001CE700BF50EA010208BF704730B54FF061
:1016E80000050AE050EA010208BF704730B511F062
:1016F800004502D5404261EB41014FF4806404F19A
:1017080032045FEA915C3FF4D8AE4FF003025FEA1F
:10171800DC0C18BF03325FEADC0C18BF033202EBA3
:10172800DC02C2F1200300FA03FC20FA02F001FAFD
:1017380003FE40EA0E0021FA02F11444BDE600BFA0
:101748004FF0FF3C06E000BF4FF0010C02E000BF85
:101758004FF0010C4DF804CD4FEA410C7FEA6C5C68
:101768004FEA430C18BF7FEA6C5C1BD001B050EA0B
:10177800410C0CBF52EA430C91EA030F02BF90EAF6
:10178800020F0020704710F1000F91EA030F58BFB5
:10179800994208BF90422CBFD8176FEAE37040F017
:1017A800010070474FEA410C7FEA6C5C02D150EAB5
:1017B800013C07D14FEA430C7FEA6C5CD6D152EA70
:1017C800033CD3D05DF8040B704700BF8446104635
:1017D80062468C461946634600E000BF01B5FFF734
:1017E800B7FF002848BF10F1000F01BD4DF808ED04
:1017F800FFF7F4FF0CBF012000205DF808FB00BFD5
:101808004DF808EDFFF7EAFF34BF012000205DF82E
:1018180008FB00BF4DF808EDFFF7E0FF94BF01207B
:1018280000205DF808FB00BF4DF808EDFFF7CEFF7C
:1018380094BF012000205DF808FB00BF4DF808EDBB
:10184800FFF7C4FF34BF012000205DF808FB00BF8C
:101858004FEA410212F5001215D211D56FF47873D0
:10186800B3EB625212D94FEAC12343F0004343EA73
:10187800505311F0004F23FA02F018BF404270474E
:101888004FF00000704750EA013005D111F00040D8
:1018980008BF6FF0004070474FF00000704700BF6E
:1018A80080F0004002E000BF81F0004142001FBF0D
:1018B8005FEA410392EA030F7FEA226C7FEA236C16
:1018C8006AD04FEA1262D2EB1363C1BFD21841400B
:1018D80048404140B8BF5B42192B88BF704710F0A1
:1018E800004F40F4000020F07F4018BF404211F044
:1018F800004F41F4000121F07F4118BF494292EAAC
:10190800030F3FD0A2F1010241FA03FC10EB0C00D7
:10191800C3F1200301FA03F100F0004302D5494264
:1019280060EB4000B0F5000F13D3B0F1807F06D311
:1019380040084FEA310102F10102FE2A51D2B1F109
:10194800004F40EBC25008BF20F0010040EA0300FE
:101958007047490040EB0000013A28BFB0F5000F7E
:10196800EDD2B0FA80FCACF1080CB2EB0C0200FA34
:101978000CF0AABF00EBC25052421843BCBFD04083
:101988001843704792F0000F81F4000106BF80F4FD
:1019980000000132013BB5E74FEA41037FEA226CC0
:1019A80018BF7FEA236C21D092EA030F04D092F08B
:1019B800000F08BF0846704790EA010F1CBF0020BF
:1019C800704712F07F4F04D1400028BF40F000401C
:1019D800704712F100723CBF00F50000704700F03C
:1019E800004343F0FE4040F4000070477FEA226263
:1019F80016BF08467FEA23630146420206BF5FEA34
:101A0800412390EA010F40F4800070474FF0000333
:101A180004E000BF10F0004348BF40425FEA000CFA
:101A280008BF704743F0964301464FF000001CE0A2
:101A380050EA010208BF70474FF000030AE000BFF8
:101A480050EA010208BF704711F0004302D5404236
:101A580061EB41015FEA010C02BF844601460020A8
:101A680043F0B64308BFA3F18053A3F50003BCFAC3
:101A78008CF2083AA3EBC25310DB01FA02FC634470
:101A880000FA02FCC2F12002BCF1004F20FA02F277
:101A980043EB020008BF20F00100704702F120026A
:101AA80001FA02FCC2F1200250EA4C0021FA02F2CB
:101AB80043EB020008BF20EADC7070474FEA40029F
:101AC800B2F1FE4F0FD34FF09E03B3EB12620DD964
:101AD8004FEA002343F0004310F0004F23FA02F0CE
:101AE80018BF404270474FF00000704712F1610F75
:101AF80001D1420205D110F0004008BF6FF000404C
:101B080070474FF00000704753B94AB9002908BF21
:101B180000281CBF4FF0FF314FF0FF3000F070B9C4
:101B2800ADF1080C6DE904CE00F006F8DDF804E02C
:101B3800DDE9022304B070472DE9F047089E0D4601
:101B480004460F46002B4AD18A42944665D9B2FA18
:101B580082F343B102FA03FCC3F120029F4020FA4A
:101B680002F217439C404FEA1C4E1FFA8CF5B7FB54
:101B7800FEF1220C0EFB117742EA074201FB05F049
:101B880090420AD91CEB020201F1FF3780F01B8159
:101B9800904240F2188102396244121AA4B2B2FB90
:101BA800FEF00EFB102244EA024400FB05F5A542B4
:101BB8000AD91CEB040400F1FF3280F00681A5422B
:101BC80040F203816444023840EA0140641B00216A
:101BD8001EB1DC400023C6E90043BDE8F0878B4214
:101BE80008D9002E00F0EC800021C6E9000508465F
:101BF800BDE8F087B3FA83F1002949D1AB4202D39B
:101C0800824200F2F780841A65EB0302012017462E
:101C1800002EE2D0C6E90047DFE702B9FFDEB2FADC
:101C280082F3002B40F08F808A1A4FEA1C471FFA74
:101C38008CFE0121B2FBF7F507FB1520220C42EAC6
:101C480000420EFB05F0904208D91CEB020205F198
:101C5800FF3802D2904200F2CA804546121AA4B256
:101C6800B2FBF7F007FB102244EA02440EFB00FE29
:101C7800A64508D91CEB040400F1FF3202D2A645A0
:101C880000F2BA801046A4EB0E0440EA05409FE734
:101C9800C1F120078B4022FA07FC4CEA030C05FA35
:101CA80001F420FA07F3FD40234300FA01F94FEA53
:101CB8001C401FFA8CFEB5FBF0F81C0C00FB1855F5
:101CC80044EA054408FB0EF5A54202FA01F20BD9D5
:101CD8001CEB040408F1FF3A80F08780A54240F22B
:101CE8008480A8F102086444641B9DB2B4FBF0F33D
:101CF80000FB134445EA044403FB0EFEA64508D93D
:101D08001CEB040403F1FF306BD2A64569D9023BF2
:101D1800644443EA0840A0FB0283A4EB0E049C42FF
:101D2800C6461D4655D352D056B1B9EB0E0364EBE7
:101D3800050404FA07F7CB40CC401F43C6E90074FA
:101D48000021BDE8F087C3F1200102FA03FC20FA64
:101D580001F225FA01F19D402A434FEA1C471FFA78
:101D68008CFEB1FBF7F007FB1015110C41EA054199
:101D780000FB0EF58D4204FA03F408D91CEB0101AF
:101D880000F1FF382FD28D422DD902386144491B0A
:101D980092B2B1FBF7F507FB151142EA014205FBC8
:101DA8000EF1914208D91CEB020205F1FF3816D258
:101DB800914214D9023D6244521A45EA004139E77A
:101DC8003146304609E73946E7E61046FCE6C145A4
:101DD800AAD2B8EB020E63EB0C050138A4E745461E
:101DE800EAE7034695E74046D1E7D0467CE7023D5F
:101DF800624433E708460BE76444023843E700BF10
:101E0800704700BF1348144A08B54FF00043C0E9B3
:101E180000230422002342610122C2614FF4805151
:101E280007220383C0E90233C0E90933C0E90C1271
:101E38000361837680F8203080F82C30826380F844
:101E48003C30C36405F020FB18B1BDE8084000F041
:101E580031BC08BDDC080020002401400268084BA2
:101E68009A4282B00AD14FF0B0431A6E42F400721F
:101E78001A661B6E03F400730193019B02B070474E
:101E8800002401400268054B9A4201BF4FF0B0425E
:101E9800136E23F400731366704700BF00240140DB
:101EA80030B585B000240546CDE901440394FFF719
:101EB800A9FF144805F080FE08B100F0FBFB1148AB
:101EC800039401A9CDE9015405F03CFC08B100F0E8
:101ED800F1FB0C4805F09AFD08B100F0EBFB4FF060
:101EE800FF31084805F0D0FB064805F047FE0548D5
:101EF80005F024FC0446034805F0EAFD204605B039
:101F080030BD00BFDC080020014B024A1A60704750
:101F1800DC0800200024014008B50948FFF7C0FF8D
:101F280068B1084BB3F8AA304FF6FF72934216BF58
:101F380040F6E442044B5343B3FBF0F398B208BDB8
:101F4800002000B40075FF1FD8084C0013B500230B
:101F5800ADF80630FFF7E0FF04461948FFF7A0FF89
:101F6800184BB3F8C820B3F8A8108A4204FB00F055
:101F780018D040F6E443B0FBF3F364205B1A434304
:101F8800521A93FBF2F31E331BB2ADF80630BDF8BC
:101F980006305BB21B02ADF80630BDF8060000B291
:101FA80002B010BD4FF47A7240F6FF73B0FBF3F342
:101FB8005343A3F53923A3F50C6340F6C412E0E7B5
:101FC800001000B00075FF1F4FF0B04382B09A6A4E
:101FD80022F480529A629A6C42F480529A649B6C02
:101FE80003F480530193019B002002B070474FF027
:101FF800B04382B09A6C02439A649B6C034001938D
:10200800019B02B0704708B50420FFF7F0FF0120DC
:10201800FFF7EDFF0220FFF7EAFF002211460B2031
:1020280005F068FE0B2005F097FE002211460C20F3
:1020380005F060FE0C2005F08FFE002211460D20F1
:1020480005F058FE0D2005F087FE002211460E20EF
:1020580005F050FE0E2005F07FFE002211460F20ED
:1020680005F048FE0F2005F077FE002211461020EB
:1020780005F040FE102005F06FFE002211461120E9
:1020880005F038FE112005F067FE002236201146C3
:1020980005F030FEBDE80840362005F05DBE0000C2
:1020A80008B506F0A1F810B16FF0040008BD064BA2
:1020B8009A6942F040429A614CF2FA321A6106F08B
:1020C800A5F80028F2D0EFE700400058F0B585B039
:1020D80000230C4600930646A8B3FFF7E1FF054628
:1020E80070BB06F081F888BB1A481B4A022301938B
:1020F800D0F8E01506F1784302EA8121B3FBF1F745
:1021080001FB1733DB0A0293D0F8E00504F17841AC
:102118000139314402EA8022B1FBF2F002FB1011CE
:10212800C3EBD1230133694601A8039306F0EEF807
:1021380020B102280CBF01256FF0010506F066F8F2
:10214800284605B0F0BD6FF00505F9E76FF0040506
:10215800F6E700BF0070FF1F00FCFF03014B18608B
:1021680000207047400900202DE9F04F89B0B0F1F8
:10217800006F06460F460092C0F0C580DFF89881D0
:10218800664DD8F8E03505EA832303F10063013B87
:10219800984200F2B880002800F0B880002900F0CA
:1021A800B58040EA02035B0740F0B080FFF778FF94
:1021B8000446A0BB06F018F8002840F0AA80D8F81A
:1021C800E01506F1784205EA8121B2FBF1F301FB43
:1021D8001322009B03F17843013B3344B3FBF1F036
:1021E80001FB1033DB0A01334FEAD22AA3EBD222D8
:1021F800012A039388BFC6F30A050AF58038C6F199
:10220800080398BF009D069388BFC5F500654FEA8F
:10221800C828B346039B9A4505D305F0F7FF204627
:1022280009B0BDE8F08FA6F10803069A1A44954252
:1022380019D804950197CDF814B04FF00009059B03
:1022480009EB0301049B99453ED3009BAB442F4403
:102258005D1BB5F5006F28BF4FF400650AF1010A50
:1022680008F50068D6E753F8081F5A68B2F1FF3F2F
:1022780008BFB1F1FF3FD8D0294B186810B96FF0EB
:102288000504CAE7B8F1000F04D04FF400624146D4
:1022980011F028FDDFF88890D9F80030CBF30A0058
:1022A80039461844AAB211F01DFD4FF400614046AA
:1022B800FFF70CFF08BBD9F8003001934FF4006317
:1022C800CDF814800493B8E7019B07914B4402931F
:1022D8000120D3E9002305F0D3FF88B90799019BB2
:1022E800D1E9000259F80310029B5B689A4208BFC3
:1022F800884205D109F10809A1E76FF001048CE7CC
:102308006FF0030489E74FF0FF3488E76FF00504A6
:1023180085E76FF0040482E70070FF1F00FCFF03ED
:1023280040090020B1F1006F70B511D30B4BD3F801
:10233800E0650B4B03EA862303F10063013B9942F6
:1023480006D840B139B192B211F0CCFC002070BD72
:102358004FF0FF30FBE76FF00500F8E70070FF1F54
:1023680000FCFF03B0F1006F10B40DD3084BD3F895
:10237800E045084B03EA842303F10063013B9842DC
:1023880002D810BCFFF7A2BE4FF0FF3010BC704758
:102398000070FF1F00FCFF034FF0B04382B0DA6CFF
:1023A8000243DA64DB6C03400193019B02B070477F
:1023B8002DE9F04186B01422002101A812F0CAF8D4
:1023C80001203B4EFFF7E8FF0220FFF7E5FF04205E
:1023D800FFF7E2FF08210122304606F00BF901253C
:1023E8004FF40417022301A94FF09040CDE90137BB
:1023F800039505F0D9FF4FF4441301A94FF090401D
:102408000024CDE902354FF02008019505F0CCFFF6
:1024180001A93046CDE90187039405F0C5FF01A95C
:102428003046CDE90187039405F0BEFF082301A9D2
:102438003046CDE90135CDE9035405F0B5FF4FF439
:10244800007301A94FF09040CDE90135CDE903545F
:1024580005F0AAFF04230DEB03013046CDE9013551
:10246800CDE9034405F0A0FF22462146062005F0E9
:1024780041FC062005F070FC22462146072005F0A5
:1024880039FC072005F068FC22462146162005F095
:1024980031FC162005F060FC22462146162005F086
:1024A80029FC162005F058FC06B0BDE8F08100BFF5
:1024B8000004004808B51248124A134BC0E900232B
:1024C80000230122C0E90232C0E90433C0E906331F
:1024D800036206F003FA08B100F0ECF8084800219E
:1024E80006F07CFB08B100F0E5F80548002106F08D
:1024F8009BFB18B1BDE8084000F0DCB808BD00BF80
:10250800040A0020005800405D3E302070B596B0A7
:1025180005461422002103A812F01CF838220021D5
:1025280008A812F017F82A68304B9A425BD180232A
:10253800089308A84FF440230E9307F0D1F808B188
:1025480000F0B8F84FF0B0444FF4C050E36C43F0DB
:102558000103E364E36C03F001030293029B12237B
:102568000026CDE903030323CDE905634FF090402E
:10257800042303A9079305F017FFA36DDFF870C0C4
:1025880043F48003A365A36D1A4C03F480030193FD
:10259800019B26620D23C4E900C320468023C4E9B9
:1025A8000266C4E90436C4E9066605F035FC08B1DC
:1025B80000F080F8104AEC63A562104C0E23C4E9C1
:1025C80000231021002380222046C4E90213C4E915
:1025D8000423C4E90633236205F01EFC08B100F0A9
:1025E80069F8AC63A56216B070BD00BF0058004022
:1025F800440002404409002058000240A409002079
:1026080000B59BB04822002108A811F0A3FF1822AA
:10261800002102A811F09EFF06F02CFB4FF0B042FB
:102628000120D2F8903023F01803C2F89030D2F885
:10263800003423F4C06343F40073C2F80034D2F8C2
:10264800003403F4C0630193019B2423089381237E
:102658000B930023CDE91003B02208A8CDE912237B
:1026680006F080FC08B172B6FEE74F23CDE90230D0
:10267800CDE90400CDE90600022102A806F00CFF0E
:1026880008B172B6FEE71BB05DF804FB08B504F0AC
:10269800A9FEFFF7B5FFFFF78BFEFFF7B4FCFFF7C6
:1026A80009FF00F0F8FD40F6B83000F049FA00F0F4
:1026B800F9FDFCE772B6FEE700B58DB02C220021CB
:1026C80001A811F047FF1748174B03601F238360C9
:1026D8004FF080420023C0E90433C0E90723836137
:1026E8004FF48073436207F081F908B1FFF7E2FF06
:1026F8000C4807F0A7FA08B1FFF7DCFF4FF00053CA
:1027080000220793074808924FF4807301A90292A8
:1027180006920B9307F0CAF908B1FFF7CBFF0DB08B
:102728005DF804FB580A00200028004010B5044654
:1027380090B03822002102A811F00CFF2268194B32
:102748009A422CD14FF48033029302A84FF480733D
:102758000F9306F0C5FF08B1FFF7ACFF4FF0B04389
:102768000220D3F8902042F40042C3F890209A6DDA
:1027780042F480629A659B6D002203F480631146DF
:102788000193019B05F0B6FA022005F0E5FA002254
:102798002A20114605F0AEFA2A2005F0DDFA10B01D
:1027A80010BD00BF002800407047000008B504F0C5
:1027B8002FFE044B0120C3F88800BDE8084006F04E
:1027C800B1BA00BF0004005804F029BE08B504F0EF
:1027D80026FE00F063FCFFF7EBFDFFF714FCBDE8F5
:1027E8000840FFF767BE08B504F012FEBDE80840D0
:1027F8000121002006F046BA70477047FEE7FEE761
:10280800FEE7FEE7FEE77047704770477047000035
:10281800014807F03DBA00BF580A0020012005F022
:10282800EFBE022005F0ECBE70477047014805F086
:102838006DBC00BF44090020014805F067BC00BF1B
:10284800300B0020014805F061BC00BFD00A002011
:10285800FFF7F2BF7047202005F0D2BE7047000096
:10286800014807F0D9BD00BF900B0020014807F0D0
:1028780041B800BF580A0020014807F034BC00BF27
:10288800BC0A00202DE9F04389B080460020109E44
:102898000790894615461F46FDF7C2FCF0B9104C53
:1028A800CDE90090CDE9020407AB0E480593142347
:1028B80004933A46434629460068FDF77BFD2346C4
:1028C800324604F1140153F8044B42F8044B8B428E
:1028D800F9D1079B337509B0BDE8F0830120FAE709
:1028E800900A00208C4701087FB5124C00253C2334
:1028F80002A86375CDE90255257500F0C3F80423D5
:1029080003AA009412210C48FFF7BCFF0B491422BC
:10291800204611F00FFE0646B0FA80F040096075B7
:102928000090074B2A462946022011F0D3F830467A
:1029380004B070BDA40A0020D24701083E0E002052
:10294800B4470108054808B50823036007F0E6F90D
:1029580018B1BDE80840FFF7ADBE08BDBC0A0020AD
:102968004FF0B04307B55A6E42F001025A665B6EEB
:10297800002203F00103019311463220019B05F068
:10298800B9F9322003B05DF804EB05F0E5B90000B1
:102998000CB407B5054A05AB1021019311F0ACFC46
:1029A80003B05DF804EB02B0704700BFE4470108CC
:1029B80030B585B0044602A80D4611F0C9FABDF934
:1029C8000C30064A00931021029B2046FFF7E0FFD7
:1029D8002046FEF7F1FC288005B030BDE447010829
:1029E8004FF0B04210B5936823F40043936011F0A0
:1029F80037FB0E4B01241C7000F0B6F811F000F8FC
:102A08000B4811F017F80B4B4FF400421A610320E2
:102A180011F016F8FFF778FA00F012F911F00CF936
:102A280021462046BDE8104011F026B9C80A00200A
:102A3800B92900080040005811F034B908B5FFF76B
:102A48006BFA40F6B83398420CD8B0F5E16F0BD367
:102A5800FE23A0F5E16058434FF49663B0FBF3F012
:102A6800C0B208BDFE20FCE70020FAE77FB5684643
:102A780000F0CAF80198FFF721F800B207B05DF836
:102A880004FB0000194A38B5D2F88035591C0446B1
:102A980019D104F0CBFC054604F0D4FC054404F03D
:102AA800CBFC2B0EE3712B0CA3712B0A6371030E65
:102AB800E370C0F30742C0F307232571C0B2A270C8
:102AC8006370207038BD190AC3718171190C1B0E0F
:102AD80041710371D2F88435C370D2F88405C0F30C
:102AE8000722C0F30743000EE9E700BF0070FF1F8D
:102AF80038B5094BD3F8803503600133054609D151
:102B080004F094FC044604F097FC444004F09AFC5A
:102B180044402C6038BD00BF0070FF1F0121022017
:102B280011F094B80021022011F090B800207047ED
:102B3800024B187808B100F0BBB87047C80A0020EB
:102B480082B00190019802B000F04EB94FF0B04346
:102B580082B0DA6C42F00202DA64DB6C03F0020342
:102B68000193019B02B070472DE9F043254C87B0D3
:102B780004F06EFC04F074FC04F07AFC01230025D8
:102B880002934FF48059032301A9204604934FF47C
:102B9800005803950595FFF7D9FFFFF7D7FFFFF713
:102BA800D5FFFFF7D3FFCDF8049005F0FDFB01A991
:102BB80020464FF40067CDF8048005F0F5FB01A925
:102BC80020464FF40046019705F0EEFB01A9204688
:102BD800019605F0E9FB2A464946204605F00AFD1C
:102BE8002A464146204605F005FD2A463946204634
:102BF80005F000FD2A463146204605F0FBFC07B0EB
:102C0800BDE8F0830004004810B50446FFF79EF9BC
:102C1800074BA36040F30F20FEF7FCFE054B064A66
:102C28002360064B6060C4E90323002010BD00BF89
:102C38000000484200007A440D093E00AB0305003D
:102C480000207047014B1868704700BFCC0A00206D
:102C58000320704708B501464FF47A7200238002BA
:102C6800890DFEF751FF08BD4FF47A73A0FB0303EB
:102C7800800A40EA83507047034B98689A689042EC
:102C8800FBD1C043704700BF0028004008B5FFF7DC
:102C9800F3FF014B186008BDCC0A002008B5FFF708
:102CA800EBFF024B1B68C01A08BD00BFCC0A00200E
:102CB800024B187808B1FFF7DFBF7047C90A002038
:102CC80010B5074B074C0122DA654FF48071204696
:102CD80006F0D6FD4FF0FF332363002010BD00BF80
:102CE80000280040580A002002460021014806F04A
:102CF800E0BF00BF580A002002460121014806F043
:102D0800D8BF00BF580A002010B58CB02C22002173
:102D1800044601A811F01EFCFFF7D2FF0C4B0D482A
:102D28001B681C440023089306934FF00053E443A8
:102D3800079301224FF4807301A902940B9306F0C4
:102D4800B5FE08B1FFF7B6FC00200CB010BD00BFFF
:102D5800CC0A0020580A002038B50546FFF78CFF3A
:102D680002210446074806F0ABFFC4F309024FF4FA
:102D78007A71A2FB0121920AA30A2A8043EA8050B1
:102D880038BD00BF580A00200148002106F098BF4E
:102D9800580A00200148012106F092BF580A002075
:102DA800F8B50F4D2E78CEB90E4C4FF0FF3727638C
:102DB800FFF782FCFFF784FF4FF48071204606F08E
:102DC8005FFD2046276306F01FFF3246204602219A
:102DD80006F06FFFFFF75AFF01232B700020F8BDA4
:102DE800C90A0020580A0020014610B54FF47A722B
:102DF80000238002890DFEF787FE0146FFF73CFF9E
:102E08000446FFF739FF031B8B4200D310BD00BFF8
:102E1800F7E711F02DBA000010B5064C0221204644
:102E280006F04EFF0221421C2046BDE8104006F085
:102E380040BF00BF580A00201648174A08B54FF48B
:102E4800E133C0E9002300230C22C0E90233C0E9C2
:102E58000523C0E90733C0E90933036108F0BDF869
:102E680008B1FFF727FC0B48002108F032FA08B137
:102E7800FFF720FC0748002108F04BFA08B1FFF7DC
:102E880019FC044808F005FA18B1BDE80840FFF736
:102E980011BC08BD900B00200044004070B596B0EE
:102EA80005461422002103A811F054FB3822002102
:102EB80008A811F04FFB2A68334B9A4261D10223CC
:102EC800089308A8314B0A9306F00AFC08B1FFF7EB
:102ED800F1FB4FF0B0430C219A6D2D4C42F40032B7
:102EE8009A659A6D02F400320292029ADA6C42F004
:102EF8000102DA64DB6C03F001030193019B0223F6
:102F08000026CDE903130323CDE905634FF0904074
:102F1800072303A9079305F047FA1E4826621423DE
:102F2800C4E900031023C4E9023620468023C4E91B
:102F38000436C4E9066604F06FFF08B1FFF7BAFB70
:102F4800154AEC67A562154C1323C4E900232046F3
:102F580000238022C4E90233C4E90423C4E9063308
:102F6800236204F059FF08B1FFF7A4FB2520C5F838
:102F7800804000220221A56204F0BCFE252004F056
:102F8800EBFE16B070BD00BF0044004004000C000A
:102F9800300B0020800002406C000240D00A002064
:102FA80002680E4B9A4210B5044616D14FF0B04253
:102FB8000C21936D23F4003393654FF0904005F096
:102FC8009FFAE06F04F09CFFD4F8800004F098FFAB
:102FD800BDE81040252004F0CDBE10BD00440040DF
:102FE80008B50A460146024807F07AF9002008BDEC
:102FF800900B002013B5114B114C18604FF40013BF
:10300800009302AB13E90600204608F0E6F82368AF
:10301800DA69D103FCD4DA695202FCD59A68084807
:1030280042F480029A6008F01EF906490448012219
:1030380008F08CF8002002B010BD00BF240C00205E
:10304800900B00202C0C002008B5074B1860FEF7E9
:10305800DAFFFFF7F1FE054AD2F8803043F000634B
:10306800C2F88030002008BD280C00200008005855
:1030780008B54FF0B04308489A6B42F400329A639F
:103088009A6B22F400329A63FFF78AFF0F2004F04C
:1030980071FE002008BD00BF900B002008B507484E
:1030A80007F09BFF08B1FFF705FB054804F0B4FEE5
:1030B80018B1BDE80840FFF7FDBA08BD900B002025
:1030C800300B00200268044B9A4203D1034B0020C6
:1030D8001B681847704700BF00440040280C0020B8
:1030E80002680B4B9A4210B504460FD1094B1B6876
:1030F8002BB1D0F8902012B90748012198472046F3
:103108000549BDE81040012208F020B810BD00BFF5
:1031180000440040240C00202C0C0020024801220E
:10312800102105F067BA00BF0004004802480022D9
:10313800102105F05FBA00BF0004004813B5134C16
:1031480023785BB9E37C03F0FF023BB9104B1146CF
:10315800022002B0BDE8104010F0BCBCFFF7C4FB71
:1031680000380C4B18BF0120400018701A78022A4A
:1031780002BF00222270E2741B7800930022064BE3
:103188001146032010F0A6FC02B010BD3E0E002030
:1031980040480108340C00205C48010838B5184C38
:1031A80023785BBBE37C03F0FF023BBB154D2B6828
:1031B800012B0CD92B68042B09D81146124B02207D
:1031C80010F088FC114A0421012000F081FB2B68D3
:1031D800042B13D900220E4B1146022010F07AFC62
:1031E800FFF782FB00380B4B18BF01204000187016
:1031F8001B78022B02BF00232370E37438BD00BF85
:103208003E0E0020300C0020734801089848010841
:103218009D480108340C002008B5FFF77FFF002205
:10322800054B1146032010F055FC01F01DFDBDE8CB
:103238000840FFF77BBF00BFD0480108022801D82B
:10324800FFF76CBF7047022801D8FFF76FBF7047C0
:10325800022808B51BD8012210210D4805F0CAF92B
:103268003220FFF76DFC0A480022102105F0C2F950
:1032780001221021064805F0BDF93220FFF760FC55
:10328800BDE8084002480022102105F0B3B908BD86
:1032980000040048704708B5FFF7A2FBBDE80840E6
:1032A80000F0D8BC4FF0FF3010F060BD7047704799
:1032B800014BD870704700BF5C000020014B1874A8
:1032C800704700BF5C00002007B5064B00221B5C5E
:1032D80000931146044B022010F0FCFB03B05DF88C
:1032E80004FB00BF0C490108F248010808B5022098
:1032F800002110F003FDBDE80840014810F066BF4A
:103308008C0D00200021012010F0F8BC13B50D4CE5
:10331800A0B120600C4810F00BFF21680A4810F09B
:103328008FFF094810F052FF236800930022074BD3
:103338001146032010F0CEFB02B010BD42F210730C
:103348002360E7E7740000208C0D00201049010875
:1033580013B50D4C206023680BB90C4B23600C4847
:1033680010F0E6FE21680A4810F06AFF084810F0DD
:103378002DFF236800930022064B1146032010F00E
:10338800A9FB02B010BD00BF0C000020A086010000
:10339800A40D00203949010837B5044600283AD061
:1033A80090F90650002D38D11F4810F0C1FE2A466A
:1033B80029461E4B022010F08DFBE379012B0CBF30
:1033C8001B4B1C4B2A46294602201B4D10F082FB42
:1033D800E3792B70194B1868FFF7BAFF184B186878
:1033E800FFF794FF2978174A174B012918BF13468E
:1033F800002200931146154B012010F06BFB94F945
:103408000530019394F9043000930022104B1146C3
:10341800022010F05FFB03B030BD00220D4B1146B7
:10342800022010F057FBEAE7280D00207E4901082A
:1034380093490108B0490108580D00200C000020EC
:10344800740000207949010875490108CD4901082F
:10345800054A0108EC49010838B504460D460748F5
:103468004FF40061FEF77EFF30B92A462146034833
:10347800BDE83840FEF778BE38BD00BF00F003084D
:103488000A460149FEF74EBF00F0030870B516481A
:1034980010F04EFE08F0A2FB044650B10022134B78
:1034A8001146022010F016FBBDE87040104810F0DD
:1034B8008DBE104D104B02460146022010F00AFB4B
:1034C80001260E4B2E7022462146022010F002FBE8
:1034D8000B4808F015FA2878314607F067FF0248CC
:1034E80010F074FEE0E700BF8C0D00202E4A0108A2
:1034F8005C0D0020000000204C4A0108604A0108C9
:103508005C00002030B587B0FFF798FA044608F051
:1035180043F8054680B10024474810F009FE474BA0
:1035280045481968A14238BF214610F089FE424833
:1035380010F04CFE07B030BD01464FF4807010F01B
:10354800DDFB02A801F0A8F923B203EB4303FE2236
:1035580003EB4313B3FBF2F3394A392111703949AC
:1035680050680978DBB28DF81430017050684570E6
:1035780050682724847050680124C470506803710F
:10358800314B187840B11D70536861F07F01197094
:103598003A23137005231CE02C4B2D48197811B9D8
:1035A80001780029F6D000210170197053680421B0
:1035B8005971BDF808305168180A88715168CB7183
:1035C800BDF8103051681B0A0B72BDF810304B72F1
:1035D8000A232049204C0978012988BF0023537009
:1035E800637A33B107F0C4FF012802D1204610F0F6
:1035F8009FFD1A4B1248D978002207F0E3FF0446D2
:1036080030B90146164B0122032010F063FA83E714
:10361800063480D107F0A6FF044600283FF47CAFAB
:1036280001224FF47A730021B0FBF3F310460093A4
:103638000C4B10F04FFA6FE78C0D0020740000203F
:1036480004000020270D0020BC0D0020530E002090
:103658003D0E0020340C0020280D00205C000020C6
:103668007F4A01088E4A010800B503468DB000283C
:103678002CD0407802280AD003282AD0164B0022E2
:10368800114602200DB05DF804EB10F023BA1A7F42
:103698000B92DA7E0A929A7E09925A7E08921A7ED4
:1036A8000792DA7D06929A7D05925A680492DA6842
:1036B800039293F914200292B3F9122001921B7C11
:1036C80000930022054B114610F004FA0DB05DF886
:1036D80004FB034BD3E700BFAC4A0108C34A010807
:1036E800354B010801284FF000020CBF024B034B79
:1036F8001146022010F0EEB9544B0108664B010840
:103708001FB50446002831D00378002B2ED01D4861
:1037180010F05CFD002211461B4B022010F0DAF974
:1037280094F91830039394F90A300293237C019397
:10373800E368009300221146144B032010F0CAF9E5
:103748000022134B1146032010F0C4F9237A012BF1
:103758000ED1617A0F4A104B002908BF1346002288
:10376800009311460D4B032010F0B4F904B010BDBE
:1037780000220B4B1146032004B0BDE8104010F0A6
:10378800A9B900BF740D00207F4B0108B04B010898
:10379800E14B01087A4B01087B4B0108EE4B01080D
:1037A800FF4B010808B5104B0122002102201A70B6
:1037B80010F0A4FA0D4810F009FD0D4B1B788BB1E1
:1037C8000C4B1A7872B9DB7C63B90B4B1A68042A64
:1037D8009EBF1A6801321A600021BDE80840102017
:1037E80010F08CBA08BD00BFBC0D0020A40D00204D
:1037F800580D00203E0E0020300C0020044B1B7892
:10380800022B03D10021082010F078BA704700BFBE
:103818000000002008B508F0EAF980B907F0A8FE12
:1038280001280CD1BFF34F8F0549064BCA6802F433
:10383800E0621343CB60BFF34F8F00BFFDE708BDC5
:1038480000ED00E00400FA0510B508F063FA10F185
:10385800080F07D1064B0022BDE810401146022090
:1038680010F038B9013001D1024BF4E710BD00BFA8
:103878000D4C0108234C010870477047022813B506
:10388800014618D0202819D001281AD14FF09040AD
:1038980004F0AAFE0022044600900B4B11460320B8
:1038A80010F018F9012C0CD10021022002B0BDE85B
:1038B800104010F023BA00210820F7E7034B01223B
:1038C8001A7002B010BD00BF3B4C0108B80E0020B2
:1038D80073B505460C46164607F05EFE03460028FB
:1038E80038D00024264810F023FC264B24481968B9
:1038F800A14238BF214610F0A3FC214802B0BDE820
:10390800704010F063BC4A68F05CD0540133DAB2FE
:10391800A242F8D31C4B0D701B78012B88BF0024E2
:103928004C701A4C637A33B107F022FE012802D199
:10393800204610F0FDFB164B1648D978002207F0F8
:1039480041FE044640B90146134B0122032010F002
:10395800C1F8C7E70F49DAE70634C2D107F002FE1B
:1039680004460028BED04FF47A730122B0FBF3F36B
:10397800002100930320094B10F0ACF8B2E700BF18
:103988008C0D002074000020340C0020280D00202D
:103998005C000020040000207F4A01088E4A0108CC
:1039A800044B1B7823B9044A05210120FFF790BF77
:1039B800704700BF340C0020594C010810B5002492
:1039C80090B03C22214601A8009410F0C3FD2F4B73
:1039D8002022DA7219788DF8001059788DF80110C4
:1039E80099788DF80210D9788DF8031019798DF827
:1039F800041059798DF8051099798DF80610D97940
:103A08008DF80710197A8DF80810597A8DF8091071
:103A1800997A8DF80A108DF80B2021460DF10B02CA
:103A280058180131007B02F8010F1C29F8D193F8CE
:103A380028208DF8282093F829208DF8292093F83C
:103A48002A208DF82A2093F82B208DF82B2093F824
:103A58002C206AB193F83F2052B10DF12B010022BE
:103A68009818013290F82C0001F8010F142AF7D1A8
:103A780007484FF40061FEF775FC20B9044840225E
:103A88006946FEF771FB10B010BD00BF780000203A
:103A980000F803080149402210F024B900F803088F
:103AA80070B52A4D28796B794D2BC0B233D1C0EB54
:103AB800001080000A2838BF0A204FF47A73584350
:103AC800234BAC791860EB794D2BE4B22BD1C4EBC6
:103AD8000414A40095F82C301E4E63BB95F83F30B3
:103AE8004BBB42F21070FFF711FC3068FFF730FC57
:103AF8002B7A194A1949DBB213706B7A184ADBB270
:103B080013700023EA1892F82C20D2B2CA54013359
:103B1800142BF7D170BD6B79482B0ABF4FF4616342
:103B28006B795843C6E7EB79482B0ABF4FF46163BA
:103B3800EB795C43CEE7FFF7E9FB012C38BF0124A2
:103B48004FF47A735C433460CFE700BF78000020FD
:103B5800740000200C000020520E00203E0E0020B1
:103B6800340C002010B590B000213C2201A800912F
:103B780010F0F0FC40223449684610F0B3F89DF884
:103B880000203AB99DF80100272803D19DF80210BA
:103B980001290FD000222D4B114603200FF09AFF68
:103BA800FFF70CFF4FF47A70FEF7CAFFFFF778FFB4
:103BB80010B010BD264B1A70587099709DF80310FC
:103BC800D9709DF8041019719DF8051059719DF868
:103BD800061099719DF80710D9719DF8081019728F
:103BE8009DF8091059729DF80A1099729DF80B10EA
:103BF80001F03F01D972D87AD1B288421BD89DF81A
:103C0800282083F828209DF8292083F829209DF86A
:103C18002A2083F82A209DF82B2083F82B200DF1E9
:103C28002B0100229818013211F8014F80F82C401E
:103C3800142AF7D1BAE701F140006844194410F892
:103C4800340C08730132D6E700F803085F4C01080A
:103C580078000020F0B50B238BB012220024012538
:103C6800CDE90632032727231721CDE9043122465F
:103C78005F4B03942146CDE90155009728460994E6
:103C88000FF028FF5B4B009522462146CDE90174D1
:103C980002200FF01FFF02260523CDE9006322460C
:103CA800554B0294214630460FF014FF534B0095B4
:103CB80022462146CDE9017430460FF00BFF09A9D1
:103CC800204607F077FF099BC3F307220292C3F34C
:103CD80007421B0E019200932246494B214630466B
:103CE8000FF0F8FE09A9284607F064FF099BDAB22D
:103CF8000392C3F307220292C3F307421B0E0192F9
:103D0800009322463F4B214630460FF0E3FE3E4BE0
:103D18003E48009422464FF4FA7110F0ABF93C4B40
:103D28003C48009422464FF4FA7110F0A3F93A4B3C
:103D38003A4800942A464FF4FA7110F09BF920464D
:103D4800FEF70CFA08B1FEF7B5FC354B00940022DB
:103D58004FF4FA61334810F08DF9334A00210120FD
:103D680010F088F8314A0021022010F083F8304A18
:103D78000021042010F07EF82E4A0021082010F0BF
:103D880079F800F005FC2C492C4807F0C9FE2C48AE
:103D980007F0B6FD214810F019FA2A4B00211878CF
:103DA80007F004FB28490094284B0968284800229A
:103DB80010F060F9264810F009FAFFF7D3FE254AFB
:103DC8000021102010F056F8234A00214FF480708B
:103DD80010F050F8214B22481968224B0094002219
:103DE80010F048F91E4810F0F1F90BB0F0BD00BF13
:103DF800A14C0108E84C0108094D01082A4D0108A9
:103E08004B4D01086C4D0108B5320008740D0020B7
:103E180083380008400D002081380008280D002054
:103E2800053800085C0D002001B700080D350008B2
:103E380051380008953400080000030110000020E4
:103E48005C0000200000002074000020F53200080B
:103E58008C0D0020A5310008213200080C0000203C
:103E6800A40D0020AD37000810B50024A2B07C22B4
:103E7800214603A8029410F06DFB53238DF80830F7
:103E880040F22713ADF80A3001238DF80C30ADF855
:103E98000440FEF7D3FD00B200EB400000EB4010F9
:103EA800FE23B0FBF3F08DF80D0001A800F004FD2F
:103EB800A0B958238DF80E300724302280211448E9
:103EC80010F048FB224602A9114810F07CFB104A6A
:103ED80021460120FFF7FCFC22B010BD430001334E
:103EE8008DF80E308DF80F0000F0BEFE094B1A68F1
:103EF80012128DF810201A688DF811205A685B6824
:103F08008DF8133012128DF812200C24D5E700BF5B
:103F1800BD0D0020E40E0020F0B50378592B95B0B4
:103F2800044640F01E8205295FD84378443B162B8F
:103F38005BD8DFE813F041015A0031015A0039011A
:103F48005A005A005A005A009A005A001C015A0096
:103F58005A005A00B9015A005A00BE005A005A00C5
:103F68005A0017008578482D17D1C34A142101201B
:103F7800FFF7AEFC41F28830FEF7E2FD0022BF4BAE
:103F8800114603200FF0A6FD40F6B830FEF7D8FD25
:103F980015B0BDE8F040FFF73DBC532D0ED13022DF
:103FA8008021B74810F0D6FAFFF75EFF41F288305B
:103FB800FEF7C6FDB24A152101208FE0432D16D128
:103FC800002404A88DF8104007F012FCAC4A4C23DA
:103FD8001370272393709DF81030547001204133DB
:103FE800D07013710521FFF773FC15B0F0BD442D97
:103FF800FBD1A34C592323705A236370A57000F09A
:104008003DFC2C228021201D10F0A4FA00232570ED
:10401800637001252723A370E5702571FEF70EFD57
:104028009849FE23B0FBF3F00B6864229BB2B3FB04
:10403800F2F3A3710B6800EB400000EB40109BB259
:104048006071B3FBF2F002FB1033E3714B689BB273
:10405800B3FBF2F323724B689BB2B3FBF2F102FBA2
:104068001133637222460A21A6E78378303BDBB21C
:10407800092BBAD8844C854A23702378DBB2537253
:104088007F4A592313704D2353702378303393702C
:1040980003210120FFF71CFC2378009300227C4BAE
:1040A800114601200FF016FD15B0BDE8F040FFF7EE
:1040B80085BC8578482D16D1714A56231370002384
:1040C80053702723937003231371172353710B2302
:1040D800012093711223D070D371082115B0BDE867
:1040E800F040FFF7F5BB432D7FF47FAF644C002110
:1040F8003C2205A8049110F02DFA04A8FFF7CAFC89
:104108002422802104F10C0010F024FA9DF81030CC
:1041180063709DF81130A3709DF81230E3709DF81C
:10412800133023719DF8143063719DF81530A37115
:104138009DF81630E3719DF8173023729DF81830FA
:10414800257063729DF81B509DF81930A3729DF875
:104158001A30E3722A4607A9257304F10D0010F0FE
:1041680032FA05F10D012246C9B201203BE78078F9
:1041780039280CD83038C0B2FFF760F8404A2378A5
:10418800137063785370A3789370032114E715B004
:10419800BDE8F040FFF704BC80783928F7D83038FC
:1041A800C0B2FFF750F8E9E780783928EFD83038FF
:1041B800C0B2FFF74DF8E1E78378303BDAB2092A5D
:1041C800E5D8C578303DEAB2092AE0D80179A1F1ED
:1041D8004802D2B20B2ADAD82E4840FA02F2D007A7
:1041E800D5D40A224D2902FB03553FD13C235D4318
:1041F800294B4FF47A7068431860284B1860FFF712
:1042080085F81F4A2378137063785370A3789370E6
:10421800E378D3702379137105210120FFF758FB48
:104228001A4B272200261E705A7001229A70DA70E3
:10423800A178303901EB8100E178303901EB400198
:10424800C9B2197122795A71154A1278D2B21A7202
:104258000D4A1278D2B25A72FFF7B0FB114B009593
:104268003246314603200FF035FCBEE64829BFD15F
:104278004FF46163BBE700BF904D0108A54D0108ED
:10428800BD0D0020E40E0020340C00207800002032
:10429800C74D0108DEF7FFFF740000200C00002066
:1042A800520E0020F04D01088378303BDAB2092A1B
:1042B8003FF66DAFC578303DEAB2092A3FF667AFE1
:1042C8000179A1F14802D2B20B2A3FF660AF7348D8
:1042D80040FA02F2D2073FF55AAF0A224D2902FBF3
:1042E800035539D13C235D436D4A4FF47A736B43D0
:1042F80013601068FFF72CF86A4A23781370637804
:104308005370A3789370E378D370237913710521E0
:104318000120FFF7DDFA644B272200261E705A7031
:1043280001229A70DA70A178303901EB8100E178C6
:10433800303901EB4001C9B299712279DA715B4ACF
:104348001278D2B21A725A4A1278D2B25A72FFF757
:1043580035FB584B009583E74829C5D14FF4616375
:10436800C1E7502B5DD102297FF63FAE4378303B41
:10437800012B3FF63AAE8378312B7FF436AE0B290A
:1043880004D8FFF70DFB0021464A15E6464D4A4F73
:104398000234002614F8012FA919303AD2B20A7350
:1043A8000B7BCDE9026323780022CDE90063114637
:1043B8003B46032001360FF08DFB0C2EEAD1FEF7A9
:1043C80069FF384B50221A7027229A700024012264
:1043D8005C70DA7003F8042F2A190134127B0C2C54
:1043E80002F1300203F8012FF6D1002250231146C2
:1043F80000930320314B0FF06DFB00232B70272314
:104408006B700123AB70EB70284B1B78DBB22B72FF
:10441800274B1B78DBB26B72EC72FFF7CFFA1121D6
:10442800B2E7412B7FF4E1AD4378432B7FF4DDAD58
:1044380016297FF4DAAD224D421C002312F8011F21
:10444800E9540133142BF9D1FEF778FE1D4B5B7D3F
:10445800012B19D114490023EA5CC8180133D2B2E0
:10446800142B80F82C20F7D1114B00221A701B78DE
:10447800DBB24B72FFF7A2FA0A4A631E15349C425C
:1044880006D1084A162197E5094B02221A70F3E76C
:1044980013F8011F02F8011BF1E700BFDEF7FFFF69
:1044A8000C000020BD0D002078000020520E0020D6
:1044B800340C0020274E0108724E01089A4E01085C
:1044C8003E0E0020A40A002070B5054686B00C46B2
:1044D80000293BD028480FF079FE2678EEB1002D50
:1044E80048D068682E78C0B1032E0BD0392E2FD053
:1044F800022E12D1697801290FD00B060DD4FFF7CF
:104508000BFD0AE06B78012B07D10078012802D057
:10451800022800D008B907F021F9237C052B15D80B
:1045280094F90A20059294F909200492134A52F842
:104538002330039394F90830CDE901630022E3683E
:10454800009311460E4B03200FF0C4FA06B070BD5D
:104558006B78012BE1D102780A4B02F001021A7044
:104568002AB9094B114603200FF0B4FAD5E7074BD7
:104578000022F7E72E46D0E7400D0020204F010823
:10458800C84E0108270D0020B54E0108BF4E01088E
:10459800034B0022C3E902220122C3E9002270472B
:1045A800540E002000487047540E00204FF0B043CE
:1045B80082B0DA6C0243DA64DB6C03400193019B3E
:1045C80002B070472DE9F04186B000240220154D55
:1045D8000594FFF7EBFF0420FFF7E8FF124F039461
:1045E8004FF4807601230DEB0001CDE901632846E5
:1045F800032304934FF4005803F0D6FE01A938466C
:10460800CDF8048003F0D0FE22464146384603F038
:10461800F1FF28462246314603F0ECFF204606B05B
:10462800BDE8F0810004004800080048032810B5E0
:104638000ED8012810D868B902460B484FF480718B
:1046480003F0D8FF002209484FF4005103F0D2FFCD
:10465800002010BD0122F0E7002203484FF48071CA
:1046680003F0C8FF0122EEE70004004800080048F4
:1046780002207047002070470120704700280CBFB7
:104688000F201620704700000D48854602F0A8FE4E
:104698000C480D490D4A002302E0D458C450043395
:1046A800C4188C42F9D30A4A0A4C002301E013606B
:1046B8000432A242FBD30FF055FFFDF7E7FFFEE7F8
:1046C8000000012000000020BC0800201C5D01083B
:1046D800BC080020BC2C0020FEE74FF0B04382B09D
:1046E800DA6C42F00102DA64DB6C03F00103019337
:1046F800019B02B07047000030B587B0FFF7EDFFAF
:104708004FF4805101224FF0904003F073FF0122D3
:104718004FF400614FF0904003F06CFF4FF4C05528
:104728001123CDE9015301A901234FF090400393D0
:1047380003F03AFE08240A2500224FF480514FF076
:10474800904003F057FF0120FEF7FAF901224FF4D9
:1047580080514FF0904003F04DFF0120FEF7F0F933
:10476800013DE9D14FF400614FF0904003F03CFF68
:1047780008B9013CDFD14FF400614FF0904003F0DD
:1047880033FF68BBFFF7A9FF04240123039001A9A5
:104798002A48CDE9014303F007FE284C01220421F1
:1047A800204603F027FF2120FEF7CAF90022042142
:1047B800204603F01FFF2120FEF7C2F90122042141
:1047C800204603F017FF2120FEF7BAF92046002201
:1047D800042103F00FFF4FF42570FEF7B1F9DDE770
:1047E800FFF77BFF4FF0B04300249A6D42F480023C
:1047F8009A659B6D03F4800300934FF4C052009BAD
:104808001223CDE901230323CDE9034304230DEB50
:1048180003014FF09040059303F0C6FD084809498D
:10482800094B8460C0E900130123C0E90334C0E9DF
:104838000744446104F052F807B030BD0004004852
:10484800640E0020005800401A091020FFF754BFDA
:1048580010B1012809D0704701394A424A414FF046
:1048680090404FF4007103F0C5BE4B1E5A420248F7
:104878005A410821F7E700BF0004004808B50120A5
:10488800FEF7DCFC6420FEF75BF900F0EDF9BDE80B
:1048980008400120FEF7D7BC054B1A6802805A6809
:1048A8009B684381034B028101221A70704700BF45
:1048B800E40E00203D0E002037B5044600F016F83F
:1048C80010F0FF051CBFEE232370AA236370019329
:1048D8000022237800931146034B01200FF0FAF8C9
:1048E800284603B030BD00BF384F01082DE9F04F0E
:1048F8000025484E484C356089B029462846FFF7C0
:10490800A7FF29460120FFF7A3FF29460220FFF74A
:104918009FFFDFF80881DFF80891424F94F864019F
:10492800522301214FF0000A84F86031C4F868A1CD
:10493800FFF78EFF0320FEF703F952468821204631
:1049480002F0B4FC0DF11E02C021204602F0FCFC6E
:10495800024650B1344B5246114603200FF0BAF8C4
:104968000021E8B2FFF774FF3DE0BDF81E304EF6B7
:10497800AA618B424AD14FEA450A0AF1540A5FFA02
:104988008AFA05905146204600F0F6F9834610B1A0
:10499800264B059AE0E70DF11E02C021204684F857
:1049A80060A102F0D1FC824610B1214B5A46D3E7F0
:1049B800204600F0A5FB0246F0B9316801231944EE
:1049C80031603968C4F86831AB400B433B600293EF
:1049D80094F860310193D4F8643100930146154B83
:1049E80003200FF077F80135032D04F5C87495D12D
:1049F800306809B0BDE8F08FBDF81E30009352460C
:104A08004B46114603200FF065F8A9E7009343468B
:104A1800F7E700BFDC0E0020BC000020FF4F0108B4
:104A2800E44F0108D80E00204D4F01085F4F0108E0
:104A3800824F01089B4F01082DE9F04F4FF4804346
:104A480087B04FF49012CDE90232684CDFF8A0A18C
:104A5800DFF8A0B105464FF00A094FF00E0848F2FA
:104A6800E8070026D4F86831002B00F0AE80002259
:104A7800614B0096114603200FF02CF8204600F0F9
:104A880033FE28B100225D4B114603200FF022F8B7
:104A98000DF112020DF11101204600F0DFFB28B1E3
:104AA80000225346114603200FF014F80DF11302AB
:104AB80005A9204600F01DFF28B10022504B1146E1
:104AC80003200FF007F80021204600F059F928B11B
:104AD80000224C4B114603200EF0FCFF012200215E
:104AE800204600F011FA28B10022474B1146032056
:104AF8000EF0F0FF01221146204600F005FA28B119
:104B08000022414B114603200EF0E4FF022D65D828
:104B18003E4B33F8153002933D4B53F82530039341
:104B28003C4B53F825703C4B13F805803B4B13F86E
:104B38000590029A0121204600F031FA28B100229E
:104B4800374B114603200EF0C5FF039A002120467B
:104B580000F025FA28B10022314B114603200EF04F
:104B6800B9FF3946204600F025F928B100222D4B1F
:104B7800114603200EF0AEFF42460021204600F009
:104B88001BF928B100225B46114603200EF0A2FF54
:104B98004A460121204600F00FF928B100225B4661
:104BA800114603200EF096FF0DF112020DF11101CE
:104BB800204600F053FB28B100225346114603203B
:104BC8000EF088FF0123C4F87C310136032E04F56A
:104BD800C8747FF447AF07B0BDE8F08F0022124BCE
:104BE800114603200EF076FFA3E700BFBC000020AB
:104BF800565001084F510108115001083B50010857
:104C08007C500108A5500108C35001080A52010848
:104C1800105201081C520108285201082B520108A1
:104C2800F550010818510108E750010810B50B7E2E
:104C38009BB9D0F87C21098912B1C0E95E1310BD77
:104C4800084BD0F878411A68C2F580734B4304FBCF
:104C580002331B12C0F87831F1E70123C0F87C3128
:104C6800EDE700BFB80000202DE9F04FDFF8E8A01D
:104C78003A4E85B0FFF7EAFDDAF800300BB1336839
:104C88004BB9FFF733FE00223060354B00901146D8
:104C980003200EF01FFF3368324D0024A3422C601E
:104CA8006C60AC6051DDDFF8C080304EDFF8C0B01A
:104CB8000220FFF7C1FE88F80040D6F86831012BC2
:104CC8002CD103FA04F90A272949304600F06CFC74
:104CD800B0B959463046FFF7A9FF9BF818307BB9A1
:104CE800D6F8783145F82430DAF8003043EA090379
:104CF800CAF8003098F8003043F0010388F8003013
:104D08000120FDF71DFF9BF818300BB3013F17F08A
:104D1800FF07D9D14FF47A7345F8243005200134C0
:104D2800FDF70EFF032C06F5C876C6D198F80030BB
:104D38005BB12B686A68A9680093CDE9012100225C
:104D48000C4B114601200EF0C5FE05B0BDE8F08FF2
:104D5800D6F87831E0E700BFD80E0020E00E00203A
:104D6800EB510108E40E00203D0E0020BC0000209D
:104D7800BC0E00209C5101084A088A2102F096BA0C
:104D8800152906D8044BCB40DB0702D50174002057
:104D980070476FF0070070470B00300010B50A46E7
:104DA8000C46092102F0A4FA18B9237803F001038C
:104DB800237010BD01F06BBE01F053BD01F04DBE74
:104DC800F7B500230C46174601210DF107020646E8
:104DD8008DF8073002F08CFA0546D8B9012F9DF8F6
:104DE800073026D1042C3AD8DFE804F003171A1D3F
:104DF800200043F01004A3420CD022460121304683
:104E080002F054FA054628B9716986F830413046EF
:104E1800FFF7D0FF284603B0F0BD43F02804EAE7C7
:104E280043F00404E7E743F04004E4E743F0800478
:104E3800E1E7042C13D8DFE804F00306090C0F009F
:104E480003F0EF04D7E703F0D704D4E703F0FB043B
:104E5800D1E703F0BF04CEE703F07F04CBE76FF0A0
:104E68000305D7E713B500230C460DF1070201210E
:104E78008DF8073002F03CFA78B99DF80730C3F393
:104E880000122270C3F3C002A270C3F380026270E2
:104E9800C3F38012DB09E270237102B010BD37B58D
:104EA8000D460DF10202F821044602F04DFA70B9E0
:104EB80001AA0421204602F067FA40B9BDF8022091
:104EC8001AB1019BB3FBF2F32B602B68A36103B00B
:104ED80030BD037F0B700020704737B50D460DF1CC
:104EE80006022021044602F02FFA28B9BDF8063040
:104EF80023B9236A2B60207703B030BDDB002B6019
:104F0800236201232377F7E70529F8B504460E46FF
:104F1800154635D862B100EB810301215A6B002395
:104F2800701E042807D8DFE800F00E171A1D2400A9
:104F380011460123F4E784F828103444E5B984F8CD
:104F48002850002007E0C2F34F224421204602F0F7
:104F5800BDF90028F1D0F8BD84F82A10EDE784F8EF
:104F68002B10EAE75B00FE226021204602F0D5F90B
:104F7800EFE71B01EF22F7E7012384F82830E0E789
:104F88006FF00300E7E7052996BF4018002390F863
:104F98002830137094BF00206FF00300704770B57D
:104FA8004318044693F828000E46154618B904EB32
:104FB8008106726370BD05291BD8DFE801F003097B
:104FC80012141616626304EB860400206563F1E789
:104FD800C2F34F224421204602F078F90028E9D193
:104FE800F1E7E263EFE72264EDE7C2F34F226421C1
:104FF800F1E76FF00300DDE737B5044615460529EC
:105008002CD8DFE801F0030717191B1B436B2B6033
:10501800002021E00DF10602442102F095F9D8B9EB
:10502800BDF8062053029AB12B60A363012384F8CC
:10503800293011E0C36BEAE7036CE8E70DF10602DB
:10504800642102F081F938B9BDF806305B02DEE769
:10505800A36B2B6084F8290003B030BD6FF0030008
:10506800FAE737B50D460DF107020121044602F0B3
:105078003FF938B99DF8073084F83031DB092B70D7
:1050880084F84C3003B030BD2DE9F843037C0C465E
:1050980001F8083B0546FFF702FF40BB207304F107
:1050A80010012846FFF719FF08BB04F11401284630
:1050B80000F021FCD8B904F1240705F1270904F10F
:1050C800170806463A46B1B22846FFF795FF70B969
:1050D800013619F8013F08F8013F062E07F10407C9
:1050E800F0D104F13C012846FFF7BBFF08B1BDE849
:1050F800F883211D2846BDE8F84301F030BD0000C3
:10510800F0B50022054693B0882102F0CFF84FF49D
:105118007A72A5F852214FF4C872A5F854214C4A66
:10512800C5F8582100234B4A85F8F030C5F8D4203B
:105138002B6202A92846FFF7A7FF044670B9ADF80D
:10514800080002AE0FCE05F110070FC70FCE0FC72C
:105158000FCE0FC796E80F0087E80F003E4BC5F843
:1051680034314FF4FA730126A5F838314FF420632F
:10517800A5F83C313246802185F85061284602F076
:1051880095F832460746FF21284602F08FF800229C
:1051980011460743284602F089F83C4364B20443A9
:1051A8000DF107029121284602F0A2F864B29DF899
:1051B800073085F83A31044332460021284602F088
:1051C80075F864B204430022FF21284602F06EF805
:1051D80064B2044300228021284602F067F864B2D2
:1051E800204340B2002488BBA1B2012228460134E2
:1051F800FFF78AFE062CF6D140BB044668850246B6
:1052080004212846FFF780FE00BB024605212846F8
:10521800FFF77AFED0B94FF490136B634FF48042D6
:1052280001212846FFF7BBFE80B94FF40C13FF227B
:10523800C5E90F3085F830210121284602F036F8FB
:10524800012385F8323108B985F8154113B0F0BD4E
:10525800856B0100A470090064008403012300F039
:1052680079BD2DE9F0428EB00C460C2304AA142116
:10527800054602F005F8844600286CD19DF81A30DE
:105288009DF81B609DF817209DF81810A07506EB77
:1052980003269DF81630206002EB03229DF8193092
:1052A800606003EB01239BB25B029DF8121023613F
:1052B8009DF81330B5F8520103EB012392B2520264
:1052C8009BB2E260A382B0F57A7F9DF8101095F842
:1052D8003171B6B20AD0704300F5FA704FF47A769D
:1052E800B0FBF6F02E7F002E39D186B2002F40D0C9
:1052F800B001C0B2B608E0750DF10F002681CDE906
:105308000040284601F086FE844620BB9DF80FE049
:1053180084F818E005F150060FCE07AF0FC796E8DE
:105328000700E37D87E80700D4E90301A28AADF806
:105338003020D4E90149CDE90A01CDE9084907AC93
:105348008DF833308DF834E00FCC50350FC597E821
:10535800070086E8070060460EB0BDE8F0822E8C94
:105368005E43B2EB262F4FEA262C04D157B948F6F4
:10537800E0260020BFE780B25043A2EB0C06B0FB4A
:10538800F6F0B2E742F2B826B2E70000F7B51746E2
:105398000E210DF106021D460B4C064601F0D4FF06
:1053A800BDF8063004EA43433B6050B90DF10602EC
:1053B8000C21304601F0C8FFBDF8063004EA43442A
:1053C8002C6003B0F0BD00BF0000FE1F73B590F85D
:1053D800DA30013B022B06460C4634D801AB6A464C
:1053E8000121FFF7D3FF009BB3F57F0F054603D8D4
:1053F800019BB3F57F0F23D915BB34B11349304650
:1054080002B0BDE8704001F00FBC0422FF21304615
:1054180001F04CFF2A4604467021304601F046FF51
:105428002A460443FF21304601F040FF64B204439A
:105438002A468021304601F039FF64B2044365B240
:10544800284602B070BD0025FAE700BF5F060020BD
:1054580037B5044601228021057C01F027FF01228F
:10546800FF21204601F022FF00221146204601F0CC
:105478001DFF94F83A219121204601F017FF0122DF
:105488000021204601F012FF0022FF21204601F0F2
:105498000DFF00228021204601F008FF012D29D0B0
:1054A800032D37D0002D3CD101222946204601F09A
:1054B800FDFE01238DF80730A0B103B030BD0146D1
:1054C8000DF10702204601F013FF9DF80730DB07B6
:1054D80005F1010508D538B9B5F5FA6FEFD16FF0C8
:1054E8000600EAE70546F0E7B5F5FA6F08BF6FF082
:1054F8000600E2E718B929462046FFF767FF0222AF
:105508000021204601F0D2FE0028D6D1042384F8D9
:105518003231D2E718B901212046FFF757FF04229C
:10552800EEE76FF00700C8E738B5057C044625B1FB
:10553800204600F054FD28B138BDFFF789FF002848
:10554800F6D0F9E7002DF7D1032384F83231F3E7D9
:1055580073B50646002501220B21304601F0A6FE50
:10556800002204460B21304601F0A0FE0DF107028F
:1055780004431321304601F0BBFE9DF8073064B2A6
:10558800044301355B0760B2EDB205D0032D08D0A6
:105598000028E0D002B070BD032D08BF6FF00B00EB
:1055A800F8E76FF00B00F5E738B5002303740446FD
:1055B8000D46FFF7B9FF50B929462046FFF751FEBF
:1055C80028B901462046BDE83840FFF7C1BF38BDBD
:1055D800152970B5054616461C4667D10122FF21DC
:1055E80001F064FE002211460446284601F05EFEE2
:1055F80000220443FF21284601F058FE64B2044308
:1056080001228021284601F051FE64B2044302229F
:105618008521284601F04AFE64B204430422FF2192
:10562800284601F043FE64B204430022CD212846F7
:1056380001F03CFE64B204431122CC21284601F05B
:1056480035FE64B204430722FF21284601F02EFEEE
:1056580064B204430022BE21284601F027FE64B24A
:1056680004430622FF21284601F020FE64B20443C9
:105678000922CC21284601F019FE64B20443002215
:10568800FF21284601F012FE64B204430122FF21E3
:10569800284601F00BFE64B2002204431146284656
:1056A80001F004FE64B2204340B270BD042A17D84A
:1056B8000A2101F0FBFD0028F7D1231E18BF0123A2
:1056C8001B01EF228421284601F027FE0028ECD197
:1056D80085F8DA6001462846BDE87040FFF738BF14
:1056E8006FF00A00E1E7000070B594B0054640226B
:1056F800002104A80EF02EFF002301212846ADF852
:1057080006308DF803308DF80430029300F0B8FCB1
:1057180095F8142195F81311012A04D840F0AD80AA
:10572800202940F2AC8001AA02A9284600F02DFBEE
:105738000446002840F09E8095F85031002B40F038
:10574800A280D5F84C11284601F06EFA04460028CC
:1057580040F090802346214604222846FFF738FF70
:105768000446002840F086800122FF21284601F0E7
:105778009DFD0DF1060206468421284601F0E4FD50
:1057880022460643FF21284601F090FD76B20643E3
:1057980074B2002C6ED1BDF806301B01C5F8D430A8
:1057A80004A92846FFF770FC0446002862D10DF1D1
:1057B80003012846FFF7F2FA044600285AD19DF85B
:1057C800033085F8313104AE0FCE05F110040FC453
:1057D8000FCE0FC40FCE0FC496E80F0084E80F0059
:1057E8000DF103020121284601F082FD044600283C
:1057F80040D19DF8033085F83031024601462846ED
:10580800FFF7DEFA0446A8BB024602212846FFF746
:10581800D7FA044670BB0323014685F832310DF1EF
:105828000502284601F019F9044618BB9DF8053011
:1058380085F8E8300DF105020121284601F00DF93F
:105848000446B8B99DF8053085F8E03003AA03216D
:10585800284600F001FF044660B9039BC5F8E43010
:1058680003AA0421284600F0F7FE044610B9039B5A
:10587800C5F8DC30204614B070BD0C2951E7284625
:1058880000F010F954E701495DE700BF6C050020FE
:1058980013B50C460DF10702132101F029FD9DF8FF
:1058A800073013F0180F03F0070218BF6FF0050058
:1058B800226002B010BD13B590F8DA30042B0C4604
:1058C8000BD101A9FFF7E4FF019B042B01D10123B0
:1058D80000E00023237002B010BD01AA142101F0DA
:1058E80007FD0028F7D19DF80430DB07EFD42070BE
:1058F800F1E700F04ABA13B50C460DF1060228216B
:1059080001F022FD78B9BDF80620C2F30B0312F4AA
:10591800006F18BFA3F580534FF0FA0214BF13FBB2
:1059280002F35343236002B010BDF0B54FEAD20C26
:105938004FF0FF341C6002F00702664600278E42D3
:1059480000D207B1F0BD845D664503BF1441E4B2DF
:1059580015463D4614F0010704D005EBC6051D6049
:105968000136ECE70135082D4FEA5404F2D1F7E788
:10597800034B800953F82000003818BF01207047F6
:105988001808002010B5B1EBD20F4FEAD20402F08C
:10599800070381BF01229A40035D13438ABF035561
:1059A8006FF03100002010BD0A460623B02101F037
:1059B80049BC0A460623B02101F062BC2DE9F04F2C
:1059C80085B08046109E0E9D01968A4693461C46D9
:1059D8004FF00009119B994508D10023129A1660CF
:1059E800F3B16FF0310005B0BDE8F08F01AB32467E
:1059F80029465846FFF799FF019F7B1C0DD00F9B46
:105A0800F818FFF7B5FF504507D13A462046FFF78B
:105A1800B9FF7E1C09F10109DCE76FF03103DDE70E
:105A280021464046FFF7C0FF0028DCD102A94046C6
:105A3800FFF7BFFF2544234602AAAB42D3D013F891
:105A4800014B12F8011B8C42F7D0CAE770B5C0228F
:105A580088B00E46012190F83041054601F026FC39
:105A6800F0B901A92846FFF79FFDC8B90122FF2117
:105A7800284601F01BFC98B93246B621284601F0A9
:105A880063FC68B90246FF21284601F00FFC38B9CB
:105A980022460121284601F009FC08B985F8304161
:105AA80008B070BDF0B50F4689B01646FF21012237
:105AB800044601F0FBFB0246A8B94F21204601F03D
:105AC800F5FB80B92C224E21204601F0EFFB02465F
:105AD80048B9FF21204601F0E9FB20B9B422B621DC
:105AE800204601F0E3FB0025C4F82451A4F828510E
:105AF800DEB9354607ABB422CDE903730623CDE9F9
:105B08000032029504F5927304F5957231462046E9
:105B1800FFF754FF30B9012384F8153184F8137165
:105B280084F8146109B0F0BD013505F1B400FFF740
:105B38001FFF0028DED12C2DF6D1DBE710B541F090
:105B480001020021044601F0B1FB78B9204600F0BB
:105B580046FA58B901462046FFF7FAFC30B9024622
:105B680001462046BDE8104001F0A0BB10BD2DE95C
:105B7800F74F4FF0000B88461746FF2101220546D4
:105B88001E469DF838A09DF83C908DF807B001F0AE
:105B98008DFB5A4604465946284601F087FB5A466B
:105BA8000443FF21284601F081FB64B2044364B238
:105BB800B8F1000F32D0BAF1000F06D00C9ACB2101
:105BC800284601F095FB204344B2B9F1000F07D0F5
:105BD8000DF10702EE21284601F08AFB204344B26A
:105BE8000122FF21284601F061FB01220443002124
:105BF800284601F05BFB64B204430022FF212846DB
:105C080001F054FB64B29DF807300D9A204323F04D
:105C1800100340B2137003B0BDE8F08FBAF1000F63
:105C280006D03A46CB21284601F040FB204344B237
:105C3800B9F1000FD4D033468022EE21284601F076
:105C48006CFBCBE72DE9F04387B09146002205466F
:105C580088468DF817201E461BB390F83071012234
:105C68001146284601F022FB044658BB402128462D
:105C7800FFF764FF044628BBB9F1010F13D10DF1FA
:105C88001703CDE90290CDE9008302460346494651
:105C98002846FFF76CFF40B10446204607B0BDE830
:105CA800F0831F46DBE788F80000002EF5D03A465F
:105CB8000121284601F0FAFA04460028EDD185F8BA
:105CC8003071EAE7002388F800302046E4E72DE940
:105CD800F043054687B0884691461E4623B390F8A0
:105CE800307102220121284601F0E0FA044660BB27
:105CF80001462846FFF722FF044630BBB9F1010FE1
:105D080014D10DF11703CDE90209009302460346A9
:105D1800CDF8048049462846FFF729FF40B10446DC
:105D2800204607B0BDE8F0831F46DAE788F8000090
:105D3800002EF5D03A460121284601F0B7FA04466C
:105D48000028EDD185F83071EAE7002388F80030A3
:105D58002046E4E7F8B51D46164600232A4690F883
:105D680030710446FFF76EFF70B903462A46314684
:105D78002046FFF7ACFF38B93A460121204601F02A
:105D880095FA08B984F83071F8BD2DE9F04F002371
:105D980093B0CDE90A12C0F82431A0F828310122C5
:105DA800FF21CDE90E33B0F83C818DF8343005463B
:105DB8008DF8353001F07AFA0446002840F0E38087
:105DC80002464F21284601F071FA0446002840F0A7
:105DD800DA802C224E21284601F068FA0446002871
:105DE80040F0D1800246FF21284601F05FFA0446C0
:105DF800002840F0C880B422B621284601F056FA9F
:105E08000446002840F0BF8002468021284601F061
:105E18004DFA0446002840F0B68003460DF13502DD
:105E28000DA92846FFF796FF0446002840F0AB80EE
:105E38000323CDE90203B421062305F5957A05F578
:105E480092790EAECDE90031049601464B46524692
:105E58002846FFF7B3FD0446002840F094800DF172
:105E6800360128460E9FFFF7F1FD0446002840F052
:105E78008A80BDF83630434540F2AA80C5F824012F
:105E8800A5F8280107F1B400FFF772FD08B92B2F18
:105E98007DD90623B4224FF0030BCDE90032CDE9BA
:105EA800027B04964B46524601212846FFF786FDA1
:105EB800002840F08B800DF1360128460E9FFFF731
:105EC800C5FD064600287CD1BDF83630434540F272
:105ED800828001260696BDF83630434560D2A3EB92
:105EE800080383EAE372A2EBE3729DF81860099253
:105EF80005F592734FF0030B0793079B18689B886F
:105F08001090ADF844303A460FAB06215046FFF7E3
:105F18000CFD0F9F7B1C56D007F1B400FFF728FD3E
:105F2800069B98423CD10BF101033A464846089338
:105F3800FFF728FD002849D149462846FFF734FDD8
:105F4800002843D10DF136012846FFF77FFD0028D0
:105F58003CD1BDF83620A2EB0803002BB8BF5B424A
:105F6800424516D9099A934218D910A92846FFF72D
:105F78001BFD079A0799034610981060BDF8442046
:105F88008A806BB11C46204613B0BDE8F08F0137FC
:105F980078E7DDF820B009930137AEE7DDF820B0E7
:105FA8000A9BC3F800B00B9B1E70012385F81531BE
:105FB8000A9B1B6885F813310B9B1B7885F81431F5
:105FC800E1E70446DFE76FF03104DCE70446DAE78F
:105FD8000026B3467EE70123834606937BE737B561
:105FE800002304468DF807304FF4FA650DF10701D8
:105FF8002046FFF760FC58B99DF80730012B07D001
:10600800013D03D0204601F0E5F9EFE76FF0060007
:1060180003B030BD02464FF08043934202D80020BF
:1060280013B970479B08F8E7C11891424FEA50002E
:106038009CBFC018521A9B08F2E773B5002283214F
:10604800054601F033F9044688B94FF4FA660DF1B4
:1060580007028321284601F04BF99DF807300343D6
:10606800DBB204461BB9013EF1D16FF006040122F0
:106078008321284601F01AF9204340B202B070BDCE
:106088002DE9F04F90F8F06091B04FF00009072E1D
:10609800CDE9079904460F4600F0A282012280212B
:1060A80001F004F901228046FF21204601F0FEF8A4
:1060B8004A4648EA00084946204601F0F7F84FFAF0
:1060C80088F848EA00080622FF21204601F0EEF889
:1060D8004FFA88F848EA00080DF115028321204696
:1060E80001F006F99DF815204FFA88F848EA0008EB
:1060F80042F004028321204601F0D8F84FFA88F8CC
:1061080048EA00080722FF21204601F0CFF84FFA9D
:1061180088F80122812148EA0008204601F0C6F8E3
:106128004FFA88F848EA0008204601F053F94FFA78
:1061380088F848EA000801228021204601F0B6F8D4
:106148004FFA88F848EA000517F0010B6DB200F025
:106158001E82F20700F11E826B229421204601F074
:10616800A5F880462046FFF768FF06AA48EA000817
:106178009021204601F008F945EA0805069B6DB212
:106188002422942105432046C3F3062AC3F3C039C9
:1061980001F08CF86DB205432046FFF74EFF6DB253
:1061A800054306AA9021204601F0EEF8069B6DB241
:1061B8001BBA2522942105432046099301F076F85D
:1061C8006DB205432046FFF738FF6DB2054306AAB6
:1061D8009021204601F0D8F8069B6DB21A0E0543AF
:1061E8001B0C6DB28DF828208DF8293017F00203AA
:1061F800029300F0DB8016F0020840F0D7800222FC
:106208009421204601F052F801902046FFF715FF2F
:10621800019B0DF116020343902120461D4301F016
:1062280067F86DB27B2294210543204601F03EF8C1
:106238006DB205432046FFF700FF6DB205430DF12F
:1062480017029021204601F053F86DB2772294216D
:106258000543204601F02AF86DB205432046FFF7B2
:10626800ECFE6DB2054306AA9021204601F08CF899
:10627800069B5A0E8DF82C20C3F386428DF82D20EC
:10628800C3F3C6228DF82E206DB2C3F30612DB00CD
:1062980003F07803942105438DF82F2020467822B7
:1062A8008DF8153001F002F86DB205432046FFF76E
:1062B800C4FE6DB2054306AA9021204601F064F899
:1062C800069B9DF8152002EB53728DF83020C3F31E
:1062D80086528DF83120C3F3C6328DF83220C3F3CD
:1062E80006228DF833206DB2C3F346029B0103F0FA
:1062F8004003942105438DF83420204679228DF8F7
:10630800153000F0D3FF6DB205432046FFF795FE28
:106318006DB2054306AA9021204601F035F8069B88
:106328009DF8152002EB93628DF83520C3F3C64221
:106338008DF83620C3F306328DF837206DB2C3F3DB
:1063480046129B0003F07C03942105438DF8382006
:1063580020467A228DF8153000F0A8FF6DB205436B
:106368002046FFF76AFE6DB2054306AA9021204633
:1063780001F00AF8069B9DF815208DF83E8002EB87
:1063880093728DF83920C3F3C6526DB28DF83A2056
:10639800C3F3064205438DF83B20C3F34622C3F3FB
:1063A80086036DB28DF83C208DF83D3017F004035C
:1063B800019300F0F180730700F1EE807B229421B5
:1063C800204600F073FF80462046FFF736FE07AAF6
:1063D80048EA00089021204600F0D6FF45EA080860
:1063E8004FFA88F848EA00057C229421204600F0FC
:1063F8005DFF6DB205432046FFF71FFE6DB20543F2
:1064080008AA9021204600F0BFFF6DB273229421A4
:106418000543204600F04AFF6DB205432046FFF7CA
:106428000CFE6DB2054306AA9021204600F0ACFF91
:10643800069B6DB21B0274229421054320461FFA65
:1064480083F800F033FF6DB205432046FFF7F5FDF2
:106458006DB2054306AA9021204600F095FF6DB263
:106468009DF81B30752294210543204643EA08080D
:1064780000F01CFF6DB205432046FFF7DEFD6DB24C
:10648800054306AA9021204600F07EFF069B6DB2C8
:106498001B029BB27622942105432046039300F009
:1064A80005FF6DB205432046FFF7C7FD6DB20543F2
:1064B80006AA9021204600F067FF6DB29DF81B20C8
:1064C800039B05436DB213430022812120460393A9
:1064D80000F0ECFE06220543FF21204600F0E6FE10
:1064E8006DB205430DF115028321204600F000FF2F
:1064F8009DF815206DB2054302F0FB02832120466A
:1065080000F0D4FE6DB205430122FF21204600F0C1
:10651800CDFE6DB2054301220021204600F0C6FEE3
:106528006DB205430022FF21204600F0BFFE6DB288
:10653800054300228021204600F0B8FE6DB20543D5
:106548006DB2039BFDB9BBF1000F29D1029AAABB1A
:10655800019AAAB1720713D4079AC4F81821089AA5
:10656800C4F81C214FEA4822C4F820213BB1A3F506
:10657800C8534FF47A7253431B095B421BB2E36062
:106588003E4384F8F060284611B0BDE8F08FD94644
:10659800DA462BE6CA4629E64FF00008434693E759
:1065A800F007D3D40998BDF8282084F813A184F8FB
:1065B8001491C4F82A01A4F82E21C7E7B107C7D45B
:1065C8009DF8162084F8F1209DF8172084F8F22011
:1065D8000BA904F1F30002930DF0E8FF029BB7E763
:1065E8004D46D0E750B10138002330F0FF019AB290
:1065F80003F1010303D100EB022080B27047400889
:10660800F3E7C3B2000A03FA00F001307047000054
:10661800084B5A434FF47A7302F5FA724FF4FA6052
:10662800B2FBF0F0B2FBF3F203FB0100B0FBF2F0B7
:10663800704700BF002F3A00064B5A434FF47A7058
:1066480002F5FA72B2FBF0F24A4302F5FA72B2FBB3
:10665800F0F07047002F3A002DE9FF4102294FF072
:106668000005074616468DF80350ADF804501CD8AF
:106678000DF102022946FEF7A1FB044630B90DF1DF
:1066880003024621384600F033FE04469DF8030015
:10669800FFF7B7FF81B29DF802203846FFF7CCFF1D
:1066A8003060204604B0BDE8F081032918D10DF10F
:1066B80002022946FEF782FB0446002846D101461D
:1066C8000DF102023846FEF779FB044628B901AA03
:1066D8005121384600F038FE0446BDF80400D7E7DB
:1066E800042935D102A9FEF7BDFB9DF80B30ABB1EB
:1066F8000DF1020229463846FEF760FB044658B9F8
:1067080001AA5121384600F01FFE0446BDF80400D6
:10671800FFF777FF85B214B1002015E01D460DF193
:10672800020201213846FEF749FB04460028F3D14E
:106738000DF106027121384600F006FE0446BDF848
:106748000600FFF75EFF80B2401BA3E72846A7E7D5
:1067580028462C46A4E7F0B5022985B0054616461A
:106768001ED80DF105020021FEF728FB0446A0B94A
:106778009DF8052031462846FFF74AFF83B2B3F556
:10678800807F9ABF00F1FF32D2B2FF22A5F8D8204D
:106798004621284600F08AFD0446204605B0F0BD93
:1067A80003291FD10DF105020021FEF707FB9DF813
:1067B8000520314604462846FFF72AFF80B2FFF736
:1067C80011FF0246ADF80600A5F8D800002CE4D168
:1067D8005121284600F07AFD04460028DDD1C5F88D
:1067E800E460DAE7042939D102A9FEF73BFB9DF8FA
:1067F8000B70B7B10DF1050200212846FEF7DEFA4D
:1068080004460028C9D10DF106025121284600F09E
:106818009BFD0446BDF80600FFF7F3FE87B2002C87
:10682800BBD10DF1050201212846FEF7C7FA04463F
:106838000028B2D19DF8052031462846FFF7E8FE2A
:106848003844FFF7CFFE71210246284600F03EFD8E
:1068580004460028A1D1C5F8DC609EE76FF0030468
:106868009BE7F0B585B000238DF80330D3070546C4
:106878000F46164605D439B9A2F10C03DAB2062A36
:1068880011D96FF00300E6E0012921D1A2F1080334
:10689800DAB2062AF5D8062B1AD8DFE803F03B1936
:1068A80069198A199D00062B12D8DFE803F0041134
:1068B8002D112F11310018225721284600F0F6FC1F
:1068C80008225621284600F0F1FC002840F0C38039
:1068D8007408013CE4B2002F00F09180012FD0D160
:1068E80001AA04212846FFF7B7FE50B922467021B5
:1068F800284600F0DBFC20B9019A04212846FFF75E
:106908002AFF85F8E06099E03022D5E74022D3E7F6
:106918005022D1E71022482100F0C8FC0822472164
:10692800284600F0C3FC022204463221284600F023
:10693800BDFC0C2204433021284600F0B7FC64B2A9
:1069480004430122FF21284600F0B0FC64B204434E
:1069580064B230223021284600F0A8FC002204430B
:10696800FF21284600F0A2FC64B2204340B2ACE705
:106978002822482100F09AFC08224721284600F0E6
:1069880095FC032204463221284600F08FFC04437C
:1069980064B209223021284600F088FC0122044311
:1069A800FF21284600F082FC64B2044364B220222E
:1069B800D0E73822482100F079FC082247212846F0
:1069C80000F074FC032204463221284600F06EFCD5
:1069D800044364B20822DDE74822114600F066FC51
:1069E80008224721284600F061FC03220446322190
:1069F800284600F05BFC044364B20722CAE702AAF7
:106A080003212846FFF728FEB0B903AA0221284629
:106A1800FFF722FE80B922465021284600F046FCA6
:106A280050B9029A03212846FFF795FE20B9039A28
:106A380002212846FFF78FFE85F8E86058B9696992
:106A48002846FEF7B7F930B9024601230DF10301D4
:106A58002846FFF73CF905B0F0BD13B5144629B137
:106A6800012910D06FF0030002B010BD0DF107022C
:106A7800502100F03DFC0028F6D19DF80730013385
:106A88005B002370F0E70DF107027021F1E7F0B524
:106A9800002385B04FF4FA62CDE9002344F61F6362
:106AA800994206460F4604D86FF00305284605B0FC
:106AB800F0BD02A9FEF7D6F905460028F6D19DF8E3
:106AC80009209DF8083013439DF80A201343A7F6C0
:106AD80036341BD06A4602213046FFF7BDFD002838
:106AE8003BD19DF808302BB1009B03F24E239C420A
:106AF800DAD9E41A9DF80A3023B3009B03F2B223D3
:106B0800B4EB430F4FEA4302CED9A41A9DF80B30D9
:106B18005BB101AA03213046FFF79EFD019B03F5F7
:106B28002573A342C0D2C0B9E41A9DF80C30002BDB
:106B3800BCD0A4F2262204213046FFF70CFE776170
:106B48000546B3E79DF80930002BDFD0009B03F51D
:106B580025739C42A8D9E41AD8E70546A6E770B57C
:106B68004FF4FA6286B00023CDE9022340F63633AB
:106B78000B600C4604A90646FEF774F90546002882
:106B880036D19DF811209DF8103013439DF812203E
:106B9800134319D002AA02213046FFF75DFD0028F1
:106BA80040D19DF810302BB1029B03F24E2223688E
:106BB800134423609DF81230EBB1029B03F2B2221A
:106BC800236803EB420323609DF81330EBB99DF86B
:106BD80014305BB101AA04213046FFF73DFD019B4B
:106BE80003F22622236813442360D8B9236873610B
:106BF800284606B070BD9DF81130002BE4D0029BEA
:106C080003F5257223681344DDE703AA0321304600
:106C1800FFF722FD039B03F52572236813442360C5
:106C28000028D4D00546E3E72DE9F74300240646BB
:106C38000D46204615F80480B8F1000F00D010B1B9
:106C480003B0BDE8F083671CB8F1FF0F15F8079093
:106C580029D1A71CEB5DB9F1030F36D8DFE809F09D
:106C6800020B131B271D2C44E27802EB0323A6F822
:106C780034313C46DEE7271D2C44E27802EB03233F
:106C8800A6F83631F5E7271D2C44E27802EB0323FA
:106C9800A6F83831EDE7271D2C44E27802EB0323F0
:106CA800A6F83C31E5E7B8F1040F0ED802344246A5
:106CB800291901A80DF087FC434601AA4946304628
:106CC80004EB080700F0BEFAD3E76FF00300D0E743
:106CD80073B500230E4613600DF1070105461446EF
:106CE800FEF7F7F840B99DF807302BB1B38A2A6A46
:106CF800534380331B0A236002B070BD13B5CB68C1
:106D08001360144601AAFFF7E3FF18B92368019A34
:106D18001344236002B010BDF8B5B0F85451D0F850
:106D2800580168438030000A0E464543DDE90717DD
:106D3800144652B1B60206EB5202B2FBF4F202EB71
:106D48004202524302F50042140C069A534301F5DD
:106D58000042120C06200332B2FBF0F2C2EBC20270
:106D6800B2F5803F38BF033103F500433EBFB1FBA6
:106D7800F0F1C1EBC10101F500414FEA134334BF03
:106D8800090C1B4903FB03F338BF494303EB5703C3
:106D98000B44B3FBF7F39B03FE2205F120007F337E
:106DA800B3FBF2F35C434FF47A7704F5FA74800985
:106DB800B4FBF7F42401FFF72DF904F5FA74BC428B
:106DC80028BF4FF4FA63064629BFB4FBF3F300204B
:106DD8005B19B4FBF7F428BFB3FBF4F0FFF71AF91B
:106DE800099B864294BF1E6018600020F8BD00BF52
:106DF8000000F0FF2DE9F04F91B0CDE90723036AB9
:106E08000E930B6909930546CB680B930F460FAA9F
:106E1800FFF774FF0EAA39462846FFF759FF58BBFB
:106E28000F9C95F8E0B0D5F8DC3005934FF47A76EE
:106E380006FB04F101F5004104910E990A910499A9
:106E4800D5F8E4300693BBF1080F04F180040CBFB9
:106E58000223032324F0FF0A090C95F8E820DFF841
:106E6800A081CDF83CA00C9109D1079BC3F8008004
:106E7800089BC5F84081186011B0BDE8F08F0699ED
:106E88000D932846FFF7C4FB5A46059981462846C4
:106E9800FFF7BEFB0D9B5B490C9A814403FB09F984
:106EA8004FEAC92940F2776309F5FA79240AB9FB50
:106EB800F6F903FB09F909F5FA79B9FBF6F909FBC3
:106EC80004F404F18003099C74430C40B4FBF2F40D
:106ED8004D4A1B0A944228BF1446012B38BF012390
:106EE8000C204FF4167258435443FFF793F83B7E37
:106EF8003A894FEA400B002B7FD14249049B0B4053
:106F080003F5FA71414B5A4341F25C23B2FBF3F2A9
:106F18000A9B7343B3F5481F28BF4FF44813A1EBEE
:106F28004303B1FBF6F1B3FBF6F31B02B3FBF1F637
:106F38003602C6F58036564306F50046360C06F589
:106F4800803676087643B60B4FF44870704304F5E4
:106F5800004300F500401B0C5B43000C00FB0030B5
:106F6800FFF758F803046422323341F28837B3FB41
:106F7800F2F340F6B532B3FBFBF302FB0377244B85
:106F88009F429CBF42F21073B7FBF3F7DDE905326D
:106F9800134403F5FA734FF47A7B4FF4FA62B3FBA8
:106FA800FBF0B3FBF2F202F5C812B2FBF0F088BFB7
:106FB8004FF47047FFF72EF8000200F5FA70B0FBA7
:106FC800FBF0404307FB0700FFF724F80BFB00F03A
:106FD800079B0B9A404528BF40461860089BC5F898
:106FE8004001CDE902934FF448730093019433466E
:106FF80051462846FFF790FE3EE74FF48036A3E758
:10700800AE878F020000FFFF666666009A99060049
:107018000F279F242DE9F04F8BB0002711F0780F30
:10702800DDE914B80446019299468DF80E708DF882
:107038000F708DF810708DF81170ADF812700997F7
:10704800C1F3C30A00F0AF80AAF10503DBB20A2B33
:1070580001D86B4AD75C0DF10E0200212046FDF7DE
:1070680092FF9DF80E500646D5B1002840F09D804D
:1070780009AB05AA59462046FFF7BCFE002840F098
:107088009680099BABF80A30014606AA2046FDF710
:10709800B3FF069D25B1059B9D422CBF0025012508
:1070A80020B904AA02212046FDF76DFF9DF8106063
:1070B80026B300287DD107AA02212046FDF79CFFB0
:1070C80088B90122FF21204600F0F0F858B90DF1E7
:1070D8001202B621204600F037F920B90246FF21F6
:1070E800204600F0E3F8BDF81230079E5B02C4F8B2
:1070F80048311EB19E422CBF0026012628B90DF149
:10710800110203212046FDF73EFF9DF8113093B18F
:10711800002873D1B9F1000F03D0019B1B02B3FB08
:10712800F9F908AA03212046FDF766FF089B4B459D
:1071380094BF0023012320B9012F3CD1FF2288F8F6
:10714800002098F800200AB9ABF80A200DF10F02C8
:10715800012120460193FDF716FF08BB9DF80E207C
:10716800019B002A08BF0125BAF1040F18BF9DF83A
:107178000F2084F82E501ABFB2FA82F25209012267
:1071880084F82F209DF81020002A9DF8112008BFB0
:107198000126002A08BF012384F8306084F83130C2
:1071A8000BB0BDE8F08F012755E700257EE735468F
:1071B8007CE70026A9E70AF1FF32092A0AD8DFE8A6
:1071C80002F0050505090907090B070B0522B6E7B3
:1071D8000422B4E7012E01D10322B0E7BAF1040F6B
:1071E80001D0012B01D10222A9E7012D1BBF0023E9
:1071F80088F8003088F800502B46A2E70023A0E763
:107208002E52010807B502F10A03009393B20A4609
:1072180090F86011D0F85C0101F0B2FB03B05DF8A2
:1072280004FB13B502F10A0390F860410093D0F80B
:107238005C0193B20A4644F0010101F037FC02B048
:1072480010BD00003F2BF8B50E46054611461C46FA
:1072580011D80A4F38461A4600F8016B0DF0B3F9F9
:10726800621C39462846FFF7CDFF00280CBF0020D6
:107278006FF01300F8BD6FF00300FBE7F00E00207D
:1072880073B515468DF8071001220DF10701044664
:107298001E46FFF7B7FF28B9324629462046FFF7B2
:1072A800C0FF08B16FF0130002B070BD08B5064BFF
:1072B80019705A7019460222FFF7A4FF002814BF5C
:1072C8006FF01300002008BDF00E002008B5074B32
:1072D8001970110A59709A7019460322FFF792FF24
:1072E800002814BF6FF01300002008BDF00E002026
:1072F80037B515468DF8071001220DF10701044630
:10730800FFF780FF28B9012229462046FFF789FFA9
:1073180008B16FF0130003B030BDF7B515460DF195
:10732800070206460F461C46FFF7E2FF50B99DF8D4
:1073380007301D4044EA0502394630468DF80720DB
:10734800FFF7B4FF03B0F0BD73B514468DF807100E
:1073580001220DF107010646FFF754FF18B16FF03F
:10736800130002B070BD074D022229463046FFF7D0
:1073780058FF0028F3D12A786B7803EB0223238087
:10738800EFE700BFF00E002073B514468DF8071024
:1073980001220DF107010646FFF734FF18B16FF01F
:1073A800130002B070BD0A4D042229463046FFF78B
:1073B80038FF0028F3D16B782A781B0403EB0263AB
:1073C800EA781344AA7803EB02232360E9E700BFB5
:1073D800F00E002008B50220FBF7B2FB002008BD24
:1073E8007047000010B5032000F072FC01F0AAFD00
:1073F800064B18600F20FBF799FB044618B9FBF7FA
:10740800FCF9204610BD0124FBE700BF2808002036
:107418004FF0E022136923F00203136170474FF025
:10742800E022136943F0020313617047014BD3F85C
:10743800900570470070FF1F014BD3F89405704703
:107448000070FF1F014BD3F8980570470070FF1FAD
:10745800024A536823F0010353607047002004E098
:10746800024A536823F0020353607047002004E087
:10747800024A536823F0040353607047002004E075
:107488008068C0F380007047F7B500230193044675
:10749800002800F0E980856D25B9FAF7DFFCE5657D
:1074A80084F8545023689A68D00040F1A1809A6803
:1074B800D10000F1B480A26D42F01002A265E26D25
:1074C80042F00102E26501251846FFF7D9FFA26DD7
:1074D80002F01002024340F0C980A26D206922F434
:1074E800817242F00202A2659A68D2075DD4226BCB
:1074F800A67E94F82CC0003A18BF01221703D4E9DD
:1075080002120A43217E42EA8132617E42EAC13296
:1075180042EA4632002842EA4C02B4BF20F0004159
:107528004FF400113A430A4394F82010012903D17B
:10753800002E76D142F48032616A21B1A66A01F444
:10754800E07131430A43D968E66C21F4FE3121F435
:10755800FF711143D96094F83C206168012A01F059
:10756800404C4CEA060609D1D4E910273A43324385
:10757800A66C324342EA0C0242F001061F693E4AF9
:107588003A4032431A6121F00042B2F1804F0CD0E8
:10759800B1F1004F09D0394ED6F8082701F470111F
:1075A80022F470120A43C6F808275A69666BA16B61
:1075B80022F0070232435A615A6922F0700242EA05
:1075C80001125A61002835D19A6A62F00F029A6254
:1075D8005B6903F007039E423CD10023E365A36D7A
:1075E80023F0030343F00103A365284603B0F0BD6D
:1075F8009A68234922F0104222F0170242F0805282
:107608009A60204A1268B2FBF1F2013252000192EC
:10761800019A002A3FF44BAF019A013AF7E7002597
:1076280052E7A16D41F02001A165E16D41F0010132
:10763800E16581E7B0F5001FCAD19A6AE269013AAB
:1076480092006FF00F0102F01C0201FA02F2216EA3
:107658000A43BCE7A36D23F0120343F01003A365AC
:10766800E36D43F00103E3650125BEE7A36D43F035
:107678001003A365F8E700BF02FCFF1F00200140CC
:10768800400D030028080020F8B54569082D044678
:107698000E460AD00368DB68D80705D5A36D43F00A
:1076A8002003A3650120F8BD0425FBF741FA07462E
:1076B80023681A682A4221D0A26D42F40072A2659A
:1076C800DA6812F4406F14D1A27E92B91A681207D0
:1076D8000FD51846FFF7D4FE28BB5A6822F00C02D3
:1076E8005A60A26D22F4807222F0010242F0010277
:1076F800A265207E00BB0C221A60D4E7711CD8D08A
:10770800FBF716FAC01BB04201D8002ED0D123686F
:107718001B682B40CCD1A26D84F8543042F004028F
:10772800A2650320BFE7A26D42F02002A265E26DC8
:1077380042F00102E265DCE70020B4E70368186C58
:1077480070470000F7B50023019390F85430012BDF
:10775800044600F0C58005680669012380F85430A6
:107768002846FFF78DFE002840F0B480D1E90020BC
:10777800022826F0040300F08280B3F1004FC2F320
:10778800110E13D1AB6A43EA0E03AB628B686869CA
:1077980003EA022323F07C4323F0FF0320EA0221BB
:1077A8000B43002A6B6126DB002055E0236E00F0B6
:1077B8001F074FF00F0C0CFA07FC6FEA0C0623EAC0
:1077C8000C0CBEF1000F11D1C2F38463BB4043EA35
:1077D8000C0323668008E36901309842D6D8A86A6A
:1077E800C2F38363BB4006403343CEE792FAA2F369
:1077F800B3FA83F3EAE73B493B48D1F808378242BA
:1078080003F0E07519D11B02CED4D1F8083723F064
:10781800E0732B4343F40003C1F80837334B1A686D
:10782800334BB2FBF3F20C2302FB03330193019BAE
:10783800002BB9D0019B013BF8E72E48824210D1BA
:1078480013F08070B0D1D1F8083723F0E0732B43E0
:1078580043F08073C1F80837002384F8543003B02C
:10786800F0BD254882429FD113F480009CD1D1F805
:10787800083723F0E0732B4343F48003EAE7B3F1BE
:10788800004F01BFAB6AC2F311018B43AB62002A00
:107898008ADA154813498242D1F8083709D1D1F854
:1078A800082703F0A07322F0E0721343C1F80837E9
:1078B8007AE71048824204D1D1F8082703F440033C
:1078C800F1E70D4882427FF46FAFD1F8082703F043
:1078D800C073E8E7A26D42F02002A2651846BBE734
:1078E8000220BCE700200140001000B0280800205A
:1078F800400D0300004000B8002000B4026838B50D
:1079080004461046FFF7BCFD08B9002038BD93684F
:10791800990707D4936823F0004323F0170343F033
:1079280010039360FBF704F9054623689B685B071F
:10793800EBD5FBF7FDF8401B0228F6D923689B68B6
:107948005A07F2D5A36D43F01003A365E36D43F026
:107958000103E3650120D9E773B5002302680193A9
:107968009368DD07044602D5002002B070BD916817
:10797800214B194209D0A36D43F01003A365E36DB1
:1079880043F00103E3650120EFE7936823F0004328
:1079980023F0170343F001039360184BD3F808371B
:1079A80018021CD4637E012BDED0FBF7C1F8144EFD
:1079B800054622681368DB07D6D49368D9075FBFEA
:1079C8009368334043F001039360FBF7B1F8401B21
:1079D8000228EED923681B68DA07EAD4CBE7094BFB
:1079E800094A1B68B3FBF2F301330193019B002B97
:1079F800D8D0019B013BF8E7170000800020014028
:107A0800E8FFFF7F28080020400D030038B5044632
:107A18000068FFF735FD054620BB94F85430012B6C
:107A280020D0012384F854302046FFF795FFB0B9E1
:107A3800A36D226823F4706323F0010343F4807379
:107A4800A3651C23E065136084F85400936823F051
:107A5800004323F0170343F00403936038BD84F810
:107A68005450FBE70220F9E7026838B5936891683B
:107A78000446C80701D4002038BD9907FBD4936891
:107A880003F00503012B19D1936823F0004323F079
:107A9800170343F00203936003231360FBF748F8CE
:107AA800054623689B68DB07E5D5FBF741F8401BD3
:107AB8000228F6D923689B68DA07F2D5A36D43F04C
:107AC8001003A365E36D43F00103E3650120D3E7E9
:107AD80070B5044600284BD0836D43F002038365DC
:107AE800FFF70CFF054668B92046FFF7BDFF0546BE
:107AF80008B90123A3652268936823F0104323F093
:107B08001703936023685A6822F4677222F003020D
:107B18005A6040F29F321A60D968164A0A40DA6001
:107B28001A6922F040421A615A6922F007025A6122
:107B38001A6A02F0F0221A625A6A02F0F0225A62B5
:107B4800DA6A02F0F022DA629A6A0B4A00269E622A
:107B5800D2F8083723F0FE73C2F808372046FAF740
:107B680091F9E6652666A66584F85460284670BDD6
:107B78000125FBE700023E830020014010B590F884
:107B88005430012B044615D0012380F85430FFF7F8
:107B9800B5FE58B92046FFF767FF38B9A36D23F43F
:107BA800807323F0010343F00103A365002384F8E5
:107BB800543010BD0220FCE7F7B50023019390F87C
:107BC8005430012B04467FD0012380F85430FFF74E
:107BD8004BFF23689A6812F00102054607D0A36D8F
:107BE80043F01003A365002384F854302DE0A16D01
:107BF800364F21F4817141F00201A165DE68D96830
:107C080026F4FF4626F07C0621F40041360421F0D4
:107C18000301360CD96008209968394041F00041C9
:107C280099609968002913DA019901310191019944
:107C3800B1F52E3FF5D3A36D23F0120343F01003E3
:107C4800A365002384F854300125284603B0F0BD0D
:107C5800D3F8B410013801F07F010A44DCD19968E7
:107C68001A48014041F001019960D3F8B41021F09D
:107C78007F0141EAD202C3F8B4209A68024042F078
:107C880002029A60FAF754FF074623689A68D207F7
:107C980008D4DA683243DA60A36D23F0030343F0B3
:107CA80001039FE7FAF744FFC01B0228EDD92368B8
:107CB8009B68D907E9D5A36D43F01003A365E36D6D
:107CC80043F00103E365BFE70225BEE7E8FFFF7F56
:107CD8000749CA6822F4E0620302120403F4E0636D
:107CE800120C134343F0BF6343F40033CB60704777
:107CF80000ED00E0164B30B5DC68C4F30224C4F193
:107D08000703251D042B28BF0423062D4FF0FF353C
:107D18008CBF033C002405FA03F321EA0303A540C2
:107D280022EA0502A340002843EA0203ACBF00F19F
:107D38006040084A4FEA0313B8BF00F00F00DBB2F7
:107D4800AABF00F56140135480F8003330BD00BF6E
:107D580000ED00E014ED00E0002807DB044A4109CB
:107D6800012300F01F00834042F82130704700BF14
:107D780000E100E000280CDB4309064900F01F0081
:107D880020330122824041F82320BFF34F8FBFF3F5
:107D98006F8F704700E100E070B5D0E9134565606A
:107DA800446D14B1D0E916456560D0E9105404F06B
:107DB8001C060124B4406C60046863608368102B5F
:107DC8000BBFA260A160E160E26070BD0268416C17
:107DD800D3B210B5083B1424B3FBF4F30B4CA24206
:107DE80088BF0B4A21F0030199BF01F1804202F5D7
:107DF8000232521807338264064AC26403F01F0332
:107E0800012202FA03F3036510BD00BF0704024014
:107E18001C0802408008024038B500285ED002687D
:107E28002F4B9A424FF014014CD82E4B1344B3FBFE
:107E3800F1F32D499B00C0E91013022380F8253087
:107E48001368056923F4FF4323F070031360D0E936
:107E5800024323432B43456911682B4385692B4310
:107E6800C5692B43056A2B430B431360FFF7AEFF2D
:107E7800B4F5804F04BF002343604268816C02F070
:107E88007F030B60D0E91314013A032A4C6020D811
:107E9800164A174981651A44013B9200012103F0F3
:107EA800030301FA03F300214265C3651160114A17
:107EB800536400230122C36380F8243080F825200E
:107EC800184638BD0C4B1344B3FBF1F30B499B0028
:107ED800B1E70023C0E91533C365EAE70120F0E7FD
:107EE80007040240F8FFFDBF000002403F82001077
:107EF8004009024000090240F8FBFDBF00040240AF
:107F080038B5002841D00268136823F001031360D4
:107F18001F4B9A424FF0140130D81E4B1344B3FB49
:107F2800F1F31D499B00C0E91013012403F01C0361
:107F380004FA03F3002515604B60FFF747FF836CD5
:107F480041681D60D0E913325A604A1E032A06D8D8
:107F5800124B0B449B0094401D60114B5C64002342
:107F6800C363C0E91533C0E90B33C0E90D33C365FA
:107F780080F8253080F82430184638BD094B134462
:107F8800B3FBF1F308499B00CDE70120F5E700BFFB
:107F980007040240F8FFFDBF000002403F820010C6
:107FA80000090240F8FBFDBF0004024070B590F8DC
:107FB8002450012D04463BD090F825600125AE429F
:107FC80080F824504FF000062CD1022580F8255067
:107FD8000568C6632E6826F001062E60FFF7DCFEF2
:107FE800036BBBB12B6843F00E032B60A36C1A68BC
:107FF800D20342BF1A6842F480721A60636D1BB1E3
:108008001A6842F480721A602B6843F001032B60EF
:10801800002070BD2B6823F004032B602B6843F00D
:108028000A03E2E78023C36380F824602846F0E768
:108038000220EEE7034640B190F82520022A06D038
:108048000422C263002280F82420012070470268BD
:10805800806C116821F00E011160016821F48071B3
:108068000160116821F001011160D3E9100202F0EA
:108078001C0101228A404260D3E9132151605A6DE4
:1080880032B1116821F480711160D3E91621516071
:108098000122002083F8252083F82400704710B5BA
:1080A80090F82530022B03D00423C363012010BDB0
:1080B80003681A6822F00E021A601A6822F0010298
:1080C8001A60826C136823F480731360D0E910136C
:1080D80003F01C02012393404B60D0E913325A602D
:1080E800436D33B11A6822F480721A60D0E91632EF
:1080F8005A60012380F82530836B002480F82440DF
:1081080013B198472046D2E71846D0E770B4426CBE
:10811800046C036826681D6802F01C020421914063
:1081280031420FD015F0040F0CD01A6892065EBFCA
:108138001A6822F004021A60036B6160002B33D0C6
:1081480070BC184702219140314217D015F0020F38
:1081580014D01A68940606D41A6822F00A021A6023
:10816800012280F82520114A93428CBF104B114BF5
:108178005960002380F82430C36ADFE70821914062
:10818800314211D029070FD5196821F00E01196065
:10819800012303FA02F26260C36380F825300023EA
:1081A80080F82430436BC9E770BC704780000240F8
:1081B80000040240000002400A4A536943F4802345
:1081C80030B55361EFF3108472B60023CD58C55013
:1081D8000433B3F5807FF9D11369DB03FCD484F34E
:1081E800108830BD00400058064B5A69002ABFBFAE
:1081F800054A9A6002F188329A60BABF5869C00F7E
:10820800002070470040005823016745044B5A6915
:1082180042F000425A615869C043C00F704700BF1E
:108228000040005870B50546FAF782FC124E044625
:108238003369D90313D43369DA0744BF01223261A1
:108248004CF2FA32134011D10B4E306910F48020F1
:108258000BD0FAF76DFC001BA842F6D304E0FAF73E
:1082680067FC001BA842E3D3032070BD024A1361D8
:10827800024A01205360F8E700400058300F002000
:108288002DE9F041184D98462B78012B06460C46EF
:10829800174626D001232B704FF47A7000236B60A9
:1082A800FFF7C0FFA0B9012E16D1104A536943F059
:1082B800010353612760BFF36F8FC4F804804FF444
:1082C8007A70FFF7AFFF094A536923EA060353613F
:1082D80000232B70BDE8F08139462046FFF76CFF7C
:1082E800EDE70220F6E700BF300F002000400058FD
:1082F800054A536923F47E7343EAC00040F4803092
:1083080040F0020050617047004000582DE9F041EC
:10831800234F3B78012B054688463FD001233B700D
:108328004FF47A7000237B60FFF77CFF044688B91E
:108338002B68042B13D11B4A536943F4803343F051
:10834800040353614FF47A70FFF76CFF0446154B32
:108358001A681B6800233B702046BDE8F0814FF087
:10836800FF33C8F800306E68D5E901321344B342D0
:108378000AD93046FFF7BCFF4FF47A70FFF752FF77
:1083880050B1C8F800600446064A536923F47E7366
:1083980023F002035361DAE70136E5E70224DBE75D
:1083A800300F0020004000582DE9F04F524C0023B8
:1083B8004FF00F090A6832FA03F501D1BDE8F08FD2
:1083C800012505FA03F818EA020200F08E804E68CB
:1083D800032706F003054FEA430E07FA0EFC6F1E4B
:1083E800012F6FEA0C0C32D8876807EA0C0ACF68AD
:1083F80007FA0EF747EA0A078760476827EA080876
:10840800C6F300179F4047EA08074760C76807EAAE
:108418000C088F6807FA0EF747EA0807022DC760AD
:1084280017D14FEAD30800EB880803F0070AD8F8F9
:1084380020704FEA8A0A09FA0AFB27EA0B0B0F6930
:1084480007FA0AF747EA0B07C8F8207001E0032D7E
:10845800DCD1076805FA0EF507EA0C073D4316F468
:10846800403F056041D023F0030707F1804707F537
:10847800803703F0030CBD684FEA8C0C4FF0070EF1
:108488000EFA0CFEB0F1904F25EA0E0E2FD01B4DC0
:10849800A8422ED005F58065A8420CBF0225072505
:1084A80005FA0CF545EA0E05BD602568D74316F4B4
:1084B800801F0CBF3D4015432560656816F4001FFA
:1084C8000CBF3D4015436560D4F8805016F4803FDA
:1084D8000CBF3D401543C4F88050D4F88450B6030F
:1084E80054BF3D401543C4F88450013362E700256A
:1084F800D6E70125D4E700BF00080058000400486B
:10850800374A2DE9F04F00234FF0010A4FF0070BCF
:108518004FF00F0931FA03F401D1BDE8F08F0AFAE0
:1085280003FC1CEA010654D023F0030404F1804440
:1085380004F5803403F00307A568BF000BFA07F8B9
:10854800B0F1904F08EA050E45D0264DA84244D018
:1085580005F58065A8420CBF02250725BD40754575
:1085680017D1D2F8805025EA0605C2F88050D2F813
:10857800845025EA0605C2F88450156825EA0605E0
:108588001560556825EA06055560A56825EA0805B9
:10859800A560056803265C0006FA04F423FA06F6CB
:1085A800254300EB8606056003F00705376AAD0032
:1085B80009FA05F527EA05073762856825EA0405FB
:1085C8008560456825EA0C054560C56825EA040408
:1085D800C46001339EE70025C0E70125BEE700BF60
:1085E80000080058000400480369194214BF01201C
:1085F800002070470AB181617047816270470000AE
:10860800044AD168014208B502D0D060FBF736F9B8
:1086180008BD00BF0008005803689A69910744BF65
:1086280000229A629A69D2075EBF9A6942F00102F3
:108638009A61704730B5039D04682B4343EA0243AF
:10864800064A6068C1F309010B4342EA555223F018
:10865800004320EA02000343636030BDFF63FF0369
:1086680003682DE9F0419C6914F0100405460F4693
:1086780016466FD010220024DA61A0462B689A694A
:10868800900661D4B8F1000F35D044F004040120FD
:108698002E68B369D90541BF4FF48072F26144F086
:1086A800010401205A0541BF4FF4806244F00804D8
:1086B800F26101209B054FD54FF4007344F002048A
:1086C800F3612846FFF7A8FF736823F0FF7323F4CC
:1086D8008B3323F4FF7323F0010373606B6C234324
:1086E8006B64202385F84130002385F8423085F8F3
:1086F8004030012032E07A1CC1D0FAF719FA801B09
:10870800B84201D8002FB9D12B68596895F8422092
:1087180098690004D2B20AD5490408D4202A06D0A0
:108728005A6842F480425A60FAF702FA06462B6801
:108738009B699B06A2D4FAF7FBF9801B1928F6D986
:1087480020244FF0010899E7B8F1000F9DD12022AD
:10875800DA619AE720469BE70028B2D1BDE8F081AC
:1087680070B504460D46164623689B699B0701D5DC
:10877800002070BD324629462046FFF771FFA0B998
:108788006A1CF1D0FAF7D4F9801BA84201D8002D51
:10879800EAD1636C43F020036364202384F84130FA
:1087A800002384F8423084F840300120E1E770B5B6
:1087B80004460D46164623689B695B070ED432466D
:1087C80029462046FFF74CFF38BB23689A69910673
:1087D80025D59A69520703D5228D0AB1002070BDAC
:1087E8009A6912F010021CBF1022DA614FF02001C2
:1087F80018BF04226264D9615A6822F0FF7222F419
:108808008B3222F4FF7222F001025A60002384F8AE
:10881800411084F8423084F840300120DFE7FAF74D
:1088280087F9801BA84201D8002DC4D1636C43F09E
:1088380020036364202384F841300023EBE72DE90B
:10884800F041069F0446884616461D4622689369ED
:1088580038EA03030CBF01230023B34201D00020F0
:1088680015E06B1CF3D0FAF763F9C01BA84201D8D6
:10887800002DEBD1636C43F020036364202384F85C
:108888004130002384F8423084F840300120BDE8AC
:10889800F08170B504460D46164623689B699B0611
:1088A80001D5002070BD324629462046FFF7D8FE84
:1088B80090B9FAF73DF9801BA84201D8002DECD1F8
:1088C800636C43F020036364202384F84130002361
:1088D80084F8423084F840300120E3E710B50446BC
:1088E80000284AD090F8413003F0FF021BB980F805
:1088F8004020F9F70BFE242384F8413023681A68D6
:1089080022F001021A60626822F070621A619A68A5
:1089180022F400429A60D4E90221012924D142F4C8
:1089280000429A605A6842F0007242F400425A606B
:10893800DA6822F40042DA60D4E904210A43A16922
:1089480042EA0122DA60D4E907210A431A601A6868
:1089580042F001021A6000202023606484F841304C
:10896800206384F8420010BD42F4044202299A6050
:1089780004BF4FF400625A60D4E70120F3E7000017
:108988002DE9F347984690F841300A9F202B04467A
:108998000E46914640F0868090F84030012B00F05A
:1089A80081804FF0010A80F840A0FAF7C1F8192336
:1089B8000546009052464FF400412046FFF73FFF1E
:1089C80018B1012002B0BDE8F087212384F84130B6
:1089D800102384F842306064A4F82A80638DC4F8B8
:1089E80024909BB2FF2B60632F4B26D9FF22228550
:1089F80000934FF0807331462046FFF71BFE638DCE
:108A08009BB22A4639462046FBB9FFF742FF0028A9
:108A1800D7D123682021D9615A6822F0FF7222F445
:108A28008B3222F4FF7222F001025A6084F841105E
:108A380084F8400084F84200C4E7628D009392B243
:108A480022854FF00073D2B2D5E7FFF789FE0028E0
:108A5800B7D1636A226813F8011B91626362638D60
:108A6800228D013B9BB26385638D013A92B29BB222
:108A78002285002BC3D0002AC1D100953B46802116
:108A88002046FFF7DCFE00289BD1638D9BB2FF2BAD
:108A980003D9FF2222850090ABE7628D009092B245
:108AA8002285CEE702208DE7002000802DE9F347DC
:108AB800984690F841300A9F202B04460E4691466E
:108AC80040F0878090F84030012B00F082804FF012
:108AD800010A80F840A0FAF72BF819230546009000
:108AE80052464FF400412046FFF7A9FE18B1012075
:108AF80002B0BDE8F087222384F84130102384F8BF
:108B080042306064A4F82A80638DC4F824909BB234
:108B1800FF2B6063304B26D9FF22228500934FF04C
:108B2800807331462046FFF785FD638D9BB22A4648
:108B380039462046FBB9FFF7ACFE0028D7D1236899
:108B48002021D9615A6822F0FF7222F48B3222F474
:108B5800FF7222F001025A6084F8411084F8400044
:108B680084F84200C4E7628D009392B222854FF0E8
:108B78000073D2B2D5E7FFF71AFE0028B7D12368F1
:108B88005A6A636A1A70636A228D01336362638D5D
:108B9800013B9BB26385638D013A92B29BB22285F9
:108BA800002BC2D0002AC0D100953B468021204628
:108BB800FFF745FE00289AD1638D9BB2FF2B03D99E
:108BC800FF2222850090AAE7628D009092B222854A
:108BD800CDE702208CE700BF0024008010B590F894
:108BE8004120202A0346D4B21CD190F84020012A03
:108BF80018D0242280F841200268106820F0010073
:108C08001060106820F480501060106801431160F3
:108C18001168002041F00101116083F8414083F898
:108C2800400010BD0220FCE710B590F84120202A32
:108C38000346D4B21BD190F84020012A17D0242231
:108C480080F841200268106820F001001060106868
:108C580020F4706040EA012111601168002041F0A1
:108C68000101116083F8414083F8400010BD0220E3
:108C7800FCE70000024A136843F4807313607047EE
:108C8800000400580D4B10B55B690C4628B99A05CD
:108C980007D500F027F820B110BD9B0501D400F0DE
:108CA80019F8074A1369012C23F00403136101D151
:108CB80030BFF1E740BF20BF20BFEDE700040058F8
:108CC80000ED00E0024B186800F4C060704700BF78
:108CD80000040058024A136843F480431360704745
:108CE800000400580C4A136823F4804313600B4BAC
:108CF8001B6832214B430A49B3FBF1F351698905DB
:108D080000D533B9536913F4007F14BF0320002042
:108D18007047013BF2E700BF000400582808002014
:108D280040420F000B4A136823F0070343F0020385
:108D38001360094B1A69012842F004021A6105D12F
:108D480030BF1A6922F004021A61704740BF20BF81
:108D580020BFF6E70004005800ED00E04FF0B043F4
:108D68001868C0F3404070474FF0B0431868C0F32C
:108D7800400070474FF0B042536823F47F4343EA02
:108D88000023536070474FF0B0431868C0F3406049
:108D9800704700007FB54FF0B0432C4AD3F8083134
:108DA800C0F3031003F00F0352F82040284A52F88A
:108DB8002330B4FBF3F4FFF785FF264B054693E811
:108DC8000700B5F5007F04AB03E9070010D0224B7C
:108DD8009C4218D303F5B70303F67F539C4229D965
:108DE80003F5741303F510639C4225D802230BE0A6
:108DF8001A4B9C4207D91A4B9C421BD903F53703DF
:108E080003F5D853F0E7002304AA02EB830353F8D1
:108E18000C4C144D2B6823F0070323432B60F9F700
:108E280087FE06462B6803F007039C4206D1002004
:108E380004B070BD0123E7E70024EAE7F9F778FEFC
:108E4800801B0228EED90320F2E700BF9C520108DC
:108E58003C52010810470108C0CF6A00BFEA21014F
:108E68003F933402004000584FF0B04310B59A6861
:108E7800D96812F00C0205D00C2A4AD101F003037C
:108E8800012B50D14FF0B0412B480B6813F0080369
:108E980006D00B6813F0080337D1D1F8941007E017
:108EA8000C68240756BFD1F894300968C3F303232C
:108EB80050F82330002A0CBF184600204FF0B0416C
:108EC8008A6802F00C020C2A1ED1CA6802F003025A
:108ED800022A2ED0032A06D10B68184A13F4801FE1
:108EE800174B18BF13464FF0B042D068D168D2680C
:108EF800C0F306205843C1F302130133B0FBF3F06B
:108F0800530F0133B0FBF3F010BD0B68C3F3031329
:108F1800CEE7042A0AD0082A05D11B6813F4801367
:108F280004D10748CAE700231846C7E703480023C7
:108F3800C4E7024BD7E700BF9C5201080024F400A5
:108F48000048E80108B5FFF78FFF4FF0B043044A27
:108F58009B68C3F3031352F82330B0FBF3F008BD4A
:108F68003C5201082DE9F0410446002853D04FF047
:108F7800B0439D68DE6803689B0605F00C0506F0A3
:108F8800030668D5026A1DB10C2D46D1012E44D1C5
:108F9800002A40D04FF0B043A16A1A68170756BF9D
:108FA800D3F894301B681B0903F0F00399421FD9CA
:108FB8000846FFF7EFFE00282DD14FF0B0421368A6
:108FC80043F0080313601368A16A23F0F0030B430E
:108FD8001360606AFFF7CEFEFFF7B4FFAB4B186073
:108FE800AB4B1868F9F7A2FD002834D0BDE8F08132
:108FF8004FF0B042136843F008031360136823F07E
:10900800F0030B431360606AFFF7B4FE0846FFF7EE
:10901800C1FE0028E0D00120E8E74FF0B043002A65
:1090280054D01A6842F001021A60F9F781FD074628
:10903800FFF79AFE002842D04FF0B042136843F081
:10904800080313601368A16A23F0F0030B4313604D
:10905800606AFFF78FFE2368D80748D4236899070A
:1090680000F18C8023681E0740F1FA80A3694FF055
:10907800B046002B00F0E180D6F89430E16903F0A7
:109088001002914200F0C48003F00302022AC2D009
:10909800D80740F1B380D6F8943023F00103C6F81E
:1090A8009430F9F745FD0746D6F89430990740F112
:1090B800A580F9F73DFDC31B112BF5D904E0F9F79D
:1090C80037FDC01B0228B3D903208FE71A6822F0A6
:1090D80001021A60F9F72CFD0746FFF745FE002844
:1090E800B9D0F9F725FDC01B0228F6D9ECE7082D01
:1090F80003D00C2D05D1032E03D16368002BADD10D
:1091080089E74FF0B043A1681A6822F480120A4335
:109118001A606268B2F5803F10D11A6842F4803252
:109128001A60F9F705FD0746FFF718FE002895D1E4
:10913800F9F7FEFCC01B6428F6D9C5E7B2F5041F91
:1091480004D11A6842F400121A60E6E7196821F49B
:1091580080311960196821F400111960002AE0D1E2
:10916800F9F7E6FC0746FFF7F9FD00283FF476AF6C
:10917800F9F7DEFCC01B6428F5D9A5E7042D23699F
:1091880003D00C2D0ED1022E0CD1002B3FF443AF8F
:109198004FF0B0426169536823F0FE4343EA01632C
:1091A80053605FE74FF0B046BBB1336843F4807358
:1091B8003360F9F7BDFC074633685A0507D573686D
:1091C800626923F0FE4343EA026373604AE7F9F7F2
:1091D800AFFCC31B022BEFD976E7336823F4807307
:1091E8003360F9F7A5FC074633685B057FF53AAFAE
:1091F800F9F79EFCC31B022BF6D965E74FF0B04286
:10920800E169D2F8943023F010030B43C2F894308C
:109218004FF0B047D7F8943043F00103C7F89430C3
:10922800F9F786FC0646D7F894309A0718D4F9F768
:109238007FFC831B112BF6D946E7D6F8943023F030
:109248000103C6F89430F9F773FC0746D6F8943052
:109258009B0705D5F9F76CFCC31B112BF6D933E72F
:109268002368580754D50B4F3B68D90514D4FFF72A
:1092780001FDF9F75DFC06463B68DA050CD4F9F701
:1092880057FC831B022BF7D91EE700BF28080020D4
:109298002C08002000040058E3684FF0B046002B6B
:1092A80058D023F08003052B02BFD6F8903043F046
:1092B8000403C6F890304FF0B046F9F739FCD6F8F9
:1092C800903043F001030746C6F8903041F28838E1
:1092D800D6F890309B0705D4F9F72AFCC31B434501
:1092E800F6D9F1E6E36823F00403812B1BD1F9F7E3
:1092F8001FFCD6F8903043F08003C6F8903007463C
:109308004FF0B04641F28838D6F89030180504D5A9
:10931800E06A00284AD1002068E6F9F709FCC01B7A
:109328004045F1D9D0E6F9F703FCD6F8903023F0A0
:109338008003C6F8903007464FF0B04641F28838AF
:10934800D6F890301905E3D5F9F7F2FBC01B404574
:10935800F6D9B9E6F9F7ECFBD6F8903023F080039C
:109368000746C6F8903041F28838D6F890301A058A
:1093780016D4F9F7DDFBD6F8903023F00103C6F8D0
:10938800903007464FF0B04841F28836D8F8903010
:109398009B07BDD5F9F7CCFBC31BB342F6D993E6BF
:1093A800F9F7C6FBC01B4045DFD98DE60C2D4ED022
:1093B8004FF0B04302281A6822F080721A6033D145
:1093C800F9F7B6FB0546FFF7DEFC38BBD4E90C31EC
:1093D8004FF0B0420B43D0682D4901400B43E16B7D
:1093E8000B43216C0B43616C0B43A16B43EA0123D4
:1093F800D360136843F080731360D36843F08053DD
:10940800D360F9F795FB0446FFF7BDFC002882D12D
:10941800F9F78EFB001B0A28F6D955E6F9F788FB01
:10942800401B0A28CFD94FE6F9F782FB0446FFF71D
:10943800AAFC30B94FF0B042164BD1680B40D3604C
:10944800D4E5F9F775FB001B0A28F0D93CE601289A
:109458003FF4CCAD4FF0B043226BDB6803F003015F
:1094680091427FF4D8AD616B03F070028A427FF4B9
:10947800D2ADA16B03F4FE42B2EB012F7FF4CBAD6A
:10948800626C03F0604393423FF445AFC3E500BF0D
:109498008C80C111FCFFFEEE2DE9F0410D4604461B
:1094A80010B90120BDE8F081684E336803F0070366
:1094B8008B4216D323689A0727D54FF0B047A26886
:1094C800BB6823F0F0031343BB60F9F731FB064692
:1094D800BB68DB0319D4F9F72BFB831B022BF7D9E5
:1094E80011E0336823F007030B433360F9F720FBDF
:1094F8000746336803F00703AB42DBD0F9F718FBE4
:10950800C01B0228F5D90320CCE72368580617D5D5
:109518004FF0B0476269D7F8083123F00F0343EAE8
:109528001213C7F80831F9F703FB0646D7F80831D4
:10953800D90305D4F9F7FCFA831B022BF6D9E2E725
:1095480023685A0713D54FF0B047E268BB6823F485
:10955800E0631343BB60F9F7EBFA0646BB689B036D
:1095680005D4F9F7E5FA831B022BF7D9CBE7236873
:10957800180714D54FF0B0472269BB6823F460532D
:1095880043EAC203BB60F9F7D3FA0646BB6859033E
:1095980005D4F9F7CDFA831B022BF7D9B3E7236873
:1095A800DA070FD4294C236803F00703AB4239D8F4
:1095B800FFF7C8FC264B1860264BBDE8F041186839
:1095C800F9F7B4BA6268022A1DD1FFF7C7FB002871
:1095D8003FF467AF4FF0B04641F28838B36823F0E4
:1095E80003031343B360F9F7A3FA0746B368626845
:1095F80003F00C03B3EB820FD4D0F9F799FAC01B30
:109608004045F3D97FE7032A02D1FFF7BCFBDEE729
:1096180012B9FFF7A9FBDAE74FF0B0431B685B0507
:10962800D8D43EE7236823F007032B432360F9F7D8
:109638007FFA0646236803F00703AB42B8D0F9F770
:1096480077FA801B0228F5D95DE700BF0040005873
:10965800280800202C08002008B5FFF773FC4FF0FD
:10966800B043044A9B68C3F3022352F82330D8401E
:1096780008BD00BF7C52010808B5FFF763FC4FF036
:10968800B043044A9B68C3F3C22352F82330D8403E
:1096980008BD00BF7C5201084FF0B043D3F89000DA
:1096A800C0F3400070474FF0B0410209D1F888304C
:1096B80002F47F22000123EA020300F47F2003431F
:1096C800C1F8883070474FF0B041020CD1F88830AB
:1096D800120423EA020343EA0040C1F888007047F5
:1096E80070B5066816F48036044638D0FFF7C2FA1B
:1096F800F9F71EFA614E05463368DB0529D54FF0A8
:10970800B043616BD3F8902002F44072914214D0B8
:10971800D3F89010D3F8902042F48032C3F8902008
:10972800D3F8902021F4407022F480328D07C3F8DA
:109738009020C3F8900000F190804FF0B042616B28
:10974800D2F8903023F440730B43C2F890300026CF
:1097580005E0F9F7EDF9401B0228CDD90326256865
:10976800E8070AD54FF0B0416268D1F8883023EA9B
:10977800124392B21343C1F88830A9070AD54FF0B3
:10978800B041A268D1F8883023EA124392B2134359
:10979800C1F88830AA0609D54FF0B0422169D2F83D
:1097A800883023F440630B43C2F88830AB0502D5F8
:1097B800206AFFF788FF680502D5606AFFF783FF14
:1097C800290502D5A06AFFF77EFF6A0602D56069FF
:1097D800FFF769FF2B0602D5A069FFF764FFE805CC
:1097E80002D5E069FFF75FFFE90610D54FF0B042F8
:1097F800E168D2F8883023F440730B43C2F888300C
:10980800B1F5807F02BFD36843F08073D3602A0428
:109818000ED54FF0B042216BD2F8883023F0404388
:109828000B43C2F8883019B9D36843F08073D3600A
:109838006B0410D54FF0B042E16AD2F8883023F0BB
:1098480040530B43B1F1005FC2F8883003D1D368AD
:1098580043F48033D360304670BDF9F769F941F2BB
:1098680088360546FFF718FF01283FF466AFF9F779
:109878005FF9401BB042F5D970E700BF00040058FB
:1098880030B590F82C30012B02464FF0020022D060
:10989800174B82F82D00CA24012582F82C505C62EF
:1098A80053245C62B1F5807F146B996914D121F45B
:1098B80088519961596C24F0010421F000415964E0
:1098C8001463DD650A4BFF2159620020012382F8E9
:1098D8002D3082F82C0030BD21F408519961D96CE3
:1098E80024F0020421F00041D9641463D865E9E743
:1098F8000028004070B50B4E036B756D1D40EA07DC
:10990800044603D50123F365F9F783FAAB0704D5B9
:109918000223F365204600F0CBF9012384F82D30AB
:1099280070BD00BF0028004038B50A4CE36823F03A
:109938002003E360F9F7FCF80546E3689B0601D5C8
:10994800002038BDF9F7F4F8401BB0F57A7FF4D958
:109958000320F6E7002800402DE9F041114DEC689E
:1099680014F0400407461AD1EB6843F08003EB601B
:10997800F9F7DEF84FF003080646EB685B0601D4FA
:10998800032C02D12046BDE8F081F9F7D1F8801BFD
:10999800B0F57A7F84BF87F82D800324EDE7002493
:1099A800F0E700BF0028004038B50F4CE36823F00B
:1099B8008003E360A3699B06054606D4FFF7B4FF5E
:1099C80010B1032085F82D0038BDA36923F02003CA
:1099D800A361FFF7A9FF10B1032085F82D00A36943
:1099E80043F02003A361EFE70028004038B50446A0
:1099F80000284BD090F82D3003F0FF021BB980F8F7
:109A08002C20F8F793FE0223214D84F82D30EB68C3
:109A1800DB0632D4CA236B6253236B622046FFF7FE
:109A28009BFF78BBAB6923F08E6323F04003AB61E7
:109A380021696368AA690B431343A2691343AB61A5
:109A4800D4E9022343EA02432B61D4E90931EA68E5
:109A58000B4322F4F8521343EB602046FFF7A4FFB0
:109A680080B9D4E90713AA690B4322F06042134373
:109A780062691343AB61FF236B62012384F82D30C5
:109A8800002002E0024BFF225A6238BD0120FCE7A9
:109A9800002800400023092803D840EA0310C0B278
:109AA80070470A380133C0B2F5E700002DE9F047E6
:109AB80090F82C30012B05464FF0020069D00123A5
:109AC80085F82C304E4B85F82D00DE6806F440767C
:109AD800B6F5807F78D04C69087891F8019091F8B4
:109AE80002A091F82470002A55D19B6913F0400315
:109AF80008BFCB70FFF7CEFF80464846FFF7CAFF86
:109B080002465046FFF7C6FF81463846FFF7C2FFB8
:109B18000B6ACF78234343EA875343EA090343EAAE
:109B2800084343EA022343EA0063354ACA205062E5
:109B3800532050628C6A8869B4F5807F946945D156
:109B480024F4885494610124D465B6F5807F09BF54
:109B5800CB6913640343536418BF5064284B4A68A5
:109B68001A672A6B42F001022A639A6942F4885202
:109B78009A61244AD2F8803043F40033C2F8803026
:109B88001F4BFF225A620020012385F82D3085F8EB
:109B98002C00BDE8F087B4F1803F07D0B4F5000F82
:109BA80004D09B6913F0400308BFCB700B6ACA78D6
:109BB8001C4344EA0A0444EA004343EA092343EA0B
:109BC800825343EA0763B0E70023AEE724F408545E
:109BD80094610224D465B6F5807F09BFCB6993648C
:109BE8000343D36418BFD064054B4A685A672A6B8D
:109BF80042F002022A639A6942F40852B8E700BFA9
:109C0800002800400008005890F82C20012A03463C
:109C18004FF0020012D00A4A83F82D00CA2151627F
:109C280053215162916941F020019161FF215162F4
:109C38000020012283F82D2083F82C00704700BFF4
:109C48000028004090F82C20012A03464FF002001B
:109C580019D00D4A83F82D00CA215162532151624F
:109C680091690A4841F080019161D0F8801041F46F
:109C78008021C0F88010FF2151620020012283F862
:109C88002D2083F82C007047002800400008005859
:109C9800064B5A6D520610B5044603D54022DA65C4
:109CA800F9F7BAF8012384F82D3010BD00280040D8
:109CB8007047890001F1804101F531410A60704720
:109CC800890001F1804101F53141086870470000C1
:109CD800034AD2F8903043F40043C2F890307047FA
:109CE80000040058034AD2F8903023F40043C2F825
:109CF8009030704700040058074B1A6822F0400261
:109D08001A6040F441704FF4B85218605A601A68EB
:109D180042F040021A6070470000015837B5054606
:109D280000284ED0837903F0FF046BB1032C0BD0CD
:109D3800254B4FF400629A612868FFF7DDFF002485
:109D480001232B71AC602FE000236B712846F8F7D4
:109D580007FE1E4AD2F8903043F48053C2F8903080
:109D6800002CE5D102234FF0B042AB71D2F8943009
:109D780023F40043C2F89430154B1B681C214B4355
:109D8800DB0C64214B430193019B93B90124AC6024
:109D9800FFF79EFF0C4B9A6842F400629A604FF4FA
:109DA80000629A61002CC7D00123AB71204603B032
:109DB80030BD019B013B0193D2F894305B04E3D49E
:109DC800E6E70124F2E700BF000400580008005845
:109DD8002808002037B5174D2B6802461C2043433E
:109DE800DB0C6420434314480193019B93B9012081
:109DF8009060114C21732B681C214B43DB0C6421B0
:109E08004B430193019B6BB9012090600A4BDB68BF
:109E180003B030BD019B013B019383689C07E4D5E7
:109E28000020E6E7019B013B0193A368DB07E9D526
:109E3800ECE700BF280800200000015837B5184D8E
:109E48002B6802461C204343DB0C6420434315481F
:109E58000193019BA3B901209060124CFF23237347
:109E68002B681C256B43DB0C64256B430193019B1A
:109E780073B9012090600B4BDB680B7003B030BDE9
:109E8800019B013B019383689C07E2D50020E4E72E
:109E9800019B013B0193A368DB07E8D5EBE700BF13
:109EA80028080020000001580F4B13B51B680F4C01
:109EB800182253431B0D64225343014601936269E0
:109EC800019B02F0040223B902238B60012002B037
:109ED80010BD019B013B0193606910F00200F6D0B0
:109EE800002AECD11046F2E72808002000040058A8
:109EF80007B50379012B0FD10A4B1B68182253436E
:109F08001B0C0193FFF7EEFE019B013B0193019BA4
:109F1800002BF9D1FFF7DCFE03B05DF804EBFFF787
:109F2800C3BF00BF28080020F8B51E468379012B5F
:109F3800154604460F46DAB22DD14379012B2AD0B3
:109F4800022342718371FFF7D3FF0D212046FFF7EB
:109F5800C9FEFFF73FFF390A2046FFF73BFFF9B27A
:109F68002046FFF737FF2E44B5420ED12046FFF7B3
:109F7800AFFEFFF799FFA06801230038A3714FF0E7
:109F8800000318BF01206371F8BD15F8011B2046B6
:109F9800FFF720FFE8E70220F6E7F8B51E468379C9
:109FA800012B154604460F46DAB22FD14379012B0F
:109FB8002CD04271FFF79CFF1D212046FFF792FE2F
:109FC800FFF708FF390A2046FFF704FFF9B22046D9
:109FD800FFF700FF00212046FFF7FCFE2E44B542A4
:109FE8000ED12046FFF774FEFFF75EFFA06801233D
:109FF8000038A3714FF0000318BF01206371F8BD4A
:10A0080029462046FFF71AFF0135E8E70220F6E760
:10A01800F8B51F468379012B154604460E46DAB279
:10A028002CD14379012B29D04271FFF761FF06F04B
:10A03800EF03A3F184025342534123713146204672
:10A04800FFF750FEFFF7C6FE2F44AF4210D1FFF7CF
:10A058003FFE842E02D02046FFF726FFA06801238A
:10A068000038A3714FF0000318BF01206371F8BDD9
:10A0780015F8011B2046FFF7ADFEE6E70220F6E7DC
:10A08800F8B51E468379012B154604460F46DAB209
:10A0980027D14379012B24D04271FFF729FF394694
:10A0A8002046FFF71FFEFFF795FE00212046FFF729
:10A0B80091FE2E44B5420ED12046FFF709FEFFF768
:10A0C800F3FEA06801230038A3714FF0000318BF06
:10A0D80001206371F8BD29462046FFF7AFFE013520
:10A0E800E8E70220F6E737B50023ADF8043001AA07
:10A0F800022312210546FFF7C3FFBDF804400223DF
:10A1080064BA01AAA4B219462846FFF781FFE207FC
:10A1180002D5284609F076FBA30702D5284609F0A0
:10A1280077FB600702D5284609F09CFB210702D57A
:10A13800284609F09DFBE20602D5284609F09EFB59
:10A14800A30602D5284609F087FB600602D52846F3
:10A1580009F064FB210606D514F4807118BF0121AB
:10A16800284609F061FBA20502D5284609F06CFBD8
:10A17800630402D5284609F087FB03B030BDF8B563
:10A188001E468379012B154604460F46DAB227D1BD
:10A198004379012B24D04271FFF7AAFE0E212046F5
:10A1A800FFF7A0FDFFF716FE39462046FFF712FE1F
:10A1B8002E44B5420ED12046FFF78AFDFFF774FE04
:10A1C800A06801230038A3714FF0000318BF0120D5
:10A1D8006371F8BD15F8011B2046FFF7FBFDE8E7A2
:10A1E8000220F6E7F8B51E468379012B154604468A
:10A1F8000F46DAB22BD14379012B28D04271FFF7F1
:10A2080077FE1E212046FFF76DFDFFF7E3FD394677
:10A218002046FFF7DFFD00212046FFF7DBFD2E4437
:10A22800B5420ED12046FFF753FDFFF73DFEA0686B
:10A2380001230038A3714FF0000318BF0120637198
:10A24800F8BD29462046FFF7F9FD0135E8E7022069
:10A25800F6E7026852E8003F23F0C00342E8003105
:10A2680002680029F5D102F1080353E8003F23F4FE
:10A27800000302F1080C4CE800310029F3D1202337
:10A28800C0F888307047000010B5026852E8003FF7
:10A2980023F4907342E8003102680029F5D10F4C8D
:10A2A80002F1080353E8003F234002F1080C4CE890
:10A2B80000310029F4D1C36E012B07D152E8003FC9
:10A2C80023F0100342E800310029F7D12023C0F819
:10A2D8008C300023C366436710BD00BFFEFFFFEF4D
:10A2E800F8B504461346D4F88850202D32D1F1B180
:10A2F800EAB1E06FA4F85620A4F8542000262122E1
:10A30800C4F890602165C4F88820226888B1124F8B
:10A31800C762124F0763124F2832C0E90D76FDF766
:10A3280045FE30B11023C4F89030C4F8885001209D
:10A338000FE0236840221A62226802F1080353E8FA
:10A34800003F43F0800302F1080141E80030002893
:10A35800F3D1F8BD0220FCE76DA30008B5A30008FF
:10A36800C1A3000808B50346806A1B681B6813F080
:10A37800200317D1A0F85630026802F1080353E809
:10A38800003F23F08003083242E8003102680029C8
:10A39800F2D152E8003F43F0400342E8003100297F
:10A3A800F7D108BDF8F78EFEFBE7704708B5806A5D
:10A3B800FFF7FBFF08BD7047806A38B50468D0F81E
:10A3C8008830D0F88C50A268120606D5212B04D10B
:10A3D8000023A0F85630FFF73CFFA3685B0606D5BC
:10A3E800222D04D10023A0F85E30FFF74DFFD0F8EE
:10A3F800903043F01003C0F89030FFF7DCFF38BD11
:10A4080008B5806A0023A0F85E30A0F85630FFF740
:10A41800D2FF08BD704700000368D9691A682DE9A2
:10A42800F04140F60F0631429D68044610D18E0671
:10A4380040F1978002F0200605F080573E4300F077
:10A448009080436F002B00F08580BDE8F0411847ED
:10A45800AB4EAC482E401040304300F08280CF070E
:10A4680009D5D00507D501201862D4F8900040F02E
:10A478000100C4F890008F0709D5E80707D5022026
:10A488001862D4F8900040F00400C4F890004F0718
:10A4980009D5E80707D504201862D4F8900040F0E1
:10A4A8000200C4F890000F070BD502F020003043DB
:10A4B80007D008201862D4F8900040F00800C4F8CB
:10A4C80090000E050AD5500108D54FF400601862B7
:10A4D800D4F8903043F02003C4F89030D4F890308A
:10A4E800002B37D08B0609D502F0200205F08055E5
:10A4F8002A4303D0636F0BB1204698472668D4F8E7
:10A508009020B36802F0280203F0400353EA0205E2
:10A51800204621D0FFF7B8FEB3685F0617D522683A
:10A5280002F1080353E8003F23F04003083242E8F1
:10A5380000310029F3D1D4F8800040B1724B836315
:10A54800FDF7ADFD30B1D4F88000836B7DE7204680
:10A55800FFF731FFBDE8F081FFF72DFFC4F89050F9
:10A56800F8E7E06E012840F08980CE0640F1868049
:10A57800D00640F1838010221A629A6851064BD5A2
:10A58800D4F8802011684A6892B2002AE2D0B4F860
:10A598005C009042DED9A4F85E200A6892062FD4A7
:10A5A80053E8002F22F4807243E800210029F7D1F4
:10A5B80003F1080252E8002F22F0010203F108001B
:10A5C80040E800210029F3D103F1080252E8002FE6
:10A5D80022F0400203F1080040E800210029F3D1ED
:10A5E8002022C4F88C20E16653E8002F22F01002E4
:10A5F80043E800210029F7D1D4F88000FDF71AFDBF
:10A6080002232367B4F85E30B4F85C10C91A89B223
:10A618002046FFF7FFFE9DE7B4F85E20B4F85E0021
:10A62800B4F85C1080B292B2002893D0891A89B22B
:10A6380000298FD053E8002F22F4907243E80020BD
:10A648000028F7D1314D03F1080252E8002F2A40C3
:10A6580003F1080646E800200028F4D12022C4F8B7
:10A668008C206067E06653E8002F22F0100243E870
:10A6780000200028F7D102232367C9E7CF0209D5B4
:10A688006E0207D54FF4801220461A62BDE8F041E9
:10A6980000F0A0BD08060BD502F0800005F4000507
:10A6A800284305D0A36F002B3FF454AF2046CCE6D7
:10A6B8004F0611D556060FD553E8002F22F0400259
:10A6C80043E800210029F7D12023C4F88830A16786
:10A6D8002046F8F7F7FC3DE70D0206D5500004D5F3
:10A6E8002046BDE8F04100F077BDCB017FF532AFE1
:10A6F800002ABFF62FAF2046BDE8F04100F06BBD41
:10A70800010000102001000409A40008FEFFFFEF6B
:10A71800D0F88C20B0F86010222A08B5036855D10B
:10A728005B6A826D0B401370836D01338365B0F8EB
:10A738005E30013B9BB2A0F85E30B0F85E309BB251
:10A74800002B42D1026852E8003F23F4907342E89C
:10A75800003103680029F5D103F1080252E8002FFF
:10A7680022F0010203F1080C4CE800210029F3D182
:10A778002022C0F88C20184A41679342016705D10E
:10A78800C26E012A0ED0F8F7ABFC1EE05A6811021F
:10A79800F6D553E8002F22F0806243E80021002913
:10A7A800F7D1EDE70022C26653E8002F22F010022D
:10A7B80043E800210029F7D1DA69B0F85C10D20625
:10A7C80044BF10221A62FFF725FE08BD9A6942F0BD
:10A7D80008029A61F9E700BF00800040D0F88C2099
:10A7E800B0F86010222A08B5036852D15A6A11409D
:10A7F800826D22F8021B8265B0F85E20013A92B29F
:10A80800A0F85E20B0F85E2092B2002A40D153E84A
:10A81800002F22F4907243E800210029F7D103F1B8
:10A82800080252E8002F22F0010203F1080C4CE85C
:10A8380000210029F3D12022C0F88C20174A416753
:10A848009342016705D1C26E012A0ED0F8F748FC81
:10A858001EE05A681102F6D553E8002F22F08062F4
:10A8680043E800210029F7D1EDE70022C26653E84A
:10A87800002F22F0100243E800210029F7D1DA69FD
:10A88800B0F85C10D20644BF10221A62FFF7C2FD6E
:10A8980008BD9A6942F008029A61F9E70080004011
:10A8A8002DE9F74F0368B0F86080DF691A689D6882
:10A8B800D0F88C1001922229044640F0B480B0F8F8
:10A8C8006890DFF86CA1DFF86CB10026B9F1000FD1
:10A8D80001D0BB0621D4B4F85E309BB2D3B1B4F832
:10A8E80068209A4216D9226802F1080353E8003F0B
:10A8F80023F08053083242E8003122680029F2D15F
:10A908004D4B636752E8003F43F0200342E80031B3
:10A918000029F7D103B0BDE8F08F2368A26D5B6A08
:10A9280003EA08031370A36D0133A365B4F85E301E
:10A93800013B9BB2A4F85E302368DF6978072CD00E
:10A94800F9070AD5019AD20507D501211962D4F869
:10A95800901041F00101C4F89010B80709D5E90733
:10A9680007D502211962D4F8901041F00401C4F807
:10A9780090107A0709D5E80707D504211962D4F899
:10A98800903043F00203C4F89030D4F8903023B1EB
:10A998002046FFF710FDC4F89060B4F85E309BB213
:10A9A800002B93D1216851E8003F23F4807341E8DC
:10A9B800003023680028F5D103F1080252E8001F8F
:10A9C80001EA0A0142E800100028F5D120215B4580
:10A9D800C4F88C10606720670AD05968090207D547
:10A9E80053E8001F21F0806143E800100028F7D1E8
:10A9F800E16E012913D1E66653E8001F21F010012A
:10AA080043E800100028F7D1D969CA0644BF1021CD
:10AA180019622046B4F85C10FFF7FCFC56E72046A4
:10AA2800F8F75EFB52E79A6942F008029A6171E70B
:10AA3800FEFFFFEF0080004019A700082DE9F74F3F
:10AA48000368B0F86080DF691A689D68D0F88C10D8
:10AA580001922229044640F0B280B0F86890DFF8ED
:10AA680068A1DFF868B10026B9F1000F01D0BB0674
:10AA780021D4B4F85E309BB2D3B1B4F868209A42BE
:10AA880016D9226802F1080353E8003F23F08053E7
:10AA9800083242E8003122680029F2D14C4B636742
:10AAA80052E8003F43F0200342E800310029F7D183
:10AAB80003B0BDE8F08F2368A26D596A08EA010166
:10AAC80022F8021BA265B4F85E20013A92B2A4F8FB
:10AAD8005E20DF6978072CD0F9070AD5019AD205DC
:10AAE80007D501211962D4F8901041F00101C4F88A
:10AAF8009010B80709D5E90707D502211962D4F8DB
:10AB0800901041F00401C4F890107A0709D5E807BD
:10AB180007D504211962D4F8903043F00203C4F831
:10AB28009030D4F8903023B12046FFF744FCC4F8A5
:10AB38009060B4F85E309BB2002B95D1216851E843
:10AB4800003F23F4807341E8003023680028F5D1E2
:10AB580003F1080252E8001F01EA0A0142E8001066
:10AB68000028F5D120215B45C4F88C106067206768
:10AB78000AD05968090207D553E8001F21F08061FF
:10AB880043E800100028F7D1E16E012913D1E666E9
:10AB980053E8001F21F0100143E800100028F7D106
:10ABA800D969CA0644BF102119622046B4F85C105E
:10ABB800FFF730FC58E72046F8F792FA54E79A690D
:10ABC80042F008029A6173E7FEFFFFEF0080004041
:10ABD800E5A7000838B5044603682169A2681D681E
:10ABE800C0690A4361690A437D49024329400A430F
:10ABF8001A605A68E16822F440520A435A60794A56
:10AC0800A16993421CBF226A11439A6822F06E42DE
:10AC180022F430620A439A60DA6A616A22F00F020B
:10AC28000A43DA62704A93421CD14FF0B043D3F81A
:10AC3800883003F0030343F44033A3F54033013B6A
:10AC4800022B00F2C780694A9B5CB0F5004F40F0C8
:10AC58008980082B24D8DFE803F061C08323802390
:10AC680023236500624A934209D14FF0B043614AF9
:10AC7800D3F8883003F00C0343F44023E4E7594A3F
:10AC880093420DD14FF0B043D3F8883003F44063BA
:10AC9800B3F5006F1AD005D853B1B3F5806F12D051
:10ACA800012009E0B3F5406FFAD14FF400400EE0FF
:10ACB800FEF7D2FC58B900204FF00113A366002319
:10ACC800C4E91D3338BDFEF7CFF8F3E74A48656895
:10ACD8004A4B626A05EB450133F81220B0FBF2F3E8
:10ACE8009942DDD8B3EB053FDAD800231946F6F7C9
:10ACF8000BFF090241EA10616B080002C0182A46DE
:10AD08004FF0000341F10001F6F7FEFE3C4BA0F5C1
:10AD180040729A42C4D82368D860CCE7FEF79CFCFE
:10AD28000028C8D06168354B626A33F81220B0FB3E
:10AD3800F2F24B0803EB42034FF6EF72B3FBF1F369
:10AD4800A3F110019142ABD823F00F02216892B20F
:10AD5800C3F342031343CB60ADE7FEF785F8DFE7A3
:10AD68002548DFE7082B9BD801A252F823F000BF43
:10AD7800C1AD0008CDAD0008D9AD0008A9AC0008E8
:10AD8800D3AD0008A9AC0008A9AC0008A9AC00081C
:10AD98009DAD00084FF400406368616A174A32F8B5
:10ADA8001120B0FBF2F000EB5300B0FBF3F04FF6CC
:10ADB800EF73A0F11002ACE7FEF74EFC00283FF459
:10ADC8007AAFE9E7FEF758FCF8E7FEF74DF8F5E744
:10ADD8000948E1E7B0F5004FF4D1FEF74DFC9FE7D5
:10ADE800F369FFCF0080004000380140DC520108C1
:10ADF80000440040DF52F5070024F400EC5201083B
:10AE0800FFFC0F00836ADA0710B506D50168C46A2B
:10AE18004A6822F4003222434A609C0706D501683A
:10AE2800046B4A6822F4803222434A60590706D5E7
:10AE38000168446B4A6822F4802222434A601A0758
:10AE480006D50168846B4A6822F4004222434A60AE
:10AE5800DC0606D50168C46B8A6822F48052224356
:10AE68008A60990606D50168046C8A6822F4005243
:10AE780022438A605A060FD50168446C4A6822F456
:10AE880080122243B4F5801F4A6005D14A68846C59
:10AE980022F4C00222434A601B0606D50268C16C30
:10AEA800536823F400230B43536010BD2DE9F04190
:10AEB800DDF8188004460E4615461F462268D369F9
:10AEC80036EA03030CBF01230023AB4201D0002064
:10AED80027E0B8F1FF3FF2D0F7F72AFEC01B404544
:10AEE800206802D8B8F1000F1DD150E8003F23F4C4
:10AEF800D07340E80032002AF7D100F1080353E884
:10AF0800003F23F0010300F1080141E80032002A64
:10AF1800F3D12023C4F88830C4F88C3084F8842016
:10AF28000320BDE8F08103685A07C7D5C3691B052C
:10AF3800C4D54FF40063036250E8003F23F4D07394
:10AF480040E80032002AF7D100F1080353E8003F37
:10AF580023F0010300F1080141E80032002AF3D18F
:10AF68002023C4F88830C4F88C30C4F89030D5E772
:10AF780073B504460026C0F89060F7F7D9FD23683A
:10AF88001B681A07054619D423681B685B070AD58E
:10AF98006FF07E43009300222B464FF48001204639
:10AFA800FFF784FFB0B900202023C4F8883084F864
:10AFB8008400C4F88C30E06620670CE06FF07E43B4
:10AFC8000093324603464FF400112046FFF76EFF08
:10AFD8000028D9D0032002B070BD10B5044650B384
:10AFE800D0F888301BB980F88430F7F757FF22680B
:10AFF8002423C4F88830136823F001031360204623
:10B00800FFF7E8FD012816D0A36A13B12046FFF721
:10B01800F9FE23685A6822F490425A609A6822F02E
:10B028002A029A601A6842F0010220461A60BDE8B6
:10B038001040FFF79DBF012010BD000030B58165AD
:10B048008168A0F85C200023B1F5805FA0F85E203D
:10B05800436735D10369002B40F2FF1318BFFF2364
:10B06800A0F860300023C0F890302223C0F88C305C
:10B07800016801F1080353E8003F43F00103083178
:10B0880041E800340368002CF2D1456E84680169F8
:10B09800B5F1005F34D1B0F86850954230D8B4F5B6
:10B0A800805F1DD1254A264C002918BF22464267D9
:10B0B800C1B153E8002F42F4807243E80021F7E75A
:10B0C80029B90369002B14BF7F23FF23C8E7B1F117
:10B0D800805FC5D10369002B0CBF7F233F23BFE7E7
:10B0E800174AE4E703F1080252E8002F42F08052C1
:10B0F80003F1080040E800210029F3D1002030BD09
:10B10800B4F5805F0FD10F4A0F4C002918BF2246B3
:10B11800426751B153E8002F42F4907243E800218E
:10B128000029F7D1EAE7084AF2E753E8002F42F08E
:10B13800200243E800210029F7D1DFE745AA0008EB
:10B14800A9A80008E5A7000819A70008D0F88C30BE
:10B15800202B30B415D1B9B1B2B100230468C3664D
:10B168000A4B9C420AD063681B0207D554E8003F8B
:10B1780043F0806344E80035002DF7D130BCFFF779
:10B188005DBF022030BC70470120FBE70080004013
:10B19800436E30B52BB90123A0F86A30A0F86830A7
:10B1A80030BD0368094D9A689968094C490FC2F384
:10B1B80042626B5C615CDB00B3FBF1F3A0F86A30C0
:10B1C800AB5CA25CDB00B3FBF2F3E7E70C530108CE
:10B1D800045301087047704770471FB504AB03E973
:10B1E800060090F88430012B04463AD0012380F8F9
:10B1F80084302423C0F8883003681A6822F00102DA
:10B208001A609A6822F440120A439A6071B95A681F
:10B21800BDF80C009DF80E1022F0100202435A608F
:10B228005A6822F07F4242EA01625A601A6842F084
:10B2380001021A60F7F77CFC6FF07E420346009229
:10B248004FF4800100222046FFF730FE38B9202352
:10B25800C4F88830002384F8843004B010BD03207B
:10B26800F8E70220F9E790F88430012B0FD001238A
:10B2780080F88430016851E8002F42F0020241E86A
:10B288000023002BF6D180F884301846704702203E
:10B29800704710B590F88430012B044617D024234A
:10B2A800C0F8883003681A68196821F0010119602C
:10B2B80042F000524FF0005141661A60FFF768FFF4
:10B2C8002023C0F88830002084F8840010BD0220B4
:10B2D800FCE770B590F88430012B044617D0056858
:10B2E8002423C0F888302E682B6823F001032B60D4
:10B2F800AB6823F060431943A960FFF749FF202397
:10B308002E60C0F88830002084F8840070BD0220C8
:10B31800FCE770B590F88430012B044617D0056817
:10B328002423C0F888302E682B6823F001032B6093
:10B33800AB6823F060631943A960FFF729FF202356
:10B348002E60C0F88830002084F8840070BD022088
:10B35800FCE7000038B5084D052455F8043B2BB927
:10B36800013C14F0FF04F8D1204638BDDB6898474B
:10B378000028F5D0F9E700BF64100020034BD8700F
:10B38800034B1B681B6C03B11847704778100020EB
:10B3980060100020034B1874034B1B685B6C03B1EF
:10B3A800184770477810002060100020F0B5314D24
:10B3B800314B95F90420314E91B00C46012795F98F
:10B3C80005108DF8047002288DF809208DF80A10F0
:10B3D80010D18DF80800D8711C7202F09FFD3378E7
:10B3E80003B114B101A803F003FA254B059A1A60BA
:10B3F80011B0F0BD59714FF480711A71D9801C7267
:10B4080033788DF8087053BB1F2306A88DF81C20CD
:10B418008DF8183002F064FF20238DF8183006A844
:10B428002B798DF81C3002F05BFF22238DF8183041
:10B4380006A86B798DF81C3002F052FF21238DF895
:10B44800183006A86B798DF81C3002F049FF2923C3
:10B458008DF8183006A80B4B079302F041FF02F055
:10B468005DFD012306A88DF818308DF81C3002F018
:10B4780037FFB4E77810002030080020541000206F
:10B4880058100020000400017FB5092301A88DF899
:10B49800043003F0ADF90038044B059A1A6018BF60
:10B4A8000120404207B05DF804FB00BF581000209F
:10B4B80070B504460B46134962784A700020A2789A
:10B4C8000A7208701A884A729A788A72DB780B7442
:10B4D8006368CB600C4B1B68DA6A2AB1237803F0E7
:10B4E800FB030A2B00D09047084E052556F8043B6D
:10B4F8001BB15B6A0BB120469847013D15F0FF056B
:10B50800F4D170BD3C0800206010002064100020B9
:10B5180070B5044610480123037063784370A3781C
:10B528008372E368C360E3780376236943762379FB
:10B5380043720A4B1B689B6A03B19847084E05255E
:10B5480056F8043B1BB19B690BB120469847013D57
:10B5580015F0FF05F4D170BD5008002060100020E0
:10B5680064100020014B1868704700BF5810002075
:10B5780000B58BB0012368468DF8003002F088FDD5
:10B5880038B99DF80400003818BF01200BB05DF8E9
:10B5980004FB0020FAE7000008B501F073FE48B983
:10B5A800FFF7E6FF012806D0054BD879197AFFF78F
:10B5B800FDFE012008BDBDE80840FFF7CBBE00BF77
:10B5C800300800202DE9F04186B005460E461746A2
:10B5D80001F058FE00287FD101F06CFE044640B906
:10B5E800FFF7C6FF012807D03D4B197AD879FFF736
:10B5F800DDFE6FF0020462E0DFF8E88088F808609A
:10B60800003E18BF01268DF80460374E68783379FC
:10B618008DF81230694602F0D9FC00283ED08DF82A
:10B6280004400394ADF810406FF0060495E8030059
:10B638002E4B83E80300337988F80A30394601A88D
:10B6480003F0DAF92A4B059A1A60112841D801A3A8
:10B6580053F820F0BBB60008E1B60008DBB60008D6
:10B66800DBB60008DBB60008DBB60008DBB600086E
:10B67800FBB50008DBB60008DBB60008DBB600083F
:10B68800D5B60008DBB60008DBB60008E1B600084E
:10B69800E1B60008E1B60008CFB600082B788DF8AF
:10B6A80008306B78ADF810306B6803934FF0FF34B7
:10B6B800BCE7104B00221A70E31D18BF1446204641
:10B6C80006B0BDE8F0816FF00404F8E76FF00504F8
:10B6D800F5E74FF0FF34F2E76FF00104EFE700BF42
:10B6E8003008002050080020781000206008002052
:10B6F800581000205C10002037B501F0E5FD144D0E
:10B70800052455F8043B5BB11B694BB155F8043C63
:10B718009B682BB1984718B155F8043C1B699847AA
:10B72800013C14F0FF04ECD1FFF714FE68B9094D91
:10B738002B7853B1084BADF80040D97801942246D4
:10B748006846FFF73FFF00B92C7003B030BD00BF5B
:10B75800641000205C1000207810002030B58BB0F9
:10B76800054601F08FFD0446002839D1FFF700FF98
:10B77800012838D168468DF8004002F089FC10B1E4
:10B788004FF0FF3004E09DF80430AB4202D10020B6
:10B798000BB030BD012DF3D0022D11D0002DF7D103
:10B7A800002BF4D068468DF8045002F099FD00286B
:10B7B800E6D10E4B1B681B6B002BE8D09847E6E7D9
:10B7C800002BDDD168468DF8045002F089FD002871
:10B7D800D6D1064B1B681B6B002BD8D02846EDE74B
:10B7E8006FF00100D4E76FF00200D1E7601000208D
:10B7F80010B504468AB018B94FF0FF300AB010BD32
:10B80800002368468DF8003002F042FC0028F3D18E
:10B818009DF804302370F1E77FB500220B462049DC
:10B828008DF8072001220A7042784A700446002ADF
:10B8380033D102790A721A884A729A788A72DB7846
:10B848000B740369CB60C378164D8DF80830037B01
:10B858008DF80930836803932B68DB6A0BB102A863
:10B8680098472B689B6B13B1227E02B198470E4E06
:10B87800052556F8043B1BB1DB690BB120469847F8
:10B88800013D15F0FF05F4D10DF10700FFF7B0FFFA
:10B89800637913B1054B01221A7004B070BD00BF63
:10B8A8003C08002060100020641000205C1000207C
:10B8B80010B504468AB018B94FF0FF300AB010BD71
:10B8C800202368468DF8003002F0E2FB0028F3D10F
:10B8D800024A9DF9043023701371EFE778100020B5
:10B8E80000B58BB02323019068468DF8003002F034
:10B8F800F7FC003818BF012040420BB05DF804FB8C
:10B9080070B5654C01468EB01822204606F0ECF85A
:10B91800624B00221A70F8F745FE2378406801222E
:10B9280002FA03F1014004D15D4B084608F0D2F851
:10B93800FEE75C495C481A4602F032F918B14FF04C
:10B94800FF300EB070BD272304A88DF8103002F028
:10B95800C7FC564E564D002870D1012333702B6812
:10B96800DB690BB100209847272304A88DF8103015
:10B9780002F08EFB059B93F84820227093F818215B
:10B9880093F81A316270A370464BD3E9020105F0AF
:10B998009DFF05460028D2D1464E062304A88DF8FF
:10B9A800103002F075FB059B736104A802F098FC47
:10B9B800022304A88DF81030059602F069FB0836BA
:10B9C800032304A88DF81030059602F061FB0F26BA
:10B9D80006F040F8012304A88DF814308DF81060A3
:10B9E80002F07EFC10230DEB03008DF810308DF86B
:10B9F800145002F075FC04238DF8103004A8A378C5
:10BA08008DF8143002F06CFC3A238DF8103004A83D
:10BA18006369059302F064FC02A920788DF8086038
:10BA280004F0E4F8003818BF0120E0711420FFF793
:10BA380057FFE07903F0A4F9284682E728238DF818
:10BA480010302B681B6943B104A802F021FB2B6856
:10BA580005981B6940F2C4519847272304A88DF81C
:10BA6800103002F03DFC50B9012304A88DF81030C5
:10BA780002F00EFB9DF81430002B7FF46EAF337884
:10BA8800002B7FF46CAF052204A88DF810200593D5
:10BA980002F026FC78E700BF781000205C10002038
:10BAA80014530108A0100020B810002054100020E2
:10BAB800601000203C10002037B500230D4601938C
:10BAC8000446D0B900F0A8FB0190019BD3B10F4AFE
:10BAD80042F824300E4A9A620E4A1268916B196332
:10BAE800916C596392690C49D9625A6128465B681E
:10BAF8000A49F2229847002006E001A900F092FBCB
:10BB08000028E2D04FF0FF3003B030BD64100020B1
:10BB1800B5B300086010002091B40008480F002059
:10BB2800194B07B51860194B194A1A60194A5A6017
:10BB3800194A9A60194ADA60194B02681A60426811
:10BB48005A6082689A60C268DA60164A1A61826925
:10BB58005A61154BC26B5A60144A019119609A6078
:10BB68001946134ADA600020FFF7A6FF48B901A872
:10BB780000F056FB003818BF0120404203B05DF8C2
:10BB880004FB4FF0FF30F9E760100020B8100020E8
:10BB980019B5000821B8000839BC0008B9B4000874
:10BBA800A0100020A5FB00089010002085B3000815
:10BBB8009DB3000851B118B1012804D00020704786
:10BBC800044B0B607047044B0B60F7E74FF0FF30F6
:10BBD800704700BF000400010100010208B503F02E
:10BBE800EBF8002814BF6FF00100002008BD08B56D
:10BBF80002F0BCF9002814BF6FF00100002008BD56
:10BC080010B504468AB018B94FF0FF300AB010BD1D
:10BC1800212368468DF8003002F03AFA0028F3D163
:10BC2800024A9DF9043023705371EFE77810002021
:10BC38002DE9F0412E4D2F4F00232B7043786B7068
:10BC48003B689B6A8AB004460BB128469847DFF8E0
:10BC5800A880052658F8043B1BB11B6A0BB1204687
:10BC68009847013E16F0FF06F4D12378052B2FD014
:10BC78000B2B35D0012B25D1204C062368468DF897
:10BC8800003002F005FA0199E07905F065FE10B977
:10BC98001B4B019A5A611B48FFF70AFE1A48FFF727
:10BCA800AFFF6B788BB9A371184B5878FFF756FD27
:10BCB8003B685B6A0BB1114898476B7813B9E07918
:10BCC80005F0DAFE0AB0BDE8F081FF23A371EFE7C3
:10BCD8000F4B01225A74227A9A74627ADA74F1E765
:10BCE8006378002BEED00AB0BDE8F041FFF7CCBB7B
:10BCF8005008002060100020641000203008002048
:10BD08003C1000203408002035080020781000205E
:10BD18003C08002030B58BB0FFF769FF0446F0B946
:10BD280003F044FF831C1DD0F8B9134D2B685B69E1
:10BD3800DBB1272368468DF8003002F0A9F92B689B
:10BD480001985B694FF4B961984703F041FF78B9EE
:10BD58002CB9094B1B68DB690BB1012098472046B9
:10BD68000BB030BD6FF00704EFE74FF0FF34ECE79E
:10BD78004FF0FF34F3E700BF60100020014B187844
:10BD8800704700BFCC100020014B5878704700BFA7
:10BD9800CC10002070470000044B9A7A0AB10122A7
:10BDA8005A70034B5B6903B118477047CC100020E9
:10BDB8006C08002073B5224C6378002B33D008F050
:10BDC80073F966680546FFF7CDFB0644AE4214D208
:10BDD800A37A93B1E0228DF800208DF80130217A02
:10BDE800E368019301226846FFF7ECFB08B10730CE
:10BDF80010D100236370A372656094F83430EBB1FE
:10BE0800002384F834300F4B5B6BBBB102B0BDE844
:10BE18007040184740F2DC510B4808F011FA0A4804
:10BE280008F0D4F9E8E794F83520002AE5D094F82A
:10BE3800360084F83530FFF791FCDEE702B070BDBC
:10BE4800CC1000206C0800200411002037B5104DDC
:10BE5800104CC8B1C1B10123627200222860E160B0
:10BE680023700D480D4B00924FF0FF3108F002F996
:10BE780000250B4825822022294605F049FE6570D9
:10BE8800A574A58603B030BD00232B602370EFE7AF
:10BE9800C8100020CC10002004110020A1BD00080B
:10BEA800E01000202DE9F0478E4C23788CB0002B51
:10BEB80056D0C2780AB9837B13B1238A013323820F
:10BEC800437B002B4CD0E02A4AD10023A372876819
:10BED80097F80080B8F1220F27D8B8F1220F30D890
:10BEE800DFE818F04100FB0052005A0061006E00C4
:10BEF80075008E009D00B400C7002F002F002F0092
:10BF08002F002F002F002F002F002F002F002F00B1
:10BF18002F002F002F002F002F002F002F002F00A1
:10BF28002F002F00C900D000D400B8F17E0F00F018
:10BF3800CC80B8F17F0F00F0DF80B8F17D0F00F002
:10BF4800AB80A57A002D00F05B81674C637A3BB922
:10BF58004FF47A71204608F073F9204608F036F954
:10BF68000CB0BDE8F087E36801220021A2721970C5
:10BF7800A37AE1689818A0720620C854A37AE168E9
:10BF88009818A072CA54DCE7584B9B6A002BD8D08B
:10BF9800012102209847D4E77B7884F836300123C2
:10BFA80084F83530CDE704238DF804307B78003BE6
:10BFB80018BF012301A88DF8083002F091F9C0E7F5
:10BFC8007878003818BF012002F0DAFEB9E7484E49
:10BFD8000FCE01AD0FC50FCE0FC596E8070085E857
:10BFE80007007B780A2BACD8424A12685268002AAC
:10BFF800A7D00CA901EB830353F82C0C9047A0E7BA
:10C008007878431E012B9CD83A4B01381B6818BF1F
:10C01800012020729B68002B93D0984791E7E26833
:10C0280001230821A3721170627A057BA17AAA42C2
:10C0380028BF2A46934284D285685A1CEB5CE5687F
:10C0480001334E1CA6726B54D3B2EDE7E3680122AC
:10C05800A27209221A70A37AE268218A581CA07277
:10C06800D154A27A238AE1681B0A501CA0728B540F
:10C0780067E7238265E705238DF8043001A802F0FD
:10C08800B7FB5EE7194BDB6A98475AE7194B787894
:10C098001B686075DB68BEE7037B072B7FF451AF35
:10C0A80006238DF80430B7F80130ADF808307B79F5
:10C0B8003A791B0443EA0223FA7813436422534370
:10C0C8000393BB798DF81030D8E73B2201A88DF88F
:10C0D80004208DF8083002F003F9012384F8343085
:10C0E8002FE700BFCC100020041100206C080020AE
:10C0F8001C470108C81000202A2301A88DF8043025
:10C1080001F0C6FF94F80A90E6689DF808009DF8CB
:10C1180009509DF80A709DF80BC09DF80D309DF8E8
:10C128000E209DF80F109DF80CE009F1010A84F823
:10C138000AA006F80980354E94F80A903668D4F8B3
:10C148000C8009F1010A84F80AA096F803A008F8FF
:10C1580009A094F80A90D4F80C8009F1010A84F82F
:10C168000AA096F802A008F809A094F80A90D4F852
:10C178000C8009F1010A84F80AA096F801A008F8D1
:10C1880009A094F80A9009F1010A84F80AA096F81F
:10C198000080E66806F8098094F80A80E66808F1E5
:10C1A800010984F80A9006F808C094F80AC0E668FD
:10C1B8000CF1010884F80A8006F80C70A77AE66882
:10C1C80007F1010C84F80AC0F555A57AE6686F1CDA
:10C1D800A7727055A07AE568461CA6722954A17A00
:10C1E800E0684D1CA5724254A27AE168501CA07206
:10C1F8008B54A37AE268591CA17202F803E0A0E606
:10C20800034807F095FF6570AAE600BFC810002034
:10C218000411002070470000004870476C08002097
:10C22800002070474FF0FF3070470000044B054A6C
:10C2380093F81831022B18BF062382F89034704700
:10C24800E0160020A81C0020034BD3F8483313B194
:10C258005B6903B118477047A81C0020034A13788C
:10C2680043F004031370FFF7EFBF00BFA41C0020C6
:10C278001FB50A4B8DF8090093F87C208DF80A2029
:10C2880093F88C2093F848000D3202A98DF8082005
:10C2980003F0ACFCC0B205B05DF804FBE01600206A
:10C2A80010B5074C04F5806007F042FF94F81A3483
:10C2B80013B1012384F81934BDE81040FFF7C4BF57
:10C2C800A81C002010B50C4CD4F8403343F0800370
:10C2D800C4F8403394F81A3413B10020FFF7E0FF94
:10C2E80094F8913423F0120343F0120384F8913444
:10C2F800BDE81040FFF79ABFA81C00202DE9F041C7
:10C30800DFF8AC8098F81831022B06460D4602D0AB
:10C31800284BDB6A984702F0E9FD044628B1022061
:10C3280002F0DAFD002002F0DCFD98F81831012B4C
:10C3380017D102F0DDFD074630B1002002F0CDFD37
:10C34800002002F0CFFD3C4602F0D4FD48B10020A9
:10C3580002F0C4FD002002F0C6FDBDE8F041FFF781
:10C3680065BF002CF9D1144C94F8902494F81A3431
:10C37800BAB90BB184F84164304602F065FFD8F8C9
:10C388002C0007F09BFED4F8B4339842E5D30B4851
:10C3980007F0CEFE94F8913443F0100384F89134FA
:10C3A800DBE70BB184F84154284602F04DFFF1E772
:10C3B800E0160020945A0108A81C00204020002004
:10C3C80073B5164C164D04F57A76EB6C95F850203B
:10C3D80095F9781095F84800009603F02DFC95F82B
:10C3E800303184F8FC3395F8480040F2012304F218
:10C3F80024423146A4F8FA3303F02AFC58B194F8E1
:10C40800243484F86A34074B00205B6B984794F80F
:10C41800FB3384F8903402B070BD00BFA81C002024
:10C42800E0160020945A0108074A10B5137843F023
:10C4380002031370FFF708FFBDE81040034B012209
:10C448000021022007F046BBA41C00205D53010810
:10C45800074A10B5137843F008031370FFF7F4FE8A
:10C46800BDE81040034B01220021022007F032BB37
:10C47800A41C00206D5301082DE9F0410F46164613
:10C488001D46804607F010FE0B4A0C4C1378278196
:10C4980023F0110343F011031370C4E90008668107
:10C4A8002573FFF7D1FEBDE8F041054B01220021BD
:10C4B800022007F00FBB00BFA41C0020542200205C
:10C4C8007D53010813B507F0EFFD0D4B6C4618605E
:10C4D800204607F03DFD94E803000A4A0A4B83E82A
:10C4E8000300137843F020031370FFF7ADFE074BEA
:10C4F80001220021022002B0BDE8104007F0EABA8C
:10C5080064220020A41C0020E01F00208A53010898
:10C51800F8B5334D95F81841012C06464BD0022C3E
:10C5280051D064B938B9D5E91B0105F1740383E822
:10C5380003002046F8BD01283DD0022801D003247D
:10C54800F7E7284F85F8180107F5747EBEE80F0055
:10C5580007F57A7CACE80F009EE8030095F8E9300F
:10C568008CE8030087F8FB63E3B195F80031022BF0
:10C5780018D1D5F804316B67C7F8EC3395F87D30DE
:10C5880095F8082187F8F83395F88C3085F87820E5
:10C5980087F8F93397F81B2487F8E82340F201332A
:10C5A800A7F8FA33002387F81A340F4BDB6A984749
:10C5B800FFF706FFBDE702F0A4FC04460028B8D147
:10C5C80085F81861B5E70028B9D1064B85F8180138
:10C5D800062283F89024044BDB6A98473446A8E780
:10C5E800E0160020A81C0020945A01082DE9F0410B
:10C5F80092B0064602F07AFC002840F05981AD4D11
:10C6080095F81831012B09D02B6BAB4C93B194F8EA
:10C618000431BBB1042B6FD0032003E002F068FCA7
:10C6280018B10F2012B0BDE8F08102F063FC0028B9
:10C63800EAD0F6E7B5F82031D4F81C24013B53437F
:10C648002B63E4E79D4803F008FA002840F02C81AA
:10C6580094F80C3123802B6B0C930DF1180895F886
:10C6680039308DF83830404695F81C318DF83A301D
:10C6780007F094FCD5F82831009302AF98E806003B
:10C68800D5F82431384607F020FC97E803000FABB3
:10C6980083E80300EB6A0D9300238DF84430238868
:10C6A800ADF8463095F8303101228DF839201BB9A4
:10C6B8008DF844208DF83930814B0093814B95F8E3
:10C6C8004800A3F179020CA903F005FBC0B10B28BF
:10C6D800A8D1D4F8941499B1002EA3D0D4F840333B
:10C6E800794843F02003C4F8403307F0A9FD7648A1
:10C6F80007F06CFD002095E7704803F0E2F9A4E725
:10C7080095F8487095F9693095F9392095F87D10B4
:10C718006E4E384603F0ECFA009641B2EB6C95F891
:10C7280050203846183603F087FA0096EB6C95F8D7
:10C73800502095F9701095F8480003F07DFAD4F868
:10C74800C413AB6DD4F8DC230B44C4F8B033EB6DE1
:10C758001344C4F8B43394F80431042B07D02B6E77
:10C768000B44C4F8B0336B6E1344C4F8B4330023DD
:10C77800089395F8303183B108A802F095FC002899
:10C788004ED195F9390094F837629DF82070FFF77B
:10C798006FFD3E4480B2B04240D300238DF8133081
:10C7A80095F839308DF8213095F838308DF82230E9
:10C7B800D5F880300993D5F884300A932388ADF8EA
:10C7C8002C3095F8303194F81B648DF82E3095F89C
:10C7D80048003F4B8DF820600DF1130208A903F0C3
:10C7E8003FFA012384F8413495F8393084F842340B
:10C7F8009DF8133084F84334D4F81C34C4F85064DA
:10C80800C4F84834C4F8583402F076FB50B1D4F870
:10C818001C0402F083FB28B1102003E7082001E77D
:10C828001320FFE695F81831012B01D102F078FBAF
:10C8380002F065FB0023059394F8043195F939500B
:10C8480094F81B649BB1042B7FF4E6AE05A802F0B4
:10C8580067FE58BB94F8183413B1059B013B059348
:10C86800164B05983246E9B202F0BCFE02E01348C6
:10C8780002F090FEC0B9D4F8403394F80C1121802E
:10C8880043F00203C4F8403394F8183411480133D4
:10C89800DBB284F8183484F845340F4B00259B6AC2
:10C8A800C4F89854984725E71120BBE61220B9E64A
:10C8B8000E20B7E6E0160020A81C0020B01D0020BE
:10C8C800101700203C2100201020002060200020AC
:10C8D800C4200020AA1C0020945A0108F0B5504C2E
:10C8E800504EB4F8DC202287D4E92D0194F8B12009
:10C8F80084F8692004F16C0282E80300D4E92F016E
:10C9080004F1740282E80300B4F8C420A4F87C207F
:10C9180091B0D4F8CC20D4F8C810C4F884200025ED
:10C92800D4F8D020C4F888200123A4F82031C4F812
:10C93800801084F83051A56284F81B5184F83A506D
:10C9480084F81D5184F81E51C4F83451C6F898541F
:10C95800A6F8185486F81A54A4F838518DF81830E7
:10C9680004F50973039304F50A7394F84800A4F8CE
:10C978004651049303A92C4B84F84551C4E94F55FB
:10C98800059303F041F9E36EC6F8D43394F87D308B
:10C9980086F8E03394F88C3086F8E1334FF48073EE
:10C9A800A6F8E23386F8D05394F8303186F8E433A9
:10C9B80006F574770FCF06F57A740FC497E803006D
:10C9C80040F2012384E80300A6F8FA33D6F8483386
:10C9D80086F81B54CDE901551BB15A685B69019271
:10C9E8000293124B0793A3F148020892A3F1140291
:10C9F80009920F4A0B9229330A93A2F19C030C93D4
:10CA0800A2F198030D93131D0E9301A902F14C0393
:10CA180007A802F599620F9302F05DFA11B0F0BD14
:10CA2800E0160020A81C0020C421002010210020AE
:10CA3800C4170020F8B50D4F0D4C0E4E0D4607F0EB
:10CA480077FB3B6B984796F8480004F22442294646
:10CA580003F0FEF848B194F8243484F86A34706D11
:10CA68007B6B9847EB7C84F89034F8BD945A0108A6
:10CA7800A81C0020E01600200F4890F81B3480F80E
:10CA8800B8330E4B93F8692080F8BB2393F87D20C8
:10CA980080F8C82393F88C2080F8C92393F83031A4
:10CAA80080F8CC330022A0F8CA2300F56E7100F597
:10CAB8006070FFF7BFBF00BFA81C0020E016002071
:10CAC800114890F89034EBB190F81B3480F8D033CB
:10CAD8000E4BDA6EC0F8D42393F87D2080F8E0235B
:10CAE80093F88C2080F8E12393F8303180F8E43310
:10CAF8004FF48072A0F8E22300F5747100F56670B7
:10CB0800FFF798BF704700BFA81C0020E016002060
:10CB180070B5344C2421204604F0FCFF636A984227
:10CB280018BF60624FF01C012F4814BF0125002573
:10CB380004F0F0FF636C984218BF60644FF4807192
:10CB48002A4818BF45F0020504F0E4FFD4F848313C
:10CB5800984218BFC4F848014FF0D401244818BFC0
:10CB680045F0040504F0D6FFD4F82032984218BFE7
:10CB7800C4F820024FF000011E4818BF45F0080510
:10CB880004F0C8FFD4F82432984218BFC4F824022D
:10CB98004FF46071184818BF45F0100504F0BAFF4B
:10CBA800D4F8A835984218BFC4F8A8054FF0140166
:10CBB800124818BF45F0200504F0ACFFD4F8C03582
:10CBC80098420F4B18BFC4F8C005D3F8483318BFB4
:10CBD80045F040052BB11B691BB12846BDE87040E4
:10CBE800184770BDE01600200817002028170020FD
:10CBF8002C18002004190020081900208C1C002083
:10CC0800A81C00202DE9F04F91B04FF00008012B2F
:10CC180005460F4602928DF81580ADF8188003D8A6
:10CC2800C84EC146B94502D311B0BDE8F08F15F81A
:10CC3800090002F077FA4844B842F5DC15F80930E3
:10CC480009F10104023BE4B2112BEDD801A252F81C
:10CC580023F000BFA5CC0008D7CC0008D7CD00082A
:10CC680001CE000889CE0008B1CE000823CF000805
:10CC780055CF0008D1CF000831CC000831CC0008CE
:10CC88002FD0000831CC000831CC0008EDD00008C6
:10CC980015D1000859D1000897D10008052002F0E5
:10CCA800EDFA90B10521002002F0ACFA2A5DA64BFE
:10CCB80009F1030409F102095FFA89F983F85C2490
:10CCC80015F8092083F85D24E4B2A146AAE70023F9
:10CCD8008DF816308DF817308DF81C308DF820300F
:10CCE800B8F1000F6CD14FF0050896F87C208DF84C
:10CCF8003920631E96F839208DF83B202B4496F88E
:10CD080038200D938DF83C2096F81A3196F8682053
:10CD18008DF83D20D6F82C218DF83A300C9273B35B
:10CD28007B1C1B1BDBB28DF8383008AB019307ABBB
:10CD3800009396F848000DF117030DF116020CA99F
:10CD480002F09AFF8DF8150000F00700072813D1AC
:10CD580096F939209DF9163086F839309A429DF8AF
:10CD6800173086F83830B8BF01229DF81C30B8BF9C
:10CD780086F81D2186F868304FF0000909E0052380
:10CD8800D1E701220DF11501032002F0DBF809F1CA
:10CD980001095FFA89F29DF82030B3FBF8F191425E
:10CDA800EFD82344DCB2631EDBB29F420DD9EA5CA4
:10CDB800032A9AD0A74288BF1C464FF0010884E78F
:10CDC80009F105095FFA89F4F7E71C46F5E72B5DD9
:10CDD800012203F00F0309F1020986F81B3102FA58
:10CDE80003F35FFA89F9A6F82031002206A9042086
:10CDF80002F0A8F84C4668E707238DF815302B5D3C
:10CE080096F84800C3F3021203F00F038DF8303090
:10CE180009F10303DBB28DF83120EA5C09F1040360
:10CE2800DBB209F10504EB5C09F102095FFA89F943
:10CE38001B0443EA022315F80920134364225343D1
:10CE48000CA90D9302F027FF00F00703072BE4B2AB
:10CE58008DF815000CD19DF8303086F8703086F8C2
:10CE680078300D9BF36673679DF8313086F869302A
:10CE78008DF81800012206A9052002F063F824E7BE
:10CE8800314BD3F848336BB11B685BB19847029BB1
:10CE98008DF8180003F03F038DF81930022206A917
:10CEA8000620EAE7FF20F2E703238DF815302B5D13
:10CEB8008DF824300CAB089309F10303DBB209F1B8
:10CEC8000604EA5C96F8480009F10403DBB208A9F5
:10CED800EB5C1B0443EA022309F10202D2B209F116
:10CEE8000509AA5C1343642253435FFA89F90C933A
:10CEF80000230D9315F809308DF8383002F0D1FE73
:10CF0800C3B20028E4B28DF81530FFF6DEAE8DF816
:10CF18001830012206A90720AFE72B5D03F00F03A5
:10CF2800012B4FF47A7238BF0123534309F10209E8
:10CF3800B36513445FFA89F9F365002206A908204E
:10CF480056E700BFE0160020A81C00202B5D96F8CD
:10CF58004800C3F340128DF81D2007A9C3F300123F
:10CF680003F00F038DF81C208DF81E3002F09FFE91
:10CF780009F1020901305FFA89F93FF43BAFBDF8C6
:10CF88001C30914AA6F87C309DF81E309DF81C4054
:10CF9800D05CF4F73BFD0223C6F880000CA996F894
:10CFA80048008DF830308DF8324002F01FFE96F9B7
:10CFB8003930089040B29842B8BF184686F8390010
:10CFC800002206A9092013E703238DF815302B5DED
:10CFD8008DF8303009F10303DBB209F10504EA5C8E
:10CFE80096F8480009F10403DBB209F10209EB5C89
:10CFF8005FFA89F91B0443EA022315F80920134351
:10D00800642253430CA90D9302F057FEC3B20028C3
:10D01800E4B28DF81530FFF658AE8DF818300122BD
:10D0280006A90A2029E7092002F028F9DFF89CA1BF
:10D03800002854D00921002002F0E4F80023ADF8BC
:10D04800263009F10203DBB24FF47A71EA5C09F188
:10D058000303DBB20DF1300BEB5C1B0443EA022344
:10D068002A5D134309F10402D2B209F1060409F159
:10D078000509AA5C5FFA89F943EA026315F80920F1
:10D0880003934A4312125846ADF8242006F060FF75
:10D09800039B03F1965303F5A91303F5EC53089387
:10D0A800DAF83C3300930DF1200999E80600DAF824
:10D0B80038330AA806F009FF0B9B00939BE806008B
:10D0C8000A9B484606F0E6FE99E8030006F018FFBA
:10D0D80001F021FF0123E4B28AF83834F5E58AF833
:10D0E8003804F2E50C2002F0C9F800283FF4EDAD51
:10D0F8000C21002002F086F8344B93F89034043B5E
:10D10800012B7FF6E2AD01F002FFDEE509F1020333
:10D11800DBB22A5DE95C09F10303DBB209F105041E
:10D12800EB5C09F104095FFA89F91B0415F8090099
:10D1380043EA012313436421594300F00F0001F02F
:10D14800E7FEE4B28DF81800012206A9112094E642
:10D158000D2002F093F800283FF4B7AD0D21002010
:10D1680002F050F809F10203DBB2194AE85C2B5DC2
:10D17800126809F1040409F103095FFA89F943EA1D
:10D18800002015F80910E4B201F0C4FE9DE52A5DFF
:10D1980009F1020309F1040409F10309DBB25FFA9A
:10D1A80089F9E95C15F809301B0443EA01231343A4
:10D1B8006420584301F0B0FEE4B28DF81800012253
:10D1C80006A9132059E600BF97530108A81C0020A0
:10D1D800542200200E4B93F89124920703D593F81C
:10D1E8008F24012A08D90B4991F81A2122B18A6A99
:10D1F800501C18BF01328A620022A3F8182483F851
:10D208001A24D3F8402322F00202C3F840237047BF
:10D21800A81C0020E016002070B5184C184D04F525
:10D228005A7006F085FFD4F84033D4F89804D5F83E
:10D23800906023F02003C4F8403338B106F03EFF75
:10D24800864203D2002385F83A3070BD0120FFF7EB
:10D25800CDF90028F9D00B28F7D095F8393084F8A3
:10D268004234092094F8183484F8453484F8410489
:10D2780001F0EAFFBDE87040FFF7ACBFA81C002032
:10D28800E0160020094BD3F84023012A0AD00849A8
:10D298000978C90708D43AB993F89204013818BF35
:10D2A800012070470020704701207047A81C00200B
:10D2B800A41C0020034BD3F84003431E5842584196
:10D2C800704700BFA81C00202DE9F04FA9B0EFF36C
:10D2D800108272B6DFF8F4820021D8F80030C8F85E
:10D2E800001082F31088BA4C002B00F0E480DAB208
:10D2F8009B06039264D5B74D95F81831022B02D0DE
:10D30800B54BDB6A9847EFF3108972B6B34F06F056
:10D31800CBFE3E68D4F8B013361A3144B04806F054
:10D328008FFFAF4806F052FFD4F8B413AD4831442C
:10D3380006F086FFAB4806F049FF89F3108894F899
:10D348001A34002B00F06D81152312A995F84800B6
:10D358008DF8483002F04AFCD4F8B4130F90014419
:10D36800A14806F06DFFA04806F030FF3B6894F82E
:10D378001B24EB620DAF38468DF870201D9306F024
:10D388000DFED5F82831009306AE97E80600D5F8CB
:10D398002431304606F099FD96E803001FAB83E878
:10D3A8000300D4F81C341E9395F8303195F84800E2
:10D3B800003B18BF01231CA98DF8713002F01FFC37
:10D3C800039BDF064BD5834DDFF820A2D5F8E42078
:10D3D800BAF90A30059298F800200493002363F301
:10D3E80000020A9388F8002084F84434049AA4F8C8
:10D3F800223484F82534C4F82834A4F82C3484F86A
:10D408002E34C4F8303484F82034C4F8343484F822
:10D418003834C4F83C34704B9AF90C90A4F88C2436
:10D4280094F89024DB6A84F88E9484F88F24DAF8D0
:10D438000470BAF80860984794F88F3413B96948AB
:10D4480006F076FE3146384601F04EFD8346002848
:10D4580000F0EA80049BA4F87E3484F88094039B4F
:10D4680019071AD55B4B93F81831022B02D05A4B87
:10D47800DB6A98470220FEF7D9FE84F8410401F0E0
:10D48800E3FE94F81A3413B1012384F8193494F89C
:10D49800913443F0100384F89134039B5A0703D561
:10D4A80006210520FEF72AFF039B9B0703D50421CD
:10D4B8000320FEF723FF01F035FD94F89124D706E9
:10D4C8005FD5002384F89234D4F840331E0644BF55
:10D4D80023F08203C4F8403312F0050F00F0FC82F9
:10D4E8000B2001F0CBFE002800F0F68294F891346E
:10D4F800DD0700F1F182580740F10883D4F8403382
:10D5080023F00203C4F84033D4F8402382BB94F8D4
:10D51800915415F001011EBF2B4662F3000384F8F5
:10D52800913494F891345E0744BF6FF3820384F812
:10D538009134012384F8923421B1D4F844332C482F
:10D548001B6898476D070BD52A4801F0A3FE01F028
:10D55800D1FE28B194F8913443F0040384F891344F
:10D5680001F0CEFC94F891346FF3041384F89134ED
:10D57800012384F8923494F8913443F0200384F81A
:10D58800913494F8913418070AD56FF3C3031A49F4
:10D5980084F89134D4F84433A1F12400DB68984727
:10D5A80094F8913499070AD56FF34103124984F826
:10D5B8009134D4F84433A1F16C005B68984794F82F
:10D5C8009034022B1AD1FEF7FBFE17E0A41C0020B2
:10D5D800A81C0020E0160020945A010864220020AC
:10D5E8002820002040200020A820002054220020CD
:10D5F800E8200020FC2000203421002094F89134F9
:10D608009A0640F1C6826FF3451384F89134D4F832
:10D618004033002B40F0BD8229B0BDE8F04FFFF742
:10D6280077BA84F84134A1E695F81821012A0CD17B
:10D6380001F05EFC804668B1584601F04EFC584641
:10D6480001F050FC042384F88F347EB9012384F858
:10D65800213450E101F04EFC0028F6D0404601F09C
:10D668003DFC404601F03FFC0523ECE73B78049382
:10D678005B09013B062B00F21882DFE813F0070074
:10D68800160295001602920016020702102EDDD926
:10D6980095F830311297F6B28DF84C60002BD5D141
:10D6A8001CA804F04BF912AA1CA9FF2002F0AEF83E
:10D6B8009DF85830C3F3030307468DF82C3095F8CE
:10D6C800480095F87D308DF82D3007220BA902F01F
:10D6D800A0FA002F5DD100285BD09DF853309DF84B
:10D6E80052201599C5F8E4101B0443EA02239DF85B
:10D6F800512002201343C5F8E03004F02DF99DF8BD
:10D70800583095F8480085F82E71C3F30212C3F318
:10D71800030385F8703085F878309DF8593085F81E
:10D728006920012B38BF01234FF47A725343AB654C
:10D738001344EB650DF15A034FF001081093113EA5
:10D7480094F81B348DF83C300FA985F868808DF863
:10D75800446002F066FA0223404685F8303101F051
:10D768008DFD18B14146384601F04CFD94F88F34D0
:10D77800012B00F2A88194F81A34002B40F09B8109
:10D7880094F8913443F0100384F89134FEF74EFD79
:10D7980065E6012001F072FD0028E7D0012107208D
:10D7A800E2E7012384F8203495F87D308DF82E3097
:10D7B80094F824348DF82D3095F88C3095F848007D
:10D7C8000D330BA98DF82C3002F010FAA6F10D03D9
:10D7D8001BB2099023EAE37300B283423FF736AFE6
:10D7E8000B2E7FF633AFBB4B25931CA8FF231C974A
:10D7F8008DF874608DF8983002F0D4F80746002848
:10D808007FF424AF95F81831012B13D101F070FB88
:10D81800002873D0384601F060FB384601F062FBFF
:10D8280004239DF87C101E9884F88F34C1F30011EE
:10D8380001F077FB9DF87C301E99C4F8341413F07E
:10D848000F0203D09DF89000002863D19DF898003E
:10D85800002862D0002A7FF4F9AE9DF89020002AB3
:10D868000CBF4FF002084FF0030800220A92D5F8C7
:10D87800EC20914254D195F8E910002950D0D5F800
:10D888000C1195F8EAB009680A9195F8181102295F
:10D8980002D1032184F88F14B8F1030F7FF4D6AEB8
:10D8A80013F0600F7FF4D2AE0592012795F82E3160
:10D8B800BBF1000F37D0BBF1010F38D1012B34D1A8
:10D8C8006FF0090646FA08F606F00106C6F10206E8
:10D8D800F6B2BDF87E100AAA304601F02DFE40B31C
:10D8E80007280CBF0823012384F821340A9BC4F8B5
:10D8F8003034C4F86C34FEF7E5FCB0E501F0FAFA10
:10D90800002897D0384601F0E9FA384601F0EBFADA
:10D91800052386E74FF00008A7E74FF00108A4E7C2
:10D928004FF0010BC2E70426D3E70326D1E7012312
:10D93800DAE71CAB009305990A9B3246584601F07A
:10D94800B7FE20B102280CBF0A230B237FE60A9BEF
:10D95800C4F83034C4F86C349DF87C3084F8210461
:10D96800C3F3401384F82E3484F8443494F88F3485
:10D9780084F82274012B9EBF0122A86285F81E211B
:10D98800012FC4F8280484F82C0484F8410438D101
:10D99800022284F8202495F83A20002A4AD19DF8DA
:10D9A8007C20D60646D4012B94F840149DF87C20A0
:10D9B80005D8012901D1900601D501F05FFBB8F126
:10D9C800020F94F88F3443D0B8F1030F0AD09DF8B2
:10D9D8007C10B8F1010F4A4601F00F0120A83BD096
:10D9E800FFF710F99DF8903084F82334259BC4F88C
:10D9F80028349DF8983084F82C34012384F82D3489
:10DA080030E0049A02F0E002A02A1BD195F82E110A
:10DA1800012285F83A2009B927996963012B84F80E
:10DA2800202407D9D5F89020C4F83C24DAF800203F
:10DA3800C4F8982495F81821002AB4D1012284F852
:10DA48002524B0E7002285F83A2084F82024A6E7A8
:10DA58009DF8981025984A46FFF7D4F89DF890301D
:10DA680084F823349DF89020E02A08D195F81F31D6
:10DA78002BB984F82324C4F82834A4F82C3494F857
:10DA8800913443F0020384F891346FE6114D013E5E
:10DA9800B2B2791C284604F027F80323A4F82034EE
:10DAA800C4F8285484F82C64E9E7012384F8213465
:10DAB800FEF708FC5AE694F84434002B3FF460AEB5
:10DAC8000020FEF7EDFB94F88F34022B3FF45EAE96
:10DAD80056E600BFE01E002094F89134590715D58A
:10DAE800012001F0CBFB60B1012001F09DFB08B9DA
:10DAF80084F81804D4F8403323F00203C4F8403300
:10DB080004E0062001F0BAFB0028F3D194F8913420
:10DB1800DA077FF5F9AC94F840240AB1032A18D142
:10DB28001D4A94F8181492F86820914205D29B0770
:10DB380023D594F88F34012B1FD8184806F0F8FA2B
:10DB4800D4F8403323F02003C4F84033FFF742FBF6
:10DB5800DAE4012A11D194F81924002A3FF4D4AC4C
:10DB68000D4A94F8181492F868209142E5D29F075C
:10DB780003D594F84434002BDFD194F89134002075
:10DB88006FF3041384F8913484F81904FFF744FB05
:10DB9800BAE429B0BDE8F08FE0160020102000207C
:10DBA8002DE9F04F89468DB090460746002800F0D1
:10DBB8008F81002900F08C810368002B00F0888198
:10DBC8004368002B00F084818368002B00F080817B
:10DBD800C368002B00F07C81104602F003F800288F
:10DBE80000F07881BD4CBE4D384601F0C1FA40F2D4
:10DBF800C4520021204603F08BFF40F21C52002142
:10DC0800284603F085FFB74BC4F82C3104F5097397
:10DC1800089304F50A7300264046099308A9B24BF5
:10DC280084F848800A9384F8186184F88C608DF829
:10DC38002C6001F0E9FF0F2306A994F848008DF83D
:10DC4800183001F0D3FF801B18BF01204FF00A0BDA
:10DC580084F81C0106A994F848008DF818B001F062
:10DC6800C5FF4FF0060A84F8DC0006A994F84800BE
:10DC78008DF818A001F0BAFF102384F8DD0006A97A
:10DC880094F848008DF8183001F0B0FF1123C4F85B
:10DC98009C0006A994F848008DF8183001F0A6FFFA
:10DCA8001223C4F8A00006A994F848008DF818308B
:10DCB80001F09CFF1323C4F8A40006A994F84800B7
:10DCC8008DF8183001F092FF1423C4F8A80006A9B3
:10DCD80094F848008DF8183001F088FF1623C4F82E
:10DCE800AC0006A994F848008DF8183001F07EFFC2
:10DCF800172384F8B10006A994F848008DF8183065
:10DD080001F074FF18230DEB0301C4F8B400C4F844
:10DD1800BC0094F848008DF8183001F067FFC0B2D5
:10DD28001D2384F8B80084F8C00006A994F84800B8
:10DD38008DF8183001F05AFF1E2384F8C40006A994
:10DD480094F848008DF8183001F050FF1F2384F82C
:10DD5800C50006A994F848008DF8183001F046FF70
:10DD68002023C4F8C80006A994F848008DF8183094
:10DD780001F03CFF0B23C4F8CC0006A994F8480036
:10DD88008DF8183001F032FF0C2306A9A4F8D00052
:10DD980094F848008DF8183001F028FFD4F89C302A
:10DDA8006365D4F8A030A365D4F8A430E365D4F84B
:10DDB800A83023664FF00108D4F8AC300590A4F8D9
:10DDC800D200636684F8B080C4F894B084F898A050
:10DDD800C4F84CB084F850A084F8688084F81F8197
:10DDE800C5F84893FEF77AFD404B009632464FF04F
:10DDF800FF3105F55A70C5F84473C4E90B6684F819
:10DE0800198185F89164C5F8408306F033F9384BD9
:10DE1800009632464FF0FF3105F5607006F02AF99A
:10DE2800344B009632464FF0FF3105F5667006F028
:10DE380021F902AF304B009632464FF0FF3105F51D
:10DE4800806006F017F9384606F0A8F897E803004E
:10DE580004F5927383E80300284B294F1E60294B71
:10DE6800C5F84C33284BC5F85433284BC5F85C33F8
:10DE7800274BC5F85033274BC5F8583305F5537071
:10DE88003B68984704F5A67003F084FB20B111267F
:10DE980030460DB0BDE8F08F204601F01DFB00288C
:10DEA800F5D101F041F8B8B91B4801F067FB064607
:10DEB8000028ECD17B69984703F0F4FDBB6D94F81A
:10DEC80019019847FB6A9847012385F89234DFE7E0
:10DED8000326DDE70926DBE71326D9E7E01600204D
:10DEE800A81C002000040001C421002021D2000841
:10DEF80081CA0008C9CA0008A9C20008A41C0020D9
:10DF0800945A0108CDC4000881C4000865C20008FD
:10DF180059C4000831C40008C817002008B5034BCD
:10DF28000020C3F84003FEF781F908BDA81C0020B3
:10DF380010B5FFF7A7F90A4C60B90A4B93F81831E6
:10DF4800022B02D1084BDB6A98470123C4F84033FF
:10DF5800002010BDD4F84003013818BF0120F8E7AD
:10DF6800A81C0020E0160020945A010838B5134C6C
:10DF780004F55A7006F0DCF804F5607006F0D8F87D
:10DF880004F5667006F0D4F804F5806006F0D0F861
:10DF980000F0B5FF0A4B0025DB6A9847C4F84053E8
:10DFA800FEF7B6FD0749084840F2C45203F09CFD4D
:10DFB8000123C4F84033284638BD00BFA81C002000
:10DFC800945A0108E01600201C11002070B52E4B51
:10DFD8008AB0054693F8DD008DF8090093F8DC0057
:10DFE8008DF80A0029489A6A90F8180403920026C6
:10DFF8008DF80B0004960C46002940D00692D3F801
:10E00800882007921A8F93F81A118DF8151052BAB2
:10E01800ADF8202093F87C2093F848308DF8243010
:10E0280003AB8DF822008DF8232000930DF10A022E
:10E038000DF10B030DF1090105A88DF8146000F02E
:10E04800DDFE9DF90900FEF713F9607004A801F0E0
:10E058002BF8B0B9049A0F2A0DD863789A420AD8D7
:10E068001544AB42A3EB02012CBF00200120217014
:10E07800C0000AB070BD002323700820F9E7032010
:10E08800F7E71320F5E700BFE0160020A81C0020E2
:10E098001FB50446002800F012810078412800F2DC
:10E0A8000881DFE810F0420048004D005200560099
:10E0B8005A005F0006010601060106010601060175
:10E0C8000601060166006A006E0079008000830080
:10E0D80086008B0089008D009100940097009A00BB
:10E0E8009D00A000AF00B300BB00B700BF00C20096
:10E0F800C600CF00CB00CD000601D3000601060103
:10E1080006010601060106010601060106010601CF
:10E1180006010601060106010601DB00DF00E30037
:10E12800E800EC00F000F400FD00674B93F81831AC
:10E13800237104B010BD644B93F83031237102E0B1
:10E14800606803F0B5FB0020F3E7606803F0F6FBB6
:10E15800F9E75D4B93F81A31F0E75B4BD3F8E03001
:10E168006360F0E7584B211D93F8300103F0FEFB84
:10E17800E9E7554B93F81931E0E7534B93F88C30A6
:10E18800DCE71C238DF808304F4B02A993F84800B0
:10E1980001F02CFD6060D6E74C4B043493E8030093
:10E1A80084E80300CFE74A4B0434F7E7494B0434CB
:10E1B800F4E7494B0434F1E71A23E3E71923E1E7CD
:10E1C800414B93F86830B9E73F4B5B6DC8E73E4B6E
:10E1D8009B6DC5E73C4BDB6DC2E73B4B1B6EBFE756
:10E1E800394B5B6EBCE702238DF80830364B02A929
:10E1F80093F87C2093F848008DF80A2001F0F6FC8B
:10E208002071A0E7304B93F8DD3097E72E4B93F859
:10E21800393093E72C4B93F8DC308FE72A4B93F88F
:10E2280038308BE7284BDB6C9AE7274B93F8503054
:10E2380084E7254BD3F88430636084E7224B8FE76B
:10E24800264B8DE7204BD3F8CC30F5E71E4BD3F89F
:10E258002C31636001F058FDA06074E71A4BD3F8C5
:10E2680090307DE7184B93F81F3167E7164BB3F8EA
:10E278008830A38067E7144BB3F88A30F9E7124B6C
:10E28800B3F8D030F5E7104BB3F8D230F1E70E4BC6
:10E2980093F848200AB1062A13D1B3F8A035E8E765
:10E2A800094B93F848200AB1062A0AD1D3F8A435B5
:10E2B80056E7204604B0BDE8104000F024BE032015
:10E2C80037E7182035E700BFE01600204C1700207C
:10E2D80094170020541700209C1700201C110020C0
:10E2E8007FB5044610B9032004B070BDA44DD5F81D
:10E2F80040339A0700F171820278412A00F26A825B
:10E30800DFE812F04200480056005C00600065003B
:10E318006A007700820088008E0094009A00A000AE
:10E32800A600AC00B6006802BB00DD00F0001701D3
:10E3380039012A0144014D015101550159015D017D
:10E348006802610173019B018901AD01B301BA0142
:10E35800BF01C40168022A026802680268026802F2
:10E368006802680268026802680268026802680255
:10E37800680268026802680236023B0240024502EF
:10E388004A024F0254025E020079FEF7C1F80028E3
:10E39800AAD105E00379022BA5D07A4A82F8303158
:10E3A80095F8913443F0200385F8913400209BE7D9
:10E3B800406803F06FFA0028F2D094E7406803F051
:10E3C800ADFAF8E76F4B027983F81A21E8E76D4B4D
:10E3D8004268C3F8E020E3E76A4E416896F83001E6
:10E3E80003F0BAFA00287FF47EAF6368C6F8E43019
:10E3F800D6E7416800293FF476AF002001F0EAF93A
:10E408000028CDD011206FE7416800293FF46BAF99
:10E418000120F3E7416800293FF465AF0820EDE7E4
:10E42800416800293FF45FAF0920E7E74168002908
:10E438003FF459AF0C20E1E7416800293FF453AF9E
:10E448000D20DBE7416800293FF44DAF0E20D5E7EA
:10E45800416800293FF447AF0F20CFE74A4C494BAA
:10E46800007983F81901A36D9847E36A984797E7FD
:10E47800444B027983F88C2092E7424E037A8DF858
:10E48800043096F8480096F87D308DF8053007225C
:10E4980001A901F0BEFB00283FF425AF636896F898
:10E4A80048000193002201A901F0B3FB00283FF4C2
:10E4B8001AAF6C36D4E9010186E8030070E7314EE3
:10E4C800037A8DF8043096F8480096F87D308DF878
:10E4D8000530072201A901F09CFB00283FF403AF97
:10E4E800B436E7E7274E037A8DF8043096F84800EB
:10E4F80096F87D308DF80530072201A901F089FBD7
:10E5080000283FF4F0AED4E9010106F1740383E872
:10E51800030096F81831022B7FF442AF96F8303199
:10E52800002B3FF43DAF184BDB6A9847FDF748FFD7
:10E5380036E7144E037A8DF8043096F8480096F8BA
:10E548007D308DF80530072201A901F062FB002813
:10E558003FF4C9AEBC36ADE74368029301238DF89A
:10E568000C30084B02A993F8480001F05FFB002823
:10E578007FF416AFB7E6436802930023EFE700BFC6
:10E58800A81C0020E0160020945A010803795A1E9E
:10E598000E2A3FF6A8AE934A82F8683000E7914BFE
:10E5A80042685A65FCE68F4B42689A65F8E68D4BDF
:10E5B8004268DA65F4E68B4B42681A66F0E6894BE6
:10E5C80042685A66ECE6874C037994F848008DF85F
:10E5D8000430062201A901F01CFB00283FF483AE99
:10E5E8009DF8043084F8DD30DAE67E4C03798DF846
:10E5F800043094F8480094F87C308DF806300522F1
:10E6080001A901F006FB00283FF46DAE9DF8043027
:10E6180084F83930C4E6734C037994F848008DF8CF
:10E6280004300A2201A901F0F4FA00283FF45BAE95
:10E638009DF8043084F8DC30B2E66A4C037994F82B
:10E6480048008DF80430092201A901F0E2FA0028F7
:10E658003FF449AE9DF8043084F83830A0E6614BA9
:10E668004268C3F89420DA649AE65E4B027983F82C
:10E67800982083F8502093E65A4B4268C3F88420C8
:10E688008EE6584B4268C3F8CC2089E6012B40F04F
:10E69800A480554C2421204603F03CFA636A984232
:10E6A80001D0172020E61C2104F1280003F032FADB
:10E6B800636C9842F5D14FF4807104F1480003F07F
:10E6C80029FAD4F848319842EBD1D42104F5A67040
:10E6D80003F020FAD4F820329842E2D1002104F560
:10E6E800097003F017FAD4F824329842D9D14FF4BC
:10E6F800607104F50A7003F00DFAD4F8A835984251
:10E70800CFD1142104F2AC5003F004FAD4F8C03588
:10E718009842C6D1334E2146304640F2C45203F0E7
:10E72800E3F9204640F2C452002103F0F1F995F8CC
:10E738001B3485F8E833736FC5F8EC3396F87D30F1
:10E7480085F8F83340F20123A5F8FA33274B96F8F9
:10E7580019019B6D984723E68379012B3FF6C3ADDA
:10E76800204B42684068C3F82C2100F0D1FE47E6F0
:10E778001C4B4268C3F8902012E61A4B027983F8C2
:10E788001F210DE6174B8288A3F8882008E6154B51
:10E798008288A3F88A2003E6124B8288A3F8D02047
:10E7A800FEE5104B8288A3F8D220F9E50D4B93F8CB
:10E7B80048200AB1062A12D1A288A3F8A025EFE5BD
:10E7C800084B93F848200AB1062A08D16268C3F8B2
:10E7D800A425E5E500F099FBD9E5012084E518209A
:10E7E80082E500BFE01600201C110020945A0108A1
:10E7F8002DE9F04387B00023ADF800300646002825
:10E8080000F0ED800361FEF73DFD20B101242046B4
:10E8180007B0BDE8F08300F073FD0028F6D100F0E2
:10E8280069FD014618B96F48142203F071F96E4D5D
:10E8380095F89134012243F0040385F8552485F8AE
:10E84800913433788DF804300021013B8DF8052090
:10E85800ADF806100C2B00F2BA80DFE803F007B819
:10E86800B8B87881B8B88FB8AC99A800D5F8407313
:10E8780017F02007CAD196F80480B8F1020F45D1E5
:10E88800DFF868815A4CFEF729F896F9051098F8D0
:10E8980048003A4601F017FA88F83900B37988F841
:10E8A8003830384607238DF80530FDF731FEFF2351
:10E8B80004F58670A5F80C31C5F8084185F804718F
:10E8C80003F03CF804F58A7002F0F2FF3846FDF7D1
:10E8D8008DFE044640B196F9051098F848000122CB
:10E8E80001F0F1F988F83900D5F894343361002C37
:10E8F80071D000F0FFFC002889D195F8913485F893
:10E908001A0460F3820385F8913480E7B8F1010FA7
:10E918004FF00204E8D1DFF8D4908DF8144099F84C
:10E92800480089F81D7102A901F06EF9337989F858
:10E9380030318DF805708DF80680FDF785FC95F867
:10E94800913443F0100385F891340024CCE7002279
:10E958006946022000F0F6FA0028F6D01324C3E72F
:10E96800244BB288DB6B96F90C10B0689847D5F841
:10E97800403343F00203C5F84033E6E702A90D200F
:10E9880000F060FB0028E0D0002269460D20E1E796
:10E99800164B93F81831D3B9347904F0070000F016
:10E9A800ADFA8DF80040012269461020D2E7002216
:10E9B80069461220CEE78DF8072000F090FA044649
:10E9C80038B900F089FA204600F08BFA8CE7022467
:10E9D8008AE7012488E701A800F0DEFB17E7032493
:10E9E80015E700BFFC200020A81C0020E01600202E
:10E9F800AA1C0020945A01082DE9F04F99B08046CE
:10EA0800059118B9032019B0BDE8F08F0023036100
:10EA1800FEF738FC0646002840F0AB8045460FCD8F
:10EA28000EAC0FC45A4C98F800A0B8F80C7098F9BE
:10EA38000EB0142204F58860314603F069F801220B
:10EA480084F84124534C94F83021022A35460BD1DE
:10EA580094F81821022A07D194F81E2122B9BAF194
:10EA6800010F38BF4FF0010ABAF1010F2DD0BAF1EA
:10EA7800030F2CD0BAF1000F35D102229DF83C309B
:10EA8800DDF84090029362F34715012694F87C1054
:10EA98008DF8321002220CA994F848008DF8302025
:10EAA80001F0A4F894F81A3194F830C194F81D11C3
:10EAB80040B20222002B6FD0BCF1010F65D10029B2
:10EAC80063D1002E6DD1104627E00422D6E700233B
:10EAD800DDF83C90BDF840709DF942B0029365F0B6
:10EAE8001F050126D2E74FF0000BD946CDF808B034
:10EAF800CCE74FF0010084F81A04DDE005F29A42F1
:10EB08000BA900F0DDFA002800F020811320049BF7
:10EB180033871F4B002283F81A241D4BD3F89434F3
:10EB2800C8F810306FE705F29A452A460BA900F09D
:10EB3800C7FA0028EAD10B9B84F82801C4F82C51A5
:10EB480084F8303102E1B9F1000F00F0FF80002AAB
:10EB580000F0FC804946E01C02F0C6FF94F837320A
:10EB680001332380F2E01220D1E70220CFE707200B
:10EB7800CFE7012047E7064B93F8912483F840A498
:10EB880042F0010283F89124C7E7EEB90220C4E7F6
:10EB9800A81C0020E0160020002E94D05845B8BFCD
:10EBA800584694F87C308DF82000052294F84800E7
:10EBB8008DF8223008A901F02CF800283FF422AF84
:10EBC8009DF8203084F83930694A6A4BD2F89804A5
:10EBD800D3F8904038B105F071FA664B84423CBFD7
:10EBE800002283F83A20198F1A8F93F83001049184
:10EBF800996A099152BA0028B9D093F81B0100B953
:10EC0800186393F81801ADF85820013893F87C2060
:10EC180093F81A411491D0F1000BD3F888108DF8AD
:10EC28005B204BEB000B93F8482093F83A0093F8DD
:10EC380068308DF85A3009AB00934F4B03904FF072
:10EC480001008DF84C0015918DF85C20A3F12F017F
:10EC5800A3F1300213A88DF84D4000F0CFF8039BC4
:10EC68004FEA0B1B4BEA431B00264BEA801B4BEA7F
:10EC7800C413B1453E4C039308BF37463A4649464C
:10EC880004F59C70CDE90A669B46268084F81A64D0
:10EC980002F02AFFE9B2A570C5F34215FAB2042DB5
:10ECA800344E039B84F837223FF423AF072D3FF4FB
:10ECB8004AAF022D7FF459AF304D84F80D1104206E
:10ECC800029984F80401FF2084F80C0184F82811C3
:10ECD80084F81431D6F8E410C4F8085105F59B738C
:10ECE8000AA8C4F8101184F83021C4F82C3100F0B7
:10ECF80017FC00287FF437AF0A9BA4F844040BA83C
:10ED0800A4F81631C4F84C3400F0CEF900287FF48A
:10ED1800FDAE0B9BD3B196F93900FDF7A9FA94F82B
:10ED28003732002B3FF4FFAE0B9B0F2B3FF6E6AEBE
:10ED380005F58B720BA90F2000F0C2F900287FF4AB
:10ED4800E5AE0B9B63F3030B84F814B10598FDF74C
:10ED58004DFC00287FF4DBAE099B86F83A00B362CD
:10ED680000F07EF900283FF406AF1320D1E600BF7B
:10ED7800A81C0020E016002048170020AA1C00202C
:10ED880037B50B4D8DF8040004460F2295F848005E
:10ED980001A900F03EFF40B1064A85F81C4192F8EF
:10EDA800913443F0200382F8913403B030BD00BFA2
:10EDB800E0160020A81C002010B5FFF7B9F804469B
:10EDC80088B90A4805F0B4F9094805F0B1F90948C5
:10EDD80005F0AEF900F093F8FDF780FD064BDB6A0D
:10EDE8009847204610BD0124FBE700BF10200020F3
:10EDF8002820002040200020945A01082DE9F04FD7
:10EE08008BB047780093149B90F90C8090F90D60B3
:10EE180090F80E908B464168196004469246002F80
:10EE280057D002238DF8103004A9C37B007C8DF8DD
:10EE3800123000F0DBFEB4F808C0618943B26068A4
:10EE4800984545466144B8BF1D46604534BF002714
:10EE58000127884209D30A218DF81010207C0193DC
:10EE680004A900F0C3FE019B46B2B4F808C060894B
:10EE780061680CEB400E714520D3A1EB0C01B1FB8E
:10EE8800F0FC00FB1C11C9B998450ADC237833B1A2
:10EE98000223207C8DF8243006A900F0B5FE4FF03F
:10EEA800010921238DF81030207CE37B8DF8115067
:10EEB80004A98DF8123000F099FE45B2009B8BF83A
:10EEC800005038468AF8006083F800900BB0BDE81F
:10EED800F08F4546F2E7704770477047704700204B
:10EEE8007047704770477047002070470020704790
:10EEF8000020704700207047002070477047704717
:10EF08007047022070470220704702207047704700
:10EF180000207047704770470020704700207047F6
:10EF2800704770477047000010B5054C4FF40372E6
:10EF38002046002102F0ECFD0020C4E9000010BDCD
:10EF4800682200202DE9F8438146174600293FD062
:10EF5800244B002503F1010C1A462801103312F83E
:10EF6800018FB8F1000F36D19A42F8D11E4E33689E
:10EF78000BB9C6F800C073680BB1C3F800C03318EA
:10EF8800002401359C6083F80C900D302B01BAB237
:10EF980006EB05153044F750C6F804C002F0A4FD8E
:10EFA800B9F1110F4FF0000398BF104C6B71D6F8F0
:10EFB800083298BF24FA09F403F1010398BF04F05A
:10EFC80001043B442C71C6F808324046BDE8F8837A
:10EFD8004FF00108F9E70135202DBBD14FF00208A9
:10EFE800F3E700BF6F2200206822002020070200FC
:10EFF80010B510B3124A1368984204D1036813601D
:10F00800002304E00B4613B119688842FAD151680D
:10F01800884208BF53600BB101681960D2F8083202
:10F028008168013B00245B1A04602146C2F808325B
:10F03800102202F06DFD204610BD0120FCE700BF44
:10F0480068220020054B1B6813B11A798242FAD155
:10F05800002B0B600CBF03200020704768220020A3
:10F0680010B5054B186800B910BD037B04680BB9CF
:10F07800FFF7BEFF2046F6E76822002038B5084BA8
:10F08800084C186800B938BD03790568112B05D8F4
:10F0980024FA03F3DB0701D5FFF7AAFF2846F1E7B7
:10F0A800682200202007020028B1044BD3F8083258
:10F0B8000360002070470120704700BF68220020CD
:10F0C8002DE9F04107460E4615463AB331B3144BC5
:10F0D8001C6800232CB93046FFF7E6FF0020BDE886
:10F0E800F081A268F91A0132914210D32279EA54C8
:10F0F800581C22895FFA80F8611D55FA80F002F0E9
:10F10800F3FCA368246898445FFA88F3E2E7204692
:10F118002468FFF76DFF002CF9D1DCE70120DEE75A
:10F12800682200200238C0B211289ABF014B185C2F
:10F1380000207047A753010830B50B4B93F82020E7
:10F148000446084672B100211C330578A54208D050
:10F1580001319842CDB20CBF04480430AA42F4D819
:10F16800002030BD1046FCE77424002080240020D5
:10F1780010B5084C00232060142204F10C00FF2174
:10F1880084F82030C4E9010002F0C2FC012384F8AD
:10F19800213010BD7424002010B50E4A92F82010BA
:10F1A800042915D8936804781C7044785C70C47876
:10F1B800807898700131DC7082F8201002F11C010F
:10F1C8008B4214BF043302F10C039360012010BD7D
:10F1D8000020FCE774240020094B93F8200068B154
:10F1E8005A6803F11C018A4200F1FF3014BF04324F
:10F1F80003F10C0283F820005A600120704700BF19
:10F208007424002010B5074B93F8202004460846C4
:10F2180032B15968FFF790FF10B101234470837031
:10F2280010BD00BF7424002008B5064B93F82020B9
:10F238002AB15968FFF780FF08B1407808BD01205E
:10F24800FCE700BF7424002030B50A4A92F8201069
:10F25800536882F8210061B1916801241C32DD787D
:10F26800587005B99C7093420CBF034B0433994204
:10F27800F5D130BD742400208024002008B5044B4B
:10F288005968FFF759FF003818BF012008BD00BFB3
:10F29800742400202DE9F3410422154E0446002170
:10F2A8000DEB020096F8208002F032FC0025EBB24C
:10F2B800984502D802B0BDE8F081736819782170CA
:10F2C8005A7862709F785FB1336820469B68984788
:10F2D800FFF782FF17B901A8FFF75EFF0135E6E7E0
:10F2E800DB788DF804108DF805208DF80730EFE7EE
:10F2F80074240020014B93F82000704774240020E8
:10F30800034B93F82000042894BF00200120704785
:10F31800742400201FB50024CDE90244C41F8DF8D1
:10F3280000408DF801100C0AADF80420090C120CED
:10F338008DF803108DF806208DF8073002461B0A59
:10F34800012168468DF802408DF8083002F04BFA2A
:10F35800002818BF0E2004B010BD2DE9F04188B078
:10F3680017460D460F9A064600284DD00024012165
:10F37800CDE904448DF810109DF838108DF815105B
:10F38800ADF81630190CCDE900441B0ECDE9024446
:10F398008DF81930ADF81A20130C120E07948DF859
:10F3A80018108DF81C308DF81D20E3B24FEA0318B1
:10F3B800002D5FFA88F803DC002008B0BDE8F08172
:10F3C800013310218DF81F303A466B460DEB0100D2
:10F3D80002F09FF90346C8B9102DAC46A8BF4FF0FC
:10F3E800100CDAB2624503F1010303DB103D2DB2C4
:10F3F8000134DAE708EB020020326A44315C12F883
:10F40800202C4A403254ECE70920D6E70E20D4E7F6
:10F418000138032815D8DFE800F002080C100A4B61
:10F428001B681B690B6000207047074B1B685B69F2
:10F43800F8E7054B1B689B69F4E7034B1B68DB691E
:10F44800F0E70520704700BF982400202DE9F0411F
:10F45800C4B00C464A9E17461D468046B8B3B1F55F
:10F46800807F36D84FF488720021684602F050FB3E
:10F47800492300934FF48073ADF804302B0C8DF8BA
:10F488000830330CADF80650ADF80A608DF80C3032
:10F4980022460023414604A82D0E360E8DF80E3064
:10F4A8008DF809508DF80D608DF80F4002F01CFBA7
:10F4B80004F110014B9A3B4689B2684602F013F9F1
:10F4C80010B1012818BF0E2044B0BDE8F081092012
:10F4D800FAE70D20F8E7000010B590B10A4C282291
:10F4E8000021206002F014FB2368084A1A600020FB
:10F4F8004FF0FF32C3E90302C3E90522C3E907223B
:10F5080010BD0820FCE700BF98240020000101017D
:10F51800024B1B6818600020704700BF9824002029
:10F5280030B1044B1B68DB6801330360002070476F
:10F53800092070479824002013B500230C46019336
:10F54800D2B101A9FFF764FF18B9019B591C02D178
:10F55800146002B010BD99B2611A002902DD0B4493
:10F568001360F6E702D113600720F2E71B0C1B04B7
:10F5780003F580332344F3E70920EAE728B1044B75
:10F588001B681C334362002070470920704700BF86
:10F598009824002013B50446D8B1114B1A689388F3
:10F5A80001339BB29380C38200F057FA98B904F1F3
:10F5B8001803009321680123132202F08BF860B925
:10F5C800204600F04AFA003818BF0120000102B0B6
:10F5D80010BD0920FBE71020F9E70E20F7E700BF70
:10F5E80098240020F0B5054687B01C463BB32F4E43
:10F5F8003368DB68834257D894F82020002A14BF68
:10F6080009220822834205D3204600F05AFA70B135
:10F6180010200AE0002301900093A36894F82810B2
:10F62800606AFFF79AFE0028EED007B0F0BD237994
:10F638002168B4F808C0A768043B9AB209B9092040
:10F64800F3E7B2F5807F2DD8ADF80EC08DF81730EE
:10F658004FEA174C04F12C033F0E8DF811700093FC
:10F668002F0C08234FF0490EADF80C008DF81470DC
:10F678008DF816002F0E0DEB0300CDF808E08DF87D
:10F6880010C0ADF812508DF8157002F023F808B1CB
:10F698000E20CAE7204600F014FA0028B8D13368D3
:10F6A800DD60C2E70D20C0E70620BEE798240020F1
:10F6B8002DE9FF410A9D80460F4616461C46002D3F
:10F6C8005AD0002303A910460393FFF7A1FE18B1EF
:10F6D800062004B0BDE8F081039B9C4201D80133A9
:10F6E800F6D1284600F05EF9002847D1264B1A7853
:10F6F800424503D01A79424542D10120AA68BA424C
:10F7080040D103EB8002EB6A92F801802979CDE9B8
:10F7180000430439927828683B4689B2FFF796FE81
:10F728000028D6D195F820300194002B4FF0010322
:10F73800009314BF4246082295F82810686A3B4691
:10F74800FFF70BFE0028C4D1013E032EC1D8DFE825
:10F7580006F002070B0F0D4B1B681C611C62B8E713
:10F768000A4B1B685C61F9E7084B1B689C61F5E76D
:10F77800064B1B68DC61ACE70920AAE70F20A8E765
:10F788000B20A6E70220A4E7A40800209824002064
:10F798001FB50A460B2A4FF00001CDE90011CDE94B
:10F7A800021107D00C2A13D00A2A0FD00A2005B05C
:10F7B8005DF804FB012802D120238DF8003068464B
:10F7C80002F011F8002818BF0E20F0E73023F4E704
:10F7D8000B21F4E738B5054602F000F8044678B97D
:10F7E8007DB9094B1B680B219878FFF7D1FF38B911
:10F7F8000C21FFF7CDFF18B90A21FFF7C9FF00B1A7
:10F808000E24204638BD00BF982400202DE9F0437F
:10F8180080468FB00C461746002A6BD0002969D065
:10F82800002529461D2206A8059504F093FE8DF8AB
:10F838001350344D2B680DF114099E88CDF80490AF
:10F848000DF1130302933B7900933B68324621463E
:10F85800404601F0E4FF00284ED138683A7949461D
:10F8680002F042F9384600F04FF8002846D13C7AB9
:10F87800FA79BB79240444EA02241C432B689A6869
:10F8880094423DD99C609DF813000B21FFF780FF3F
:10F89800034658BB0C21FFF77BFF034630BB0A2108
:10F8A800FFF776FF034608BB7B7ABA7AFF7A3F04F4
:10F8B80047EA02271F433A46334621460920FFF705
:10F8C80029FD034690B933463A4621460820FFF7FA
:10F8D80021FD034650B92A689DF813109170002144
:10F8E800D1604FF0FF31C2E90411916118460FB0A1
:10F8F800BDE8F0830923F9E70E23F7E70F23F5E7BF
:10F908000323F3E79824002010B50446002845D0C7
:10F918000168002942D011F8013B437103220630E7
:10F9280002F0E2F82046032250F8091B043102F0E5
:10F93800DBF82168CB79E3600A7A43EA0223E360C3
:10F948004A7A43EA0243E3608A7A43EA0263E3605D
:10F95800CB7A23740B7B63742379212B1AD1102261
:10F968000D3104F1120002F0BFF81D222168501C6D
:10F978008B5C6362085C43EA0023901C6362085C4A
:10F98800033243EA004363628A5C43EA02636362C8
:10F99800002010BD112B03DC0D22E7E70220F8E759
:10F9A8000120F6E710B50446002854D00168002964
:10F9B80051D00B7843714B7883608A7843EA0223ED
:10F9C8008360CA7843EA024383600A7943EA0263A0
:10F9D80083604B7903738B79C381CA7943EA022325
:10F9E800027BC38102F00F020831103002F07CF86C
:10F9F800237B002203F00F0384F8202084F82820BA
:10FA0800227903F10800111A04290DDD2168093350
:10FA1800043AD21A085C84F82000D2B2606A84F8EA
:10FA28002820194402F060F8237922681A4400203B
:10FA380012F8043CE36212F8031C43EA0123E36270
:10FA480012F8021C43EA0143E36212F8012C43EA6C
:10FA58000263E36210BD0220FCE710B5044660B300
:10FA6800036853B30279162A29D942791A700146D4
:10FA7800082251F8060B013002F040F8214608220E
:10FA880051F80E0B093002F039F82368E28A5A74EB
:10FA9800E38A22681B0A93742368A269DA74A3694B
:10FAA80022681B0A13752368628B5A752368E27EE5
:10FAB8009A7517232371002010BD0120FCE702204E
:10FAC800FAE738B50446002863D00168002960D0F9
:10FAD800037B90F8282003F00F03002A57D108333E
:10FAE800207904321344984255D363790B70236804
:10FAF800A2685A70A36822681B0A937023686289F7
:10FB0800DA702368E27A1A712368227B5A712368B3
:10FB1800E2899A71E38922681B0A2146D371227B04
:10FB280051F8100B02F00F02083001F0DDFF237BC3
:10FB380094F8282003F00F0303F108052AB122687E
:10FB480094F82010515503F10905206894F82820ED
:10FB5800616A284401F0C8FF94F828302268E16AF5
:10FB68002B44D1545A1CE16A206892B2090A815484
:10FB78009A1C2168E08D92B28854DA1C216894F8A6
:10FB88002F0092B2043388542371002038BD093302
:10FB9800A6E70120FAE70220F8E70000024B1A88DE
:10FBA80010431880704700BF9C24002008B5074BFD
:10FBB8001B883BB1FEF7BCF900280CBF00206FF092
:10FBC800020008BD6FF00100FBE700BF9C24002085
:10FBD80010B5034B00241C80FEF7A0F9204610BD89
:10FBE8009C240020B0FA80F04009704782B018B910
:10FBF800084602B000F0CAB8002002B0704710B939
:10FC0800084600F077B9704710B9084600F08EB979
:10FC180070470346084611460BB900F0E5B90020C5
:10FC2800704710B9084600F071BD704710B9084612
:10FC380000F006BA0020704710B404460846114682
:10FC48001A46019B14B910BC00F018BA10BC7047D2
:10FC58000346084611460BB900F042BA0020704727
:10FC680010B40446084611461A4614B910BC00F0F0
:10FC7800AFBA002010BC704730B40546084611469C
:10FC88001A46DDE902341DB9029430BC00F02EBBDF
:10FC9800002030BC704710B9084600F0DFBB0020D8
:10FCA800704710B9084600F06FBD0020704710B9C2
:10FCB800084600F0EEBB0020704710B9084600F077
:10FCC800EBBB002070470346084611460BB900F00D
:10FCD80005BC0020704710B40446084611461A4671
:10FCE800019B14B910BC00F0FBBB092010BC704785
:10FCF80010B40446084611461A4614B910BC00F060
:10FD080063BDC8B210BC70470048704701000102CB
:10FD1800064B10B51B6A0446984730B10448054B9A
:10FD2800204498428CBF0020012010BD945A01083D
:10FD380040C220C980B92A00F0B5114B85B00C46E5
:10FD480010491F56054601F049F80F4BE4B25E6AA8
:10FD5800072D4FF00103CDE9024301460AD10522E0
:10FD68000023CDE900234FF47A727A431846B0474E
:10FD780005B0F0BD08220020CDE900203A46F5E79D
:10FD8800E3530108BC530108945A01081FB5002326
:10FD980000930378013B372B21D8DFE803F01C24BC
:10FDA8002020201E202020204143454E2055585B0E
:10FDB8005E6164206C1E6E73787A20207D81262017
:10FDC80020202020202020202020202083858A20F9
:10FDD80020838A208C90C3780BB10223009300986B
:10FDE80005B05DF804FB8378F6E743788DF80430B6
:10FDF80005238DF805308378003B18BF01235B008D
:10FE08008DF8063010238DF80730304B1B6801A899
:10FE180003F55872CDE9022300F0C0FF0090DEE739
:10FE28004023DBE72023D9E7827890F9013012B923
:10FE3800274AD35CD2E7274AFBE7827890F901305A
:10FE4800002AF8D1244AF4E740F6B833C6E74FF45D
:10FE58007A73C3E74FF4FA63C0E741F28833BDE72A
:10FE680041F27073BAE71D484FF47A7101F020FE31
:10FE780000F5FA60D2E71A4BB0E7144B1B6803F59C
:10FE88005873ABE7114B1B6803F55B73A6E71023A8
:10FE9800A4E70E4B1B68A1E74FF0834300939EE74E
:10FEA800104BFBE7104B99E740F21113ADF8003007
:10FEB80095E7032392E790F901300C4AB9E70C491A
:10FEC80090F9010000F08AFFA8E700BFA4240020F1
:10FED8006B540108735401087B54010818FCFFFF98
:10FEE80000EA06379A99094040F70937E3530108B1
:10FEF800BC53010837B50B4B02781B680C2101FB7A
:10FF080002335B7A03EB4304074B1D6803690093D4
:10FF1800C3684278816805EBC40000F0DFFC03B0D9
:10FF280030BD00BFA4240020A024002070B586B0F6
:10FF3800027B6423ADF80030012A4FF00003CDE9BD
:10FF48000133CDE903338DF802308DF8143030D009
:10FF5800022A39D05ABB03684BB343683BB31F4DE1
:10FF680080682B601E4B18226946186001F0BCFDA2
:10FF78001C4B2C6893E807000C3384E8070093E8CF
:10FF8800070004F10C06032386E80700A4F86C3385
:10FF9800012204F55B7104F5587000F090FC2B68A1
:10FFA8004FF6B072A3F878230522C3F87C2306B075
:10FFB80070BD0A4908684360036100F55B7100F58C
:10FFC800587000F07CFCF2E7044B1B68B3F8602320
:10FFD800B3F86C130A43A3F86023E8E7A4240020CD
:10FFE800A02400204847010808B503460A2924D858
:08FFF800DFE801F006232323DA
:020000040801F1
:10000000230B161B23212100BDE808400068FFF7E1
:1000100083BE90F900009978052271B900F013FCB5
:10002000003818BF012008BD052293F90000002107
:10003000F4E790F900005978EEE70221EEE7072295
:10004000F3E70020EFE7000010B504791CB1012CA4
:100050000BD0002010BD0A4B01681B68012203F57C
:10006000587000F030FC0120F4E7054B01681B6874
:10007000224603F55B7000F026FC2046EAE700BF4D
:10008000A4240020F7B50528144D1C46A8BF052060
:1000900058700E462946174600F0A4FE94F9013028
:1000A000A070072B13D1322000F09CFD0C4BDB6DB0
:1000B0000546984704F10C02083403460192009467
:1000C0003A463146284600F092FD03B0F0BD054A9D
:1000D00055F82310D05C00F07DFDE7E7BC53010824
:1000E000945A0108E35301082DE9F04F344F90F979
:1000F00001607B68D0F804908BB00446884698472E
:100100000546002859D1E37C73B92E4A237812683A
:1001100003EB4303990002EB8303D3F80490B9F196
:10012000000F01D152F80190274B484613F906B051
:10013000FB689847A37CD7F818A022890993072E5B
:1001400028D100230121CDE90223204A0693CDE9DD
:100150000431CDE907330521CDE900214FF47A724E
:1001600002FB0BF24CF250311846D047637C13B3BC
:10017000174B995D7B6D0D31C9B228469847E07CDD
:100180003246494600F040FE88F8006001200BB07E
:10019000BDE8F08F002101250823CDE90013CDE94A
:1001A0000715CDE90511CDE903110292A1782B467F
:1001B0005A462846D9E7074BDBE70020E7E700BFB0
:1001C000945A0108A4240020E35301088545010046
:1001D0007B5401086B5401082DE9F04F8DB090F964
:1001E0000130DFF8FCA0DFF8FC90CDE90A123E4AAE
:1001F00012F903B00278DAF800300C2505FB02335F
:100200003A4A5B7A126803EB430302EBC3030446EA
:1002100093F9021090F9020000F0DFFD3449064620
:1002200094F9010000F0DEFDA26861688046304666
:1002300000F005FD2178DAF80020D9F80C30694388
:10024000074650589847D9F81C309C4694F901301D
:100250000025072B4FF47A63CDE90753CDE9055507
:100260002DD10123CDE903530523CDE901534FF4EB
:100270007A7303FB0BF300933946434646F2A81208
:1002800028466746B8472378DAF800200C214B430C
:1002900094F90110D05800F0D9FDA18994F901001A
:1002A000FFF74EFD0B9B217B1860D9F85430284690
:1002B00098470A9B01201E700DB0BDE8F08F012009
:1002C0000823CDE90350CDE901032A46CDF800B05B
:1002D000654643463946A84701200546D3E700BF97
:1002E000A4240020945A0108E3530108A02400200C
:1002F000BC5301082DE9F04F8FB0002405468A4613
:10030000914698460494ADF81440ADF80240072693
:100310004FF0010B2B7AA34206D9686804A9204448
:1003200000F0F2FB00285ED102238DF8083002A80D
:100330006B7A8DF80A30FFF72DFDAB7A8DF81D3002
:100340009DF811308DF81E309DF812308DF81F3059
:100350009DF810308DF82030EB7A8DF821302B7B12
:100360008DF822306B7B8DF8233010238DF81C60C4
:100370008DF824303A4E8DF82C000DF102030A93CB
:1003800005238DF82D3033680C930723ADF83430F6
:100390002B6806930DF1120204AB0DF1110106A8B2
:1003A00000F0CCFB072805460BD130680C22002159
:1003B00000F5587001F0B0FB3368BDF80220A3F8D7
:1003C00060239DF811308AF800309DF8123089F8CA
:1003D00000309DF8103088F80030189B28461C70BB
:1003E0000FB0BDE8F08F9DF81330BDF81470ADF874
:1003F00002702044C4B2F3B917B3194A002011683F
:10040000072602464FF00C0C062B1BD10CFB00FEFE
:1004100051F80EE0BEF1000F04D00BFA00F23A439F
:1004200097B2012201301028EED1002A3FF472AFBA
:10043000ADF802706EE75A1E042A01D9062BDCD0F3
:10044000062667E747FA00FE1EF0010FEAD00CFB14
:1004500000FE51F80EE0BEF1000F08BF0626E1E7EE
:10046000A424002038B505464068FFF755FC052256
:10047000841D002195F90000E4B200F0E4F908B908
:1004800004F0FD0495F901000722002100F0DBF9DA
:1004900008B904F0FB04204638BD00207047000076
:1004A00010B503780F2B044618D84068FFF734FCCA
:1004B00022780B4902EB42020968831C01EB82009F
:1004C00051F82220DBB21AB903F0FD0358B210BD77
:1004D000032B06BF626842600223F7E70020F6E7BD
:1004E000A4240020022070472DE9F04FDFF8388166
:1004F0000446D8F8000099B08946174600211E46E8
:100500000122032300F55870CDE90611CDE9081149
:100510008DF814108DF81510ADF8163000F0B5F9FF
:1005200038B9D8F80020B2F8603343F00303A2F8DA
:100530006033D8F80020637A8DF8283002F55871BE
:10054000CDE90B12394A94F9083012680D920DF179
:1005500016020F922268109262681192D4E9030188
:10056000A27A8DF8482001228DF8492013AA82E84A
:1005700003001025227DE18A8DF8293018468DF878
:100580005420ADF83850FFF7DBFB0AAB17930DF1A1
:100590001503169000933146019705AB06AA10A8E3
:1005A00000F0BCFB064698BB9DF81410204F0139A3
:1005B00001F082FA1F4B1B690393C4B24FF00C0B7E
:1005C00004F160036B44D8F8000013F848AC9DF8C0
:1005D00014300BFB0AFC01343946B4FBF3F203FB85
:1005E0001244D0F87C33B0F9782350F80C00DDF8D1
:1005F0000CC0E4B2E04728B189F800A0304619B039
:10060000BDE8F08F013D15F0FF05D9D10D26F5E7C6
:100610000C2801BFD8F80020B2F8603343F0030380
:10062000A2F86033EAE700BFA4240020A024002041
:10063000400D0300945A0108F8B50679012E0546CD
:1006400001D80620F8BD0F2E2BD80368187A40F386
:1006500003000522002140B200F0F5F82B680446A3
:10066000187A40F303100522002140B200F0EBF8A5
:10067000A8B1B4FA84F4640929680B7A086843F3D2
:10068000030243F3031352B25BB29A42C8BF012480
:10069000FFF742FB48B9002CD3D10420D2E7012454
:1006A000EAE70320CEE70520CCE7002CFBD10C4F76
:1006B00029683B6806EB460003EB80000C2201F042
:1006C00017FA3A680C2303FB062320465C72B2F843
:1006D00060130123B3400B43A2F86033B2E700BFBD
:1006E000A424002010B4017801290ED9084B186801
:1006F0000C234B43C4180022C250C4E9012200F568
:10070000587010BC102200F0A7B8002010BC704731
:10071000A42400202DE9F04186B050238DF8143038
:10072000037A102B074630D14368DD7B6DBB022472
:10073000A8466426062C14D87A68535D03932A448D
:10074000517843EA01230393927843EA02437343C7
:10075000CDE9033863B968468DF80040FFF7C2FF62
:100760000DE0CDF80C808DF81480CDF81080F2E704
:1007700003AB01A801938DF80840FFF75DFF01343A
:10078000E4B2102C05F10305D4D106B0BDE8F08128
:100790001FB502680379116851B901A88DF80430BA
:1007A000FFF7A0FF78B9002040B205B05DF804FB68
:1007B00002A802928DF80C30FFF73EFF0628F2D80F
:1007C000024B185CF0E70320EEE700BFDC530108A2
:1007D000C90020B9034B0B449856C0B27047024B76
:1007E000F9E700BFEB5301082B540108F0B59A421A
:1007F000069D03DB9DF914309A4220DD0020F0BDF8
:1008000003EB430331F814C005EB830300264CFAD5
:1008100006F7FF0707D51F7A07F00F0E724502DBB8
:10082000B2EB171F0DDD0136102E03F10C03EED1D4
:100830000134E4B22301DBB29842E1D8DEE70024C0
:10084000F8E70120DBE7884204DB9042CCBF0020C0
:10085000012070470020704710B51409B4EB111F38
:1008600003464FEA11100ED391420CD202B201F0AE
:100870000F0133F81240012000FA01F124EA0101CE
:1008800023F8121010BD0020FCE7F0B528B100EBF2
:10089000410501270020914200D3F0BD002435F826
:1008A00002CB234607FA04F636EA0C0608BF0133EA
:1008B00004F1010408BFDBB2102CF3D1184401315C
:1008C000C0B2C9B2E7E710B500B149B910BD31F8FF
:1008D000134020F813400133DCB2A242F7D8F5E709
:1008E0000023F9E782B030B5048804936AB9B3F500
:1008F000616F18D349F6AF2542F21072AB4298BF30
:100900004FF47A72944238BF1446012C38BF012448
:100910006143BDE83040C3688B428CBF5B1A002343
:10092000C36002B070476422ECE700002DE9F04F8D
:1009300091B01546DDF86C8004939DF868300993FA
:100940000C46064603F0B4FB684ADFF8A4B10590F4
:10095000A8F5F633303BB3FBF2F3534303F5F6321D
:1009600003F5A83303F5C0730393182313FB054362
:1009700030320692089300254FF0FF3A089BA342BD
:1009800007D1002D14BF50464FF0FF3011B0BDE825
:10099000F08FBDF97030ADF82C300B99CDF86C802C
:1009A0004046CDF8288003F013FBB4F800906EB9F0
:1009B000B8F5616F5BD349F6AF2242F210739045F0
:1009C00098BF4FF47A73994538BF99464B46012B2F
:1009D00038BF01230793002E52D1B9F1640F48D1DB
:1009E000A0605F46A1680EA803F014FB0F9B009364
:1009F000DDE90A120E9B0CA803F06BFA049B0C9A1B
:100A00000BB9099B2BB12369BB4202D1394B9A42E6
:100A10000DD9394BE760984509D90023ADF834303A
:100A2000069B0D990C93184603F0D2FAA0606068FB
:100A300000B9E760276126B103F044FBE368034493
:100A4000E360D4E903329342059B1D996360079BE1
:100A500088BFE2604B43E168994202D20498A8B98A
:100A6000A6B101231D442375EDB2183486E7642333
:100A7000A9E7B9F57A7F0ABF204F214FA060B1E7FF
:100A8000049B0BB9C4F80CB05F46D0E7002093423A
:100A9000207506D85B1A9A4505F1010528BF9A46CC
:100AA000EDB2002EE1D1B9F1640F164AADF8346011
:100AB00019D049F6B023B9F57A7F18BF134690458F
:100AC00084BF039A9B180C931C9B00930CAF97E870
:100AD00006001B9B384603F0FCF997E8030003F07F
:100AE00077FA8246C1E74FF46163E8E7805101007D
:100AF00040771B007F5101002FEC010080A81201FC
:100B0000002E930230EC01000378032B14D14378BC
:100B100003F00F021B098A704B7083788B80C278B8
:100B200043EA02238B800379C3F3021203F00F031D
:100B3000CA700B7005207047002070472DE9F347FD
:100B400098464379057990F907609146044690F9F3
:100B500006208A4683B190F9087075B30F2A12D126
:100B600094F909200F2E1ED194F90A60072D24D183
:100B7000002F08BF012720E090F90B7090F90920A1
:100B800090F90A60E9E7A369019394F9153000939D
:100B9000216994F91430207BFFF728FE0028E1D169
:100BA00005F0FD05DEE794F91D30B3420FDC94F942
:100BB0001C30B342DADA05F0FB0528468AF800203B
:100BC00089F8006088F8007002B0BDE8F0871E4622
:100BD000CCE70000024B03FA00F0B0FBF1F07047E5
:100BE00040420F004FF4FA53B3FBF0F0704730B5BA
:100BF0004FF47A750C1F6A4300FB042252001EBF9B
:100C000000F1FF341219B2FBF0F2914238BF1146E5
:100C1000039A1160820048431CBF013040084FF422
:100C20007A71121A01FB1323002BCABF03F2E733B8
:100C300093FBF1F1B3FBF1F1049B196030BD38B5C2
:100C4000400014460D46F0F7E5FE01462846F0F751
:100C50002FFE2146F0F72CFEF0F71EFD03F0CCFC32
:100C6000F0F7FAFD40B238BD2DE9F74F01930023AC
:100C70001F469C461C01058A5FFA84FE04F0F004BE
:100C8000A54206D8019B82F800C01F7003B0BDE8E2
:100C9000F08F0EEB4E054FEA4309AD000024466885
:100CA00036F809602641F60727D5866806EB050A5F
:100CB000765916B3067836B9466926B136F8096012
:100CC0002641F60719D59AF8086090F901B046F365
:100CD00003084FFA88F8D8450FDC46F3031676B2BE
:100CE0005E450ADB9AF8096006EB4608C66806EB23
:100CF000C806367D4EB90137FFB20134102C05F11C
:100D00000C05CCD10133DBB2B4E70CF101060EEBDC
:100D1000040801F80C805FFA86FCEEE72DE9FF4736
:100D200004464068DDE90C671D468A46914603F09B
:100D3000C9F923681B1A3B604FF000080123337088
:100D400085F80080636813B12368834224D8CAF809
:100D50000080D4F81CC0A3699CF800E00393D4E998
:100D6000030101AB83E80300237D0093DCF80C1042
:100D7000237A627A7046FFF7D9FD334638602A46F7
:100D8000E0694946FFF770FF2B782BB1C7F8008068
:100D9000002004B0BDE8F0873378002B14BF0B208F
:100DA0000C20F6E737B590F9002090F902509542F3
:100DB00004460FD0013A52B295420BD0A36801937A
:100DC00094F9013000936168E0782B46FFF70EFD3F
:100DD0000028EFD0104603B030BD8842B8BF0846A7
:100DE0007047000051F82000054B984205D0054B94
:100DF000C31A58425841400070470120704700BF55
:100E000090D0030020A1070005281FB50ED80C4B79
:100E100053F820300093CDE901120A4B0122002142
:100E2000022002F05BFE05B05DF804FBCDE9001284
:100E3000054B01220021022002F050FEF3E700BF23
:100E4000EC54010883540108A254010807B5054B6E
:100E5000CDE9000101220021022002F03FFE03B093
:100E60005DF804FBBE54010810B5102204460021B1
:100E7000F13000F051FE0021C4F814112046F02298
:100E8000BDE8104000F048BE02460846102100F0C0
:100E9000A5B92DE9F0430446D0F8140185B00E46FB
:100EA000154604F2011988B3C0F110089045474671
:100EB00028BF1746BAB2484400F01AFED4F81431DD
:100EC0003B440F2BC4F814312DD9A8452BD204F183
:100ED000F00304F5807113F8012F187C8B4282EA2D
:100EE00000021A70F7D104F1F10810224146684659
:100EF00000F0FEFD22466946684600F0E9F910223E
:100F00006946404600F0F4FD3E44ED1B04F5807850
:100F100004F1F107102D09D8AAB23146484600F075
:100F2000E7FDC4F8145105B0BDE8F08304F1F00307
:100F3000711E13F8012F11F8010F434582EA0002D8
:100F40001A70F6D110223946684600F0D1FD2246CB
:100F50006946684600F0BCF910226946384600F040
:100F6000C7FD1036103DD5E7F0B589B00C4610220C
:100F700000210546684600F0CFFD224669466846D6
:100F800000F0A6F99DF90030002B6A464FF00001F1
:100F900043DA137812F8010F01315B0043EAD013F2
:100FA0000F2902F8013CF4D19DF80F305B0083F06B
:100FB0008703D4F81401DBB210288DF80F303BD131
:100FC00004F58073694604F5887013F8016F11F811
:100FD000012B984282EA06021A70F6D104F1F0035E
:100FE00004F5807113F8012F187C8B4282EA00020D
:100FF0001A70F7D110220DEB020004F1F10100F09C
:1010000077FD2246294604A800F062F9102200214B
:10101000684600F081FD09B0F0BD137812F8010FA9
:1010200001315B0043EAD0130F2902F8013CF4D1EF
:101030009DF80F305B00BCE79DF90030002B6A463D
:101040004FF0000137DA137812F8016F01315B00BD
:1010500043EAD6130F2902F8013CF4D19DF80F3072
:101060005B0083F08703471CDBB28DF80F30102F35
:1010700004EB0003C0F10F064FF0800288BF00268A
:1010800000F5817083F801210021324620443E445E
:1010900003F064FAC4F8146104F58073694604F53A
:1010A000887013F8016F11F8012B984282EA06024A
:1010B0001A70F6D192E7137812F8016F01315B00D4
:1010C00043EAD6130F2902F8013CF4D19DF80F3002
:1010D0005B00C8E70A780378534003704A78437886
:1010E000534043708A78837853408370CA78C378BA
:1010F0005340C3700A790379534003714A794379A5
:10110000534043718A79837953408371CA79C37993
:101110005340C3710A7A037A534003724A7A437A7E
:10112000534043728A7A837A53408372CA7AC37A6D
:101130005340C3720A7B037B534003734A7B437B58
:10114000534043738A7B837B53408373CA7BC37B47
:101150005340C373704710B50B7814786340037025
:1011600054784B786340437094788B7863408370F5
:10117000D478CB786340C37014790B7963400371E2
:1011800054794B796340437194798B7963408371CF
:10119000D479CB796340C371147A0B7A63400372BC
:1011A000547A4B7A634043728B7A947A63408372A9
:1011B000D47ACB7A6340C372147B0B7B6340037396
:1011C000547B4B7B63404373947B8B7B6340837383
:1011D000CB7BD27B5340C37310BD0000A1F1100341
:1011E000DBB2102B2DE9F04704D8374C24FA03F377
:1011F000DB0705D4002382F8F030FF20BDE8F0873C
:10120000531E4418A0424ED101F11C039B005FFA0B
:1012100083F9C3F30313013B2C4D82F8F030012412
:101220000B46D618B3FBF1F001FB103010F0FF00B5
:1012300016F804AC16F803EC16F802CC16F8017C8C
:1012400036D115F80E8015F80CE015F807C015F822
:101250000A70E00900EB400084EA080800EBC000D7
:101260006400C0B2E4B24440C246581AC0B212F898
:1012700000808AEA080A02F803A01044043390F8B8
:1012800001808EEA080E86F801E090F802E08CEA10
:101290000E0C86F802C0C078DBB247409945F77063
:1012A000BFD80020AAE710F8015B03F8015FA9E7A7
:1012B0001829DAD9102801BF15F80AA015F80EE090
:1012C00015F80CC0EF5DD0E70101010004570108DB
:1012D0002DE9F04FA3B092F8F0301D911B920193CD
:1012E000002B00F0538101461EA8FFF734FF1B9B23
:1012F000A74CA84DA84E10330293002303939DF8EA
:101300007C0004909DF886000590205C06909DF876
:101310007B000790205C089004989DF881C0205CB9
:10132000099014F80C000A909DF880000B909DF82D
:1013300085009DF878809DF87DE09DF882A09DF85D
:1013400087900C909DF87A00029B1C9314F80A2059
:1013500014F8093014F8081014F80E700D90205C81
:101360000E909DF87F000F90205C10900B98205CF1
:1013700011900C98205C12909DF8840013909DF8B9
:10138000790014909DF87E001590205C16909DF8D1
:1013900083001790205C18901398205C1990149883
:1013A000205C1A900398013003900298DDF804B095
:1013B000103002909DF80C00834536D88DF87810D7
:1013C0008DF87A2009990E9A8DF87C108DF882207C
:1013D0001199069A8DF880108DF87E201999169A29
:1013E0008DF884108DF886200A99189A8DF87D1052
:1013F0008DF887201299109A8DF87B301B9B8DF801
:1014000081108DF883201A99089A1D988DF88510FF
:101410008DF87F201EA903EB0B128DF87970FFF772
:101420009AFE002023B0BDE8F08F15F808B082EADC
:1014300003008BEA000016F80EB080EA0B008DF86E
:10144000780015F80E004B40434016F80A00434060
:101450008DF8793081EA070315F80A10594016F81B
:101460000930594016F808308DF87A107A40534008
:1014700015F8092053408DF87B30089A069B53409D
:10148000049AAA5C534016F80C2053408DF87C3027
:10149000DDE908325A4015F80C305340059AB25C29
:1014A00053408DF87D30DDE909325A40059BEB5CF5
:1014B0005340079AB25C53408DF87E30069B0A9ADF
:1014C0005340049AB25C5A40079BEB5C5A408DF83B
:1014D0007F200E9B109A53400B9AAA5C53400C9AA3
:1014E000B25C53408DF88030DDE910325A400C9BDD
:1014F000EB5C53400D9AB25C53408DF88130DDE9CE
:1015000011325A400D9BEB5C53400F9AB25C534032
:101510008DF88230129A0E9B53400B9AB25C5A405F
:101520000F9BEB5C1C995A408DF88320169B189AF0
:101530005340139AAA5C5340149AB25C53408DF8FE
:101540008430DDE918325A40149BEB5C5340159A05
:10155000B25C53408DF88530DDE919325A40159B55
:10156000EB5C5340179AB25C53408DF886301A9A60
:10157000169B5340139AB25C5340179AAA5C1EA85C
:1015800053408DF88730FFF7A5FDB8E6FF2049E707
:1015900004570108045501080456010808B538B17C
:1015A000044A05491060D82200F0A2FA002008BDC4
:1015B0000220FCE7A8240020345C01080A4B1A68CA
:1015C00070B5002302F1180503EB03142E5D86426B
:1015D00004D1183422440A60002070BD01330B2B63
:1015E000F2D10320F9E700BFA82400202DE9F04143
:1015F000CCB00646DDF8488117461C460D4631B38F
:10160000B8F1000F23D006A8FFF72EFC204601A951
:10161000FFF7D4FF0446B0B9019906A80131FFF7DE
:1016200033FC26B11022314606A8FFF732FC3A46B9
:10163000294606A8FFF72DFC06A902A8FFF794FC8F
:10164000029BC8F8003020464CB0BDE8F08102246F
:10165000F9E7000030B595B013A90446FFF7AEFFD7
:10166000002830D11B490C2303FB00F2555CA54236
:101670002BD1139B187C1090D87B0F90987B0E90E9
:10168000587B0D90187B0C90D87A0B90987A0A9022
:10169000587A0990187A0890D87907909879069026
:1016A0005879059018790490D8780390987802902A
:1016B0000A445B780193936800930022064B11461D
:1016C000022002F00BFA15B030BD01300B28CBD14F
:1016D000F9E700BF7C590108045801080B2B10B42E
:1016E00002D810BCFFF782BF032010BC704730B592
:1016F0000D4685B01446014668B103AA0020009249
:101700002A460390FFF772FF18B90398001B18BF11
:10171000012005B030BD0220FBE72DE9F0430D4666
:10172000BFB014469946804620B31BB311F00F0199
:1017300022D1F02201A800F0EFF920466946FFF718
:101740003DFF044648B9009801AA10210130FFF777
:1017500045FD2E46AF1BFFB21EB920463FB0BDE887
:10176000F08301AA09EB070108EB0700FFF7B0FDC2
:10177000103EEFE70224F0E70524EEE7F0B5184E3F
:101780003468024685B00846002304F1180103EBD3
:1017900003154F5D97421ED10D2A05F1190513D18E
:1017A0000023CDE90033CDE902330C2210216B4632
:1017B000FFF7B3FF0446306810226946284400F062
:1017C00097F9204605B0F0BD01461022601900F0DF
:1017D0008FF90024F5E701330B2BD8D10324F0E770
:1017E000A824002009B1FFF7C9BF022070471FB528
:1017F0001446A0B10C2A01D10B2912D10023CDE946
:101800000033CDE902330A466B461021FFF785FF0E
:1018100018B969462046FFF7B1FF04B010BD022099
:10182000FBE70320F9E7F8B51E46DDE907479DF819
:1018300018505BB354B34FB3212D29D819462A460B
:10184000204600F055F90122631C691EB018FFF70D
:1018500064FFF8B9E37ADB093B70EBB96319204602
:1018600013F8012C13F8021C120642EA014213F885
:10187000041C0A4313F8031C012342EA0122291F16
:10188000FFF735FF003818BF0120F8BD0220FCE744
:101890000520FAE70720F8E70420F6E708B5014637
:1018A00030B1044B0822186800F022F9002008BD6E
:1018B0000220FCE7A824002008B530B1044B082220
:1018C000196800F015F9002008BD0220FCE700BFF0
:1018D000A82400207FB5124E0023044602A80193DD
:1018E0000D46FFF7E9FF33685B6901936CB102AA0B
:1018F000082312F8011B41B9013B13F0FF03F8D193
:1019000002A8A04702A8FFF7C9FF35B1019B23B980
:1019100001A8A8473368019A5A61002004B070BD3D
:10192000A824002008B5014638B1054B18680822E4
:10193000104400F0DDF8002008BD0220FCE700BFE5
:10194000A824002008B538B1044B196808221144B6
:1019500000F0CEF8002008BD0220FCE7A8240020FB
:10196000034B1B6802280CBF1961596100207047A6
:10197000A824002041B1054B1B6802280CBF1B693D
:101980005B690B600020704702207047A82400208C
:1019900030B58FB0002405460CA80994FFF78CFFE2
:1019A0009DF8373007939DF8363006939DF8353013
:1019B00005939DF8343004939DF8333003939DF8DC
:1019C000323002939DF8313001939DF8303000930E
:1019D000224621461E4B022002F080F80AA8FFF79B
:1019E000B1FF9DF82F3007939DF82E3006939DF898
:1019F0002D3005939DF82C3004939DF82B300393E4
:101A00009DF82A3002939DF8293001939DF82830E3
:101A1000009322460F4B2146022002F05FF809A9ED
:101A20002846FFF7A7FF9DF8243003939DF8253043
:101A300002939DF8263001939DF8273000932246AB
:101A4000054B2146022002F049F80FB030BD00BF1F
:101A5000605801089E580108DC58010808B50020AC
:101A6000FFF7F8FD0120FFF7F5FD0920FFF7F2FD74
:101A70000820FFF7EFFD0020FFF78AFF002008BDD8
:101A800010B504460B20FFF7E5FD0C20FFF7E2FD43
:101A90000920FFF7DFFD0820FFF7DCFD0A20FFF734
:101AA000D9FD2046FFF774FF002010BD014B1860E0
:101AB000704700BFAC0800200B4A30B514680B4DCE
:101AC00043F2390305FB04331360091A6FF0004237
:101AD000B3FBF2F2C2EBC27201319B1A93FBF1F23B
:101AE00001FB1233184430BDAC0800206D4EC641D6
:101AF00001380A44914200D1704711F8013B00F8C7
:101B0000013FF7E710440A44914200D1704711F8B1
:101B1000013B00F8013DF7E702F020BD30B530B1E0
:101B20000A4D01444FF0FF33814201D1D84330BD0B
:101B300010F8012B5340082243F30004013A2C40D3
:101B400092B284EA5303002AF6D1EDE72083B8ED80
:101B500001207047054B4FF400529A62044B1B68FA
:101B600013B15B6803B11847704700BF0004004819
:101B7000AC250020054B4FF480529A62044B1B6841
:101B800013B1DB6803B11847704700BF0004004879
:101B9000AC250020012070470120704701F048B9B2
:101BA00001F036B910B501F019FE0E21044640F6D9
:101BB0001F1001F02DF92046012101F0F9FDBDE8CB
:101BC000104001F0D7BA000070B50C4E01EB400395
:101BD0000D46B3654FF6FF71002304461A460846CA
:101BE00001F05EFB96F85600002101F0E1FD294668
:101BF0002046BDE8704001F095BA00BFC82500201E
